:020000040802F0
:10000000FFFF012049FA0208752F0208B52F0208E8
:10001000C52F0208C72F0208C92F020800000000E0
:10002000000000000000000000000000ED4C02088D
:10003000CB2F020800000000B54D0208F94D020860
:1000400099FA020899FA020899FA0208492D020859
:1000500099FA020899FA020899FA020899FA02082C
:1000600099FA020899FA020899FA020899FA02081C
:1000700099FA020899FA020899FA020899FA02080C
:1000800099FA020899FA020899FA020899FA0208FC
:1000900099FA020899FA020899FA020899FA0208EC
:1000A00099FA020899FA020899FA020899FA0208DC
:1000B00099FA020899FA020899FA020899FA0208CC
:1000C00099FA020899FA020899FA020899FA0208BC
:1000D00099FA020899FA020899FA020899FA0208AC
:1000E00099FA0208712D020899FA020899FA020891
:1000F00099FA020899FA020899FA020899FA02088C
:1001000099FA020899FA020899FA020899FA02087B
:1001100099FA020899FA020899FA020899FA02086B
:1001200099FA020899FA020899FA020899FA02085B
:1001300099FA0208CD2F020899FA020899FA0208E2
:1001400099FA020899FA020899FA020899FA02083B
:1001500099FA020899FA020899FA020899FA02082B
:1001600099FA020899FA020899FA020899FA02081B
:1001700099FA020899FA020899FA020899FA02080B
:0801800099FA020899FA02083D
:1001880008B540F2D040074BC2F200001B1A062BFC
:1001980000D808BD40F20003C0F20003002BF8D0DD
:1001A8009847F6E7D304002008B540F2D04040F263
:1001B800D043C2F20000C2F200031B1A9B1003EBEB
:1001C800D373591000D108BD40F20002C0F20002FA
:1001D800002AF8D09047F6E710B540F2D044C2F2B2
:1001E8000004237873B9FFF7CBFF40F20003C0F295
:1001F80000032BB147F25440C0F60300AFF3008070
:100208000123237010BD00BF08B540F20003C0F2FF
:1002180000034BB147F2544040F2D441C0F603000A
:10022800C2F20001AFF3008040F2D040C2F20000F9
:1002380003682BB140F20003C0F2000303B19847F2
:10024800BDE80840FFF7B0BF81F0004102E000BF01
:1002580083F0004330B54FEA41044FEA430594EA7E
:10026800050F08BF90EA020F1FBF54EA000C55EAB9
:10027800020C7FEA645C7FEA655C00F0E2804FEA8A
:100288005454D4EB5555B8BF6D420CDD2C4480EA6C
:10029800020281EA030382EA000083EA010180EA9C
:1002A800020281EA0303362D88BF30BD11F0004FEA
:1002B8004FEA01314FF4801C4CEA113102D0404220
:1002C80061EB410113F0004F4FEA03334CEA13335B
:1002D80002D0524263EB430394EA050F00F0A78073
:1002E800A4F10104D5F1200E0DDB02FA0EFC22FA6E
:1002F80005F2801841F1000103FA0EF2801843FA62
:1003080005F359410EE0A5F120050EF1200E012A52
:1003180003FA0EFC28BF4CF0020C43FA05F3C01890
:1003280051EBE37101F0004507D54FF0000EDCF109
:10033800000C7EEB00006EEB0101B1F5801F1BD3B2
:10034800B1F5001F0CD349085FEA30004FEA3C0CB6
:1003580004F101044FEA445212F5800F80F09A80AC
:10036800BCF1004F08BF5FEA500C50F1000041EBB0
:10037800045141EA050130BD5FEA4C0C404141EBB4
:10038800010111F4801FA4F10104E9D191F0000FDB
:1003980004BF01460020B1FA81F308BF2033A3F15E
:1003A8000B03B3F120020CDA0C3208DD02F1140C55
:1003B800C2F10C0201FA0CF021FA02F10CE002F190
:1003C8001402D8BFC2F1200C01FA02F120FA0CFC89
:1003D800DCBF41EA0C019040E41AA2BF01EB0451D2
:1003E800294330BD6FEA04041F3C1CDA0C340EDCD0
:1003F80004F11404C4F1200220FA04F001FA02F313
:1004080040EA030021FA04F345EA030130BDC4F1D0
:100418000C04C4F1200220FA02F001FA04F340EAC5
:100428000300294630BD21FA04F0294630BD94F076
:10043800000F83F4801306BF81F480110134013D5D
:100448004EE77FEA645C18BF7FEA655C29D094EACE
:10045800050F08BF90EA020F05D054EA000C04BF4C
:100468001946104630BD91EA030F1EBF0021002037
:1004780030BD5FEA545C05D14000494128BF41F0D6
:10048800004130BD14F580043CBF01F5801130BD3A
:1004980001F0004545F0FE4141F470014FF00000C5
:1004A80030BD7FEA645C1ABF194610467FEA655C76
:1004B8001CBF0B46024650EA013406BF52EA033518
:1004C80091EA030F41F4002130BD00BF90F0000F06
:1004D80004BF0021704730B54FF4806404F1320442
:1004E8004FF000054FF0000150E700BF90F0000FFB
:1004F80004BF0021704730B54FF4806404F1320422
:1005080010F0004548BF40424FF000013EE700BFF1
:1005180042004FEAE2014FEA31014FEA02701FBF81
:1005280012F07F4393F07F4F81F06051704792F053
:10053800000F14BF93F07F4F704730B54FF46074CD
:1005480001F0004521F0004120E700BF50EA010218
:1005580008BF704730B54FF000050AE050EA0102C5
:1005680008BF704730B511F0004502D5404261EB35
:1005780041014FF4806404F132045FEA915C3FF476
:10058800DCAE4FF003025FEADC0C18BF03325FEA0F
:10059800DC0C18BF033202EBDC02C2F1200300FAC4
:1005A80003FC20FA02F001FA03FE40EA0E0021FAE9
:1005B80002F11444C1E600BF70B54FF0FF0C4CF4D3
:1005C800E06C1CEA11541DBF1CEA135594EA0C0F89
:1005D80095EA0C0F00F0DEF82C4481EA030621EAC4
:1005E8004C5123EA4C5350EA013518BF52EA0335FF
:1005F80041F4801143F4801338D0A0FB02CE4FF0B1
:100608000005E1FB02E506F00042E0FB03E54FF0E0
:100618000006E1FB03569CF0000F18BF4EF0010ED8
:10062800A4F1FF04B6F5007F64F5407404D25FEAD4
:100638004E0E6D4146EB060642EAC62141EA555187
:100648004FEAC52040EA5E504FEACE2EB4F1FD0CC9
:1006580088BFBCF5E06F1ED8BEF1004F08BF5FEA47
:10066800500E50F1000041EB045170BD06F00046F9
:1006780046EA010140EA020081EA0301B4EB5C04A6
:10068800C2BFD4EB0C0541EA045170BD41F480119E
:100698004FF0000E013C00F3AB8014F1360FDEBFC3
:1006A800002001F0004170BDC4F10004203C35DA9F
:1006B8000C341BDC04F11404C4F1200500FA05F322
:1006C80020FA04F001FA05F240EA020001F00042C3
:1006D80021F0004110EBD37021FA04F642EB060139
:1006E8005EEA430E08BF20EAD37070BDC4F10C0463
:1006F800C4F1200500FA04F320FA05F001FA04F227
:1007080040EA020001F0004110EBD37041F1000112
:100718005EEA430E08BF20EAD37070BDC4F120051D
:1007280000FA05F24EEA020E20FA04F301FA05F285
:1007380043EA020321FA04F001F0004121FA04F22D
:1007480020EA020000EBD3705EEA430E08BF20EAFD
:10075800D37070BD94F0000F0FD101F00046400037
:1007680041EB010111F4801F08BF013CF7D041EAB9
:10077800060195F0000F18BF704703F000465200BD
:1007880043EB030313F4801F08BF013DF7D043EA8E
:100798000603704794EA0C0F0CEA135518BF95EA44
:1007A8000C0F0CD050EA410618BF52EA4306D1D1CB
:1007B80081EA030101F000414FF0000070BD50EAEA
:1007C800410606BF1046194652EA430619D094EA74
:1007D8000C0F02D150EA013613D195EA0C0F05D15E
:1007E80052EA03361CBF104619460AD181EA0301B2
:1007F80001F0004141F0FE4141F470014FF000006A
:1008080070BD41F0FE4141F4780170BD70B54FF004
:10081800FF0C4CF4E06C1CEA11541DBF1CEA135584
:1008280094EA0C0F95EA0C0F00F0A7F8A4EB050466
:1008380081EA030E52EA03354FEA013100F088805D
:100848004FEA03334FF0805545EA131343EA126326
:100858004FEA022245EA111545EA10654FEA0026DB
:100868000EF000419D4208BF964244F1FD0404F594
:10087800407402D25B084FEA3202B61A65EB0305F0
:100888005B084FEA32024FF480104FF4002CB6EBAD
:10089800020E75EB030E22BFB61A754640EA0C002D
:1008A8005B084FEA3202B6EB020E75EB030E22BF6D
:1008B800B61A754640EA5C005B084FEA3202B6EBAE
:1008C800020E75EB030E22BFB61A754640EA9C006D
:1008D8005B084FEA3202B6EB020E75EB030E22BF3D
:1008E800B61A754640EADC0055EA060E18D04FEAFB
:1008F800051545EA16754FEA06164FEAC30343EA9B
:1009080052734FEAC2025FEA1C1CC0D111F4801F67
:100918000BD141EA00014FF000004FF0004CB6E760
:1009280011F4801F04BF01430020B4F1FD0C88BFFF
:10093800BCF5E06F3FF6AFAEB5EB030C04BFB6EB0A
:10094800020C5FEA500C50F1000041EB045170BDFD
:100958000EF0004E4EEA113114EB5C04C2BFD4EB2A
:100968000C0541EA045170BD41F480114FF0000EAE
:10097800013C90E645EA060E8DE60CEA135594EA2A
:100988000C0F08BF95EA0C0F3FF43BAF94EA0C0F2D
:100998000AD150EA01347FF434AF95EA0C0F7FF4A2
:1009A80025AF104619462CE795EA0C0F06D152EAF6
:1009B80003353FF4FDAE1046194622E750EA4106DA
:1009C80018BF52EA43067FF4C5AE50EA41047FF4EB
:1009D8000DAF52EA43057FF4EBAE12E74FF0FF3C50
:1009E80006E000BF4FF0010C02E000BF4FF0010C21
:1009F8004DF804CD4FEA410C7FEA6C5C4FEA430C9A
:100A080018BF7FEA6C5C1BD001B050EA410C0CBFE8
:100A180052EA430C91EA030F02BF90EA020F00204A
:100A2800704710F1000F91EA030F58BF994208BFB1
:100A380090422CBFD8176FEAE37040F0010070476E
:100A48004FEA410C7FEA6C5C02D150EA013C07D1C5
:100A58004FEA430C7FEA6C5CD6D152EA033CD3D010
:100A68005DF8040B704700BF8446104662468C460A
:100A78001946634600E000BF01B5FFF7B7FF00283D
:100A880048BF10F1000F01BD4DF808EDFFF7F4FF66
:100A98000CBF012000205DF808FB00BF4DF808EDF1
:100AA800FFF7EAFF34BF012000205DF808FB00BF14
:100AB8004DF808EDFFF7E0FF94BF012000205DF836
:100AC80008FB00BF4DF808EDFFF7CEFF94BF0120EB
:100AD80000205DF808FB00BF4DF808EDFFF7C4FFE4
:100AE80034BF012000205DF808FB00BF4FEA410237
:100AF80012F5001215D211D56FF47873B3EB625268
:100B080012D94FEAC12343F0004343EA505311F08E
:100B1800004F23FA02F018BF404270474FF0000020
:100B2800704750EA013005D111F0004008BF6FF05E
:100B3800004070474FF00000704700BF4BB942B902
:100B4800002908BF002802D04FF0FF31084600F006
:100B58003BB882B0EC462DE9005000F01DF8DDF8F6
:100B680004E002B00CBC70472DE9F8439046994662
:100B780006460F4600F02AF8089BA8FB004508FB2C
:100B880001F800FB09825519341B67EB0505C3E919
:100B98000045BDE8F88300BF2DE9F04190460646C0
:100BA8000F461D4600F0C8F900FB05F3A0FB0845F9
:100BB80008FB0138069B4544341B67EB0505C3E970
:100BC8000045BDE8F08100BF704700BF2DE9F04F38
:100BD8000025002985B01C46C0F24981002CC0F2CE
:100BE80041818C460F468246914614460646194670
:100BF800002B4BD1624559D9B2FA82F343B1C3F104
:100C080020020CFA03F720FA02F29C4017439E4098
:100C18004FEA1448384641461FFA84F900F018FB99
:100C280041468246384600F041FC330C09FB0AF085
:100C380043EA014188420AD909190AF1FF3205D26B
:100C4800884284BFAAF1020A091900D89246C0EB6B
:100C5800010B41465846B6B200F0FAFA414607463B
:100C6800584600F023FC09FB07F946EA014189458B
:100C780007D97B1E0C1980F05781023FA14540F22D
:100C8800538147EA0A404FF0000804E0634558D909
:100C98004FF0000840460246434615B1524263EB06
:100CA80043031046194605B0BDE8F08F22B901206C
:100CB800114600F0CDFA0446B4FA84F3002B40F054
:100CC800DC803F1B4FEA14491FFA84FA4FF00108F1
:100CD8004946384600F0BCFA49468346384600F093
:100CE800E5FB330C0AFB0BF043EA014188420BD9C0
:100CF80009190BF1FF3380F01581884284BFABF1ED
:100D0800020B091940F20E810B1A49461846019345
:100D180000F09EFA019B4946B6B20746184600F015
:100D2800C5FB0AFB07FA46EA01418A4506D97B1E3C
:100D38000C1902D2023FA24500D81F4647EA0B40D1
:100D4800A9E7B3FA83F4002C00F0E480C4F120038F
:100D580001FA04F122FA03FA2CFA03FB4AEA010A1F
:100D680020FA03F80CFA04FC58464FEA1A4748EAF6
:100D78000C08394602FA04F9CDF80C9000F068FA2C
:100D880039468146584600F091FB1FFA8AFC4FEA23
:100D980018430CFB09F043EA014398420CD913EBC2
:100DA8000A0309F1FF3180F0C380984284BFA9F19A
:100DB8000209534440F2BC801B1A39461846CDF844
:100DC80008C0019300F044FA019B39461FFA88F8DD
:100DD8008346184600F06AFBDDF808C00CFB0BF3ED
:100DE80048EA01418B420CD911EB0A010BF1FF30A3
:100DF80080F09C808B4284BFABF1020B514440F2DF
:100E08009580039F4BEA0940C91A1FFA80FCBAB2C1
:100E18004FEA1749070C02FB0CF802FB07F209FB23
:100E28000C2309FB07F903EB18439A4288BF09F51D
:100E3800803909EB1349494510D31FFA88F814BFC4
:100E48000022012206FA04F408EB03439C422CBF5B
:100E5800002302F00103002B3FF415AF01384FF0D7
:100E6800000818E7524263EB4303ED43B9E64042FA
:100E780061EB41014FF0FF35B0E69C40C3F1200B18
:100E880027FA0BF807FA03F74FEA14494046494690
:100E980026FA0BFB9E4000F0DBF949461FFA84FA5C
:100EA8004BEA070B03464046019300F0FFFA019B0B
:100EB8004FEA1B420AFB03F042EA0141884206D985
:100EC8005A1E091936D2884234D9023B09190F1A19
:100ED80049463846019300F0BBF949461FFA8BFB97
:100EE8008046384600F0E2FA019B0AFB08F74BEA15
:100EF80001418F420AD9091908F1FF3205D28F4200
:100F080084BFA8F10208091900D89046CF1B48EA07
:100F18000348DDE60120634528BF5245A0467FF619
:100F2800BAAEB5E69B46EFE61F46AAE6834668E7F3
:100F3800894641E71346CAE72DE9F04F064683B0D4
:100F48000D46144607468846002B4AD18A4255D991
:100F5800B2FA82F34BB1C3F1200201FA03F820FA86
:100F680002F29C4042EA08089F40250C4046294668
:100F78001FFA84FA00F06CF929468146404600F0D1
:100F880095FA3B0C0AFB09F043EA014188420AD969
:100F9800091909F1FF3205D2884284BFA9F1020973
:100FA800091900D89146C0EB010829464046BFB24E
:100FB80000F04EF929460646404600F077FA0AFB4B
:100FC80006FA47EA01418A4507D9731E0C1980F0D1
:100FD8002281023EA24540F21E8146EA09400026CF
:100FE80058E08B4254D8B3FA83F4002C56D18B4284
:100FF80028BF82424CD8264601204BE022B9012066
:10100800114600F025F90446B4FA84F3002B40F0A9
:10101800B9802D1B4FEA14481FFA84FA012641466D
:10102800284600F015F941468146284600F03EFA68
:101038003B0C0AFB09F043EA014188420BD9091924
:1010480009F1FF3380F0E980884284BFA9F10209E1
:10105800091940F2E280C0EB010B41465846BFB285
:1010680000F0F6F841460546584600F01FFA0AFB1C
:1010780005FA47EA01418A4507D96B1E0C1980F029
:10108800CE80023DA24540F2CA8045EA094001E00F
:1010980000263046314603B0BDE8F08FC4F1200188
:1010A80003FA04F322FA01F825FA01F748EA0308DB
:1010B80020FA01F105FA04F538464FEA18490D43BC
:1010C800494602FA04F2019200F0C2F84946824603
:1010D800384600F0EBF91FFA88F22F0C02FB0AF0F1
:1010E80047EA0147B84206D917EB08070AF1FF316A
:1010F800C0F09F808A463F1A49463846009200F061
:10110800A7F84946ADB28346384600F0CFF9009AB1
:1011180002FB0BF745EA01418F4205D911EB0801A3
:101128000BF1FF327DD39346019B4BEA0A40C91B62
:101138004FEA104C9DB24FEA134A83B205FB03F203
:1011480005FB0CF50AFB03530AFB0CFA03EB1243ED
:101158009D4288BF0AF5803A0AEB134A51450ED3DF
:1011680092B214BF0021012106FA04F602EB0343F0
:101178009E422CBF002601F00106002E8AD00138BD
:10118800002687E79C40C3F1200225FA02FA26FAD6
:1011980002F94FEA14485046414605FA03F506FAA3
:1011A80003F700F055F8414649EA050983465046D9
:1011B80000F07CF91FFA84FA4FEA19430AFB0BF096
:1011C80043EA0141884209D909190BF1FF3338D2A2
:1011D800884284BFABF1020B091932D90D1A414676
:1011E80028461FFA89F900F033F841460646284692
:1011F80000F05CF90AFB06F549EA01418D4206D97F
:10120800731E09191FD28D421DD9023E09194D1BA3
:1012180046EA0B4603E71E46DFE699461BE71D46EE
:1012280033E78F4284BFABF1020B41443FF67CAFFA
:1012380079E7B84284BFAAF1020A47443FF65BAF98
:1012480058E79B46CAE71E46E1E700BF00000000DA
:101258004A1E08BF7047C0F02481884240F21681B8
:10126800114200F01781B0FA80F3B1FA81F2A2EBD3
:101278000303C3F11F0304A202EB03134FF00002A0
:101288009F4600BFAFF30080B0EBC17F00BF42EBC9
:10129800020228BFA0EBC170B0EB817F00BF42EB18
:1012A800020228BFA0EB8170B0EB417F00BF42EB88
:1012B800020228BFA0EB4170B0EB017F00BF42EBF8
:1012C800020228BFA0EB0170B0EBC16F00BF42EB78
:1012D800020228BFA0EBC160B0EB816F00BF42EBF8
:1012E800020228BFA0EB8160B0EB416F00BF42EB68
:1012F800020228BFA0EB4160B0EB016F00BF42EBD8
:10130800020228BFA0EB0160B0EBC15F00BF42EB57
:10131800020228BFA0EBC150B0EB815F00BF42EBD7
:10132800020228BFA0EB8150B0EB415F00BF42EB47
:10133800020228BFA0EB4150B0EB015F00BF42EBB7
:10134800020228BFA0EB0150B0EBC14F00BF42EB37
:10135800020228BFA0EBC140B0EB814F00BF42EBB7
:10136800020228BFA0EB8140B0EB414F00BF42EB27
:10137800020228BFA0EB4140B0EB014F00BF42EB97
:10138800020228BFA0EB0140B0EBC13F00BF42EB17
:10139800020228BFA0EBC130B0EB813F00BF42EB97
:1013A800020228BFA0EB8130B0EB413F00BF42EB07
:1013B800020228BFA0EB4130B0EB013F00BF42EB77
:1013C800020228BFA0EB0130B0EBC12F00BF42EBF7
:1013D800020228BFA0EBC120B0EB812F00BF42EB77
:1013E800020228BFA0EB8120B0EB412F00BF42EBE7
:1013F800020228BFA0EB4120B0EB012F00BF42EB57
:10140800020228BFA0EB0120B0EBC11F00BF42EBD6
:10141800020228BFA0EBC110B0EB811F00BF42EB56
:10142800020228BFA0EB8110B0EB411F00BF42EBC6
:10143800020228BFA0EB4110B0EB011F00BF42EB36
:10144800020228BFA0EB0110B0EBC10F00BF42EBB6
:10145800020228BFA0EBC100B0EB810F00BF42EB36
:10146800020228BFA0EB8100B0EB410F00BF42EBA6
:10147800020228BFA0EB4100B0EB010F00BF42EB16
:10148800020228BFA0EB0100104670470CBF0120E4
:1014980000207047B1FA81F2C2F11F0220FA02F06F
:1014A800704708B14FF0FF30FFF78EBB0029F8D026
:1014B8002DE90340FFF7CCFEBDE8064002FB00F330
:1014C800A1EB0301704700BF70B547F2744647F2BD
:1014D8007445C0F60306C0F60305761BB61007D0A0
:1014E800043D002455F8043F01349847A642F9D139
:1014F80047F2784647F27445C0F60306C0F603057E
:10150800761B15F0A3FFB61008D0043D002455F84B
:10151800043F01349847A642F9D170BD70BD00BFA1
:10152800032A70B422D941EA00039B0713D0057837
:10153800013A0C780023A54206D01BE010F8015FA1
:1015480011F8014FA54215D1934203F10103F5D1DA
:10155800002070BC70470C460346043104301E68F6
:101568002568AE4208D1043A032AF4D8002ADED10D
:101578001046EEE7281BECE721461846002AD6D18C
:10158800F6E700BF032A2DE9F00F09D82AB1002396
:10159800CC5CC45401339342FAD1BDE8F00F7047D4
:1015A800830702440ED0441C4D1C15F8017C04F03E
:1015B8000306234601342946013504F8027C002E2F
:1015C800F3D100E0034611F003046DD0D71A0D1BC8
:1015D800032F2E6819DDC4F1040C4FEAC4081C1D42
:1015E8004FEACC0C55F8047FC4EB020923460431BA
:1015F8000434B9F1030F26FA08FA07FA0CFB3E4641
:101608004BEA0A0744F8087CECDC9A42C5D9013356
:101618000131013211F8014C01330131934203F8D1
:10162800024CF7D1B9E70C684033403143F8404CDD
:1016380051F83C4C43F83C4C51F8384C43F8384C82
:1016480051F8344C43F8344C51F8304C43F8304C92
:1016580051F82C4C43F82C4C51F8284C43F8284CA2
:1016680051F8244C43F8244C51F8204C43F8204CB2
:1016780051F81C4C43F81C4C51F8184C43F8184CC2
:1016880051F8144C43F8144C51F8104C43F8104CD2
:1016980051F80C4C43F80C4C51F8084C43F8084CE2
:1016A80051F8044C43F8044CD41A3F2CBBDC11E02D
:1016B8000C681033103143F8104C51F80C4C43F8B7
:1016C8000C4C51F8084C43F8084C51F8044C43F8BA
:1016D800044CD41A0F2CEBDC032C96DD1C1D0D1DBD
:1016E80055F8047C161B2346294604340435032E7A
:1016F80044F8087CF4DC88E7032AC9B270B408D837
:101708002AB10346121803F8011B9342FBD170BC9F
:1017180070478307024409D0441C04F0030523469C
:1017280004F8011C0134002DF7D100E00346D51A56
:1017380001EB01243F2D04EB04442CDD1C604033F5
:10174800D51A43F83C4C3F2D43F8384C43F8344CF9
:1017580043F8304C43F82C4C43F8284C43F8244CBD
:1017680043F8204C43F81C4C43F8184C43F8144CED
:1017780043F8104C43F80C4C43F8084C43F8044C1D
:10178800DCDC08E01C601033D51A43F80C4C43F835
:10179800084C43F8044C0F2DF4DC032D08DD1D1D07
:1017A800561B45F8044C032E2B4605F10405F7DCBF
:1017B8009A42ACD90133013203F8011C0133934238
:1017C800FAD1A4E7830770B5064614D10368A3F1DC
:1017D800013222EA030313F0803F0CD1031D1A469D
:1017E80053F8044BA4F1013525EA040414F0803FB2
:1017F800F5D0104600E0304603782BB1431C18465C
:1018080001330478002CFAD100F0F0F8304670BDAE
:1018180080EA010212F0030F40F03A8010F0030250
:1018280020F0030021F0030150F804CB08BF51F861
:10183800043B0DD082F003024FEAC2026FF07F43EF
:1018480023FA02F251F8043B4CEA020C43EA020381
:10185800ACF101329C4501BF22EA0C0212F0803F34
:1018680050F804CB51F8043BF2D04FEA0C604FEA31
:101878001C2C012828BFB0EB036F08BF1B0AF4D04B
:1018880003F0FF034FEA1060A0EB0300704700BFAE
:1018980010F0030F0AD010F8012B11F8013B012AB0
:1018A80028BF9A42F4D0A2EB030070474DF8045DBC
:1018B8004DF8044D4FF0010242EA022242EA024288
:1018C80001F0030C21F0030150F8044B51F8045BBC
:1018D800BCF1020F26D04BD824F07F4CBCEB152F5F
:1018E800A4EB020323EA04030DD113EAC21308BFD1
:1018F80051F8045B0AD18CEA040CBCEB056F0CD1DF
:1019080050F8044BE8E74FEA15255CE033F07F43D5
:1019180052D10D784FEA146C55E04FEA146C05F07B
:10192800FF0550E04FEA044CA4EB02034FEA1C4CBD
:1019380023EA0403BCEB154F17D113EAC21308BFFF
:1019480051F8045B07D18CEA040CBCEB054F08D1B5
:1019580050F8044BE6E71B042ED10D884FEA144CCF
:1019680031E04FEA05454FEA144C4FEA15452AE0A5
:1019780004F0FF0CBCEB156FA4EB020323EA04038D
:101988000DD113EAC21308BF51F8045B0AD18CEADF
:10199800040CBCEB052F0AD150F8044BE8E74FEADA
:1019A800156510E014F0FF0F06D051F8045B4FEAFC
:1019B800142C25F07F4506E04FF000005DF8044B3D
:1019C8005DF8045B70470CF0FF0205F0FF0001288A
:1019D80028BF904204BF4FEA1C2C2D0AF3D0A2EB7B
:1019E80000005DF8044B5DF8045B704780EA010273
:1019F800844612F0030F4FD111F0030F32D14DF886
:101A0800044D11F0040F51F8043B0BD0A3F101323F
:101A18009A4312F0803F04BF4CF8043B51F8043B52
:101A280016D100BF51F8044BA3F101329A4312F0CA
:101A3800803FA4F101320BD14CF8043BA24312F0D1
:101A4800803F04BF51F8043B4CF8044BEAD02346CE
:101A58000CF8013B13F0FF0F4FEA3323F8D15DF880
:101A6800044B704711F0010F06D011F8012B0CF848
:101A7800012B002A08BF704711F0020FBFD031F8C0
:101A8800022B12F0FF0F16BF2CF8022B8CF8002047
:101A980012F47F4FB3D1704711F8012B0CF8012BCA
:101AA800002AF9D1704700BF20F0030110F00300AD
:101AB800C0F1000051F8043B00F1040C4FEACC0CD3
:101AC8006FF000021CBF22FA0CF213434FF0010C16
:101AD8004CEA0C2C4CEA0C4CA3EB0C0222EA030255
:101AE80012EACC1204BF51F8043B0430F4D013F0CE
:101AF800FF0F1FBF013013F47F4F013013F47F0F26
:101B080018BF0130704700BF830770B413D1036852
:101B1800A3F1013424EA030313F0803F0BD1031D22
:101B28001D4653F8044BA4F1013626EA040414F0C8
:101B3800803FF5D000E005462B782BB16B1C1D4685
:101B480001332C78002CFAD10139013D531E5AB1CA
:101B580011F8014F1A4605F8014F2CB1002BF5D1A9
:101B68006B70531E002AF3D170BC704770B4002A02
:101B780045D041EA000313F0030329D1032A27D9EA
:101B880005680C68A54223D1141F3AD0A5F101328B
:101B980022EA050515F0803F0DD03AE05B686A68D7
:101BA800A3F10135934225EA03052ED1043C28D040
:101BB80015F0803F27D10D46034604310430032C2D
:101BC800ECD8661E2CB91C792A79A01A70BC70470B
:101BD800561E04780A789442F7D1C6B18CB1013602
:101BE8008B1C891904E08B4203F101030BD044B12B
:101BF80013F8012C10F8014F9442F4D0E5E7104691
:101C0800E4E72046E2E70020E0E7661EE1E7304629
:101C1800DCE71846DAE700BF41EA000313F0030FD8
:101C2800034670B425D0AAB10C78013A03F8014BE9
:101C38004CB11C4672B111F8015F013A04F8015B1E
:101C48002346002DF6D12AB19A18002103F8011B6A
:101C58009342FBD170BC70470E4651F8044BA4F177
:101C6800013525EA040515F0803F05D1043A43F80B
:101C7800044B032AF0D8D6E73146D4E7F0B4047809
:101C8800002C21D00F7806463046AFB1A74219D0B4
:101C98004B1C01E0944209D01D4613F8012B002A81
:101CA800F8D144780136002CEED12A78002A14BFE6
:101CB80030460020F0BC704744780D460136002CB1
:101CC800E2D1F2E73A46F1E72046F3E72DE9F007DB
:101CD80001273C4600254FF0FF36631900EB060C40
:101CE8008B420DD21CF804C010F80380E0452ED2B8
:101CF80001241D469F1B63198B4200EB060CF1D390
:101D08004FF0010A002554464FF0FF3C1760631955
:101D180000EB0C0899420ED918F8048010F80390CB
:101D2800C1451AD901241D46CCEB030A631999420F
:101D380000EB0C08F0D80CF101000136B0423CBFB2
:101D4800BA463046C2F800A0BDE8F00770470BD08D
:101D580001272E463C46ED19BFE709D04FF0010A8E
:101D6800AC4654465544D2E7BC4205D00134B4E7EA
:101D7800544505D00134CAE727461D460124ACE77F
:101D8800A2461D460124C2E72DE9F04FADF2244DCD
:101D9800164680460C461046194607AA1D46FFF708
:101DA80095FF07AB0DF21C42039043F8045F934282
:101DB800FBD16F1E002308A835B1F25CF91A013374
:101DC800AB4240F82210F8D107993046039A7118AF
:101DD800FFF7A6FB00287FD1DDF80CC0224682461B
:101DE8006F1E0CF1FF3CCDF808C0B444CDF814C008
:101DF800DDF80CC004460195CCF1010CCDF810C0FB
:101E080009E034B1079A93423EBF04460199C2EBF8
:101E180001039A442A46019B08EB020000210AEBC1
:101E28000305AA1A00F078FA00284FD1002D4DD0EA
:101E380008EB050308A913F8013C51F82330002BDF
:101E4800DFD1039A944228BF2246BA4211D208EB46
:101E58000A0316F802C0B118985C844506D02FE032
:101E680011F8010F13F802C0844529D10132BA4292
:101E7800F6D3039B02989C4228BF184618D2DDF877
:101E880008C008EB0A0316F80C1013F80C2091424E
:101E980040F08580059A06EB040B06E013F801C0B4
:101EA80012F8019DE14503D10846411E5A45F5D176
:101EB8000134844275D8079C019BA2441C1BA9E7E6
:101EC800DDF810C00024E2449244A3E7002009B0E2
:101ED8000DF5806DBDE8F08FDDF80CC04FF0000AFD
:101EE800DDF80CB00DF12009CCEB05036F1E63453E
:101EF80038BF63462246013307930CF1FF33019341
:101F0800039BB444CDF808C0C3F1010304930AEB62
:101F1800050408EB02000021A21A00F0FDF90028D0
:101F2800D4D1002CD2D008EB040313F8013C59F8A3
:101F3800233063BBBB4508EB0A0015D2DDF808C0A7
:101F480010F80B309CF800209A4218BF5B4621D14C
:101F5800029A5B4605E012F8011F10F803C08C4591
:101F680018D10133BB42F6D3019B5A1CAFD0DDF820
:101F780004C016F80C1010F80C20914206D113F189
:101F8800FF33A4D3F15CC25C9142F8D0079B9A441A
:101F98002246BCE7DDF810C0E2449A44F8E703980B
:101FA80086E708EB0A0092E72DE9F04F80460378B0
:101FB80087B00E46002B00F0F7800A789AB1844665
:101FC8000131012702E011F8012B5AB1934214BFE5
:101FD800002707F001071CF8013F0D46002BF2D13E
:101FE8002B7803BB1FB1404607B0BDE8F08F08F15E
:101FF8000100317800F0DAF9AD1B012D18BF002877
:10200800074608BF8046EED0A844404594BFC0EBC1
:10201800080401241F2D09D9214632462B46FFF713
:10202800B3FE8046DFE74FF00008DCE7294605AA43
:102038003046FFF74BFE0599711801903046019A1A
:10204800FFF76EFA002852D1019B83468046013B78
:102058000093F3180393019BC3F1010302932246F3
:1020680008EB0504B8180021A21A00F055F9002859
:10207800D9D1002CD7D0019B9B4528BF5B469D42F8
:1020880013D9F918F05CF21811F80810884240F0DA
:10209800858007EB080C05E012F8011F1CF8030007
:1020A80088427BD101339D42F6D89DE80A005B4502
:1020B8007DD907EB0809725C19F801309A4276D18C
:1020C800039B06EB0B0A06E019F8020013F801CD92
:1020D800844503D111464A1E5345F5D10BF1010B36
:1020E8008B4566D8059B9844C3EB050BB7E7019869
:1020F8004FF0000B22462B1A06EB000900F1FF38BF
:102108008246834238BF034639180133009105934C
:10211800C0F1010302930BEB0504B8180021A21AC1
:1021280000F0FAF800287FF47EAF002C3FF47BAF74
:10213800554598BF07EB0B0014D9009899F8002073
:1021480010F80B309A4224D14A46534607EB0B004D
:1021580005E012F8011F10F803C08C451AD10133AD
:102168009D42F6D8B8F1FF3F43463FF45AAF16F800
:10217800081010F80820914207D113F1FF33FFF43B
:1021880050AFF15CC25C9142F7D0059B9B4422465C
:10219800C1E75346029A93449B44F8E702994FF0EB
:1021A800000B884498445AE70D46012718E701991F
:1021B80094E7B84417E700BF2DE9F04F40F2000458
:1021C800C2F2000485B099460B46D4F8008002910B
:1021D80003901C4614F8015B08EB05012346497877
:1021E80001F00801C9B20029F3D12D2D7BD02B2D88
:1021F80005BF24460B460B4614F8015B39F0100165
:1022080012D1D9F1010038BF0020302D04D058B1C7
:102218004FF00A09CB4608E0217801F0DF01582980
:1022280065D008B14FF00809CB46002B59460CBFC2
:102238006FF000464FF000468DE80C00304600274E
:10224800FFF734F930468A465946FFF701F8BC468D
:102258009DE80C0016E0303DA94525DD844594BF76
:102268000021012151EAD77729D15545D4BF002152
:102278000121844518BF002109BB0BFB0C5C012719
:1022880014F8015B08EB0501497801F00406F6B281
:10229800002EE0D111F0030106D0012914BF572107
:1022A80037216D1AA945D9DC791C0BD0C3B9604612
:1022B80012B197B9029B136005B0BDE8F08F4FF0DB
:1022C800FF37DDE70399002B0CBF6FF000404FF09C
:1022D800004022230B60002AEED0013C0294E9E77B
:1022E800CCF1000CE3E714F8015B012386E74FF01B
:1022F80010096578CB46023497E700BF30B440F246
:102308000404C2F200040D46134601462A4620681A
:1023180030BCFFF751BF00BF8307C9B270B440D0CB
:10232800541E002A3FD003788B4221D0431C04E07E
:1023380004B30278013C8A421AD013F0030F1846FE
:1023480003F10103F4D1032C16D8651E94B1037868
:102358008B420DD0421C002302E004788C4207D047
:102368009D42104603F1010302F10102F5D100205C
:1023780070BC70472046FBE741EA012646EA06465C
:102388000246043013687340A3F1013525EA0303BC
:1023980013F0803F03D1043C032CF1D8D5E7104655
:1023A800D3E71446CFE71046E2E700BFC9B2F0B45E
:1023B80000294BD083070FD00378002B73D09942A4
:1023C80042D0431C05E013F8012B002A3BD0914270
:1023D8003AD09A071846F6D1036841EA0127A3F1D3
:1023E800013247EA074722EA030212F0803F1CD174
:1023F8007B40A3F1013222EA030313F0803F14D19A
:10240800021D02E014F0803F0FD1104652F8043B41
:10241800A3F1013687EA030426EA0303A4F1013590
:1024280013F0803F25EA0404ECD00378002B3AD05F
:10243800994209D0431C01E0914205D0184613F88F
:10244800012B002AF8D11046F0BC704781070DD047
:102458000378002BF8D0431C02E00278002AF3D05E
:1024680013F0030F184603F10103F6D10368A3F133
:10247800013222EA030313F0803F0AD1021D1046FD
:1024880052F8041BA1F1013424EA010111F0803F44
:10249800F5D00378002BD7D0431C184601330278B7
:1024A800002AFAD1D0E71846CEE700BF40F0BF6057
:1024B800024B40F40030D860704700BF00ED00E0E8
:1024C800C3780BB3164B4178DB68DB43C3F30223B5
:1024D800C3F10402D2B201FA02F20F2141FA03F366
:1024E8008178D2B20B401A43037803F1604303F5B5
:1024F8006143120183F8002303780122590903F08C
:102508001F0302FA03F307E003780122590903F0D5
:102518001F0302FA03F32031024A42F821307047C0
:1025280000ED00E000E100E021F0604121F07F01D2
:10253800014B08439860704700ED00E0014B012211
:102548009A6070470030024010B50023054C03E044
:1025580050F82320013322608B42F9D1014B1868CF
:1025680010BD00BF00300240044B1A69002A04DA8B
:10257800034A5A6002F188325A607047003C0240B0
:1025880023016745024B1A6942F000421A617047FD
:10259800003C0240014BD860704700BF003C02403D
:1025A8000B4BDA68D0030DD4DA68D1060CD4DA689C
:1025B80012F0EF0F0AD1DB6813F0020F0CBF0820EE
:1025C8000720704701207047052070470620704794
:1025D800003C024007B508238DF80730FFF7E0FFFD
:1025E8008DF807009DF80730012BF7D09DF80700FC
:1025F8000EBD000070B505460E46FFF7EBFF082834
:1026080011D1094C236923F44073236123692361A1
:10261800236943F0010323612E70FFF7DBFF236971
:1026280023F00103236170BD003C024070B50546EC
:102638000E46FFF7CFFF082813D10A4C236923F46D
:1026480040732361236943F400732361236943F0D2
:10265800010323612E60FFF7BDFF236923F0010307
:10266800236170BD003C024070B5064641B10129A6
:1026780008D0022914BF4FF440754FF4007503E0E9
:102688000D4601E04FF48075FFF7A4FF08281ED11E
:102698000F4C236923F44073236121690D4325619D
:1026A800236923F0F8032361236943F002031E43DF
:1026B8002661236943F480332361FFF78BFF236985
:1026C80023F002032361236923F0F803236170BD1B
:1026D800003C024008B52C4B984205D10120014628
:1026E80000F022F9012048E0284B984205D1022049
:1026F800012100F019F902203FE0254B984205D14D
:102708000420012100F010F9042036E0214B984202
:1027180005D10820012100F007F908202DE01E4B03
:10272800984205D11020012100F0FEF8102024E085
:102738001A4B984205D12020012100F0F5F82020FD
:102748001BE0174B984205D14020012100F0ECF81E
:10275800402012E0134B984205D18020012100F05F
:10276800E3F8802009E0104B98420BD14FF48070B9
:10277800012100F0D9F84FF480700021BDE808402D
:1027880000F0D2B808BD00BF0000024000040240BB
:1027980000080240000C02400010024000140240F1
:1027A80000180240001C0240002002402DE9F047BA
:1027B8000F6800234FF0010C4FF003080CFA03F2E6
:1027C80002EA0705954231D15A00066808FA02F470
:1027D800E443264006600E79D0F8009006FA02FA23
:1027E800013E4AEA0909012EC0F8009015D886680A
:1027F80091F8059026408660866809FA02F949EA48
:1028080006068660466826EA050545608D794668AD
:1028180005FA03F5ADB235434560C5682C40C46080
:10282800CD79C46805FA02F22243C2600133102B45
:10283800C4D1BDE8F087018370474183704701F038
:102848000703C908083130B59B0050F821500F2400
:1028580004FA03F425EA040440F8214050F8214022
:1028680002FA03F2144340F8214030BD1E4B9A6827
:1028780002F00C02042A10B503D0082A03D01B4B1F
:1028880018E01B4B16E059685A6811F4800F596814
:1028980014BF174B154B02F03F02B3FBF2F3124A79
:1028A8005268C2F30142C1F3881101324B4352000E
:1028B800B3FBF2F30C4903608B680E4AC3F30313AE
:1028C800D45C036823FA04F343608C68C4F382245D
:1028D800145D23FA04F484608968C1F34231525CC0
:1028E80023FA02F3C36010BD003802400024F4004C
:1028F80040787D01F8000020044B1A6B09B11043A1
:1029080001E022EA00001863704700BF0038024067
:10291800044B5A6C09B1104301E022EA00005864E4
:10292800704700BF00380240044B1A6909B11043D0
:1029380001E022EA00001861704700BF0038024039
:102948000A4B1A6C10B59C68D96802F0040202EAB6
:10295800D03200EA0403134306D08BB213EA1013F3
:102968000CBF0020012010BD184610BD00280040F3
:10297800054BDA68C0F30F1040F0800002F08002C7
:1029880062EA0002DA60704700280040014B1860D4
:10299800704700BFDC002742354B1A6842F001023D
:1029A8001A6000229A60196821F0847121F480313C
:1029B800196030495960196882B021F48021196082
:1029C800DA60009201921A6842F480321A601A683A
:1029D80002F400320192009A01320092019A1AB967
:1029E800009AB2F5A06FF2D1214B1B6813F40033A3
:1029F80018BF01230193019B012B33D11C4B1A6C87
:102A080042F080521A641C4A116841F480411160F6
:102A18009A689A609A6842F400429A609A6842F406
:102A2800A0529A60154A5A601A6842F080721A6079
:102A380019680F4A8901FBD5114B40F205611960ED
:102A4800936823F003039360936843F00203936051
:102A58009168074B01F00C010829F9D11A6842F472
:102A680000221A60074B4FF000629A6002B070476C
:102A7800003802401030002400700040195440070C
:102A8800003C024000ED00E04B00DBB270B50324CF
:102A9800056804FA03F4E44325400560066802F07B
:102AA800030505FA03F5354305604668012505FA6F
:102AB80001F526EA050545604568C2F3800606FA71
:102AC80001F1294341608168214081608568C2F332
:102AD800011101FA03F129438160C1680C40C46007
:102AE800C168C2F3811202FA03F30B43C36070BDDD
:102AF80010B5134B03EBC00253F830301279072A94
:102B08000ED892001C6AD2B20F2000FA02F024EA12
:102B180000001862186A01FA02F202431A6210BD34
:102B2800083A92005C6AD2B20F2000FA02F024EA56
:102B380000005862586A01FA02F202435A6210BD54
:102B48000C0100200E4B03EBC002D28802F01002E9
:102B580092B20AB181F00101C20041B153F83010BC
:102B68009B1801221B7902FA03F30B83704753F871
:102B780030109B1801221B7902FA03F34B8370472C
:102B88000C01002070B51E4E06EBC0050446E9880E
:102B980001F400739BB23BB1890AFFF7A9FF56F80D
:102BA80034002979322205E0CB0707D556F83000E2
:102BB80029793022BDE87040FFF766BF01F00203B3
:102BC8009BB223B156F83000297970220DE001F04C
:102BD80004039BB29BB101F020018AB256F8300081
:102BE8002979002A0CBF31223522FFF74DFFE988E9
:102BF8002046C1F3C001BDE87040FFF7A3BF70BD18
:102C08000C01002038B51248124DFFF763FD124839
:102C1800FFF760FD1148FFF75DFD1148FFF75AFD0A
:102C28001048FFF757FD104B1A6B42F01F021A634A
:102C3800002405EBC403DB8803F080039BB213B9BF
:102C4800E0B2FFF79FFF0134112CF2D138BD00BF6D
:102C5800000002400C01002000040240000802406D
:102C6800000C024000100240003802402DE9F041FB
:102C7800427A40F2B27302F5FA6200214FF4C87545
:102C880064269C0708D1B3FBF6F406FB1434A4B2FF
:102C980014B14FF4B77408E0B3FBF5F405FB143432
:102CA800A4B2002CF5D040F26D1401339BB29342CC
:102CB8002144E6D36423B2FBF3F703FB17239FB247
:102CC8004FF4C873B2FBF3F403FB1424A4B2D4F199
:102CD800010438BF0024067ADFF858C0002302F048
:102CE80003024FF00C080CE022B9002F0CBF254658
:102CF800012500E0254608FB053501331CF8055081
:102D080049195D1CADB2B542EED3C3794479013B94
:102D1800591803799A009B019A1A4FF4616303FBCF
:102D28000423027802489B1800FB0130BDE8F081BB
:102D380080510100940100207047704770470000DF
:102D480008B54FF48040FFF7FBFD28B14FF48040F1
:102D5800FFF70EFEFFF7F0FF024B4FF480025A61B7
:102D680008BD00BF003C014008B54FF48050FFF794
:102D7800E7FD28B14FF48050FFF7FAFDFFF7DDFFBC
:102D88004FF40050FFF7DCFD28B14FF40050FFF777
:102D9800EFFDFFF7D3FF024B4FF400325A6108BD35
:102DA800003C014030B5002285B013460A2506E0F4
:102DB80005FB0212303A013302F0FF02DBB2C15CBC
:102DC800A1F13004092CF3D901338DF80720DBB2C7
:102DD80000220A2506E005FB0212303A013302F010
:102DE800FF02DBB2C15CA1F13004092CF3D9033333
:102DF8008DF80820DBB200220A2506E005FB021246
:102E0800303A013302F0FF02DBB2C15CA1F13004B9
:102E1800092CF3D902338DF80920DBB200220A25E8
:102E280006E005FB0212303A013302F0FF02DBB282
:102E3800C15CA1F13004092CF3D901338DF80520C8
:102E4800DBB200220A2506E005FB0212303A013304
:102E580002F0FF02DBB2C15CA1F13004092CF3D906
:102E680000238DF800309DF809308DF804200133D7
:102E780068468DF80930FFF7F9FE024B186005B077
:102E880030BD00BF5028004010B5002484F0010474
:102E9800102004F00101FFF755FE7D2001F058FDD8
:102EA800F4E700001FB500240E4900948022234651
:102EB8000194029403940C4801F0B4FA00F03AFF2C
:102EC8000CF03EF90BF052FF02F074F94FF47A60FF
:102ED80001F03EFD204601F07DFB04B0BDE8104046
:102EE80001F012BFA0FB0208912E02081FB572B6AE
:102EF8004FF000604FF40031FFF716FB184AD16815
:102F08004FF6FF030B4043F0BF6343F40033D36035
:102F18004FF44070FFF7CAFA62B601214FF48050AF
:102F2800FFF7EAFC4020FFF735FB80200024FFF77D
:102F380031FBFFF767FE4FF44070FFF7B7FA094916
:102F480000944FF47A72234601940294039406483D
:102F580001F068FA01F098FB204604B010BD00BFEC
:102F680000ED00E0A4FB0208AD2E020808B50C4BEA
:102F7800DA68120603D5DA6842F40002DA6040F231
:102F8800F23001F0E5FCBFF34F8F064A064BD168DB
:102F980001F4E0610B43D360BFF34F8FFEE700BF3E
:102FA8000038024000ED00E00400FA0508B50248C8
:102FB80000F06CFBFEE700BFADFB0208FEE7FEE792
:102FC800FEE7704707B50023402001930CF056FB3D
:102FD800012804D1094B01A9186801F013F9402010
:102FE8000CF062FB4FF480300CF05EFB019B1BB1D0
:102FF800034B4FF080521A600EBD00BFB4C00020D2
:1030080004ED00E02DE9F84FD368D2F810B08146FE
:103018008A4690461E4600270124002506E004FB48
:1030280007F306FB0533A4FB06455D1948465146E0
:1030380022462B46FDF782FDB94208BFB042EED2C8
:1030480000262DE022462B4648465146FDF776FDE0
:10305800514622462B4607464846FDF76FFD204657
:10306800294691469A46D8F80C200023FDF766FDBC
:1030780004460D4626B9002F02DC54EA0503E1D1C7
:10308800092FFAB207DD98F8003013F0040F0CBFCF
:103098005723372300E030239B180BF8013B0136F8
:1030A80054EA0503CED100238BF80030BDE8F88F31
:1030B80070B5CA680C69012300E05343B0FBF3F50F
:1030C8009542FAD200251AE0CE68B0FBF3F203FB72
:1030D8001200B3FBF6F31DB9002A01DC002BF3D173
:1030E800092AD6B206DD0A7812F0040F0CBF57225F
:1030F800372200E03022921904F8012B0135002B09
:10310800E2D1237070BD70B5CA680C69012300E074
:103118005343B0FBF3F59542FAD200251AE0CE6886
:10312800B0FBF3F203FB1200B3FBF6F31DB9002A60
:1031380001DC002BF3D1092AD6B206DD0A7812F099
:10314800040F0CBF5722372200E03022921904F8EE
:10315800012B0135002BE2D1237070BD2DE9F04120
:103168001369546806460F46154600E0013C13F8FB
:10317800012B12B92B7A1BB903E0002CF6DCF9E716
:10318800013C2B78990707D5EB68102B01D1023C3D
:1031980002E0082B08BF013C2B7813F0090F0DD172
:1031A800A04604E030462021B84708F1FF38B8F1BE
:1031B800000FF7DC631E24EAE4741C1B297A09B1AA
:1031C8003046B8472B789A0712D5EB68102B0AD1EE
:1031D80030213046B8472B7813F0040F30460CBF27
:1031E8007821582103E0082B02D130463021B84716
:1031F8002B78DB070DD5A04604E030463021B847D0
:1032080008F1FF38B8F1000FF7DC631E24EAE47414
:103218001C1BD5F8108001E03046B84718F8011B90
:103228000029F9D12B7803F00903082B06D103E014
:1032380030462021B847013C002CF9DCBDE8F0817C
:1032480090E80C00D1540133436070472DE9F04FEA
:103258009BB0174604AA05460E461C460E9208E285
:10326800252900D03AE19DF82820002302F0FC022D
:1032780063F3C3028DF828200221D2B202F0010CB8
:10328800C2F340000B938DF830308DF83C10C2F338
:10329800C00212E02D290FD004D8232908D02B29E9
:1032A8000FD107E0302900D00BE04FF0010C04E00B
:1032B800012002E0012300E0012217F8011B002988
:1032C800E8D19DF828808DF830306CF30008C446AA
:1032D80060F3410C6046A1F1300362F3C300092B8F
:1032E8008DF828001DD804E000FB023217F8011BF6
:1032F80001E000220A20A1F130035FFA83FCBCF14F
:10330800090FF1D9A1F16103052B02D8A1F15703E7
:10331800B5E1A1F14103052B02D8A1F13703AEE1D4
:103328000B922E290ED13A78303AD2B27B1C092A58
:1033380098BF8DF83C2013F8011BA1F13002092A2F
:103348001F46F8D97A2902D117F8011B05E06C2924
:1033580009D139786C2902D00137012304E0797842
:103368000223023700E00023692936D016D86329E2
:1033780000F0A1800CD8462900F0B38006D80029B7
:1033880000F08181252940F07481A7E0582912E0D6
:10339800642922D0662940F06C81A2E0732900F0EC
:1033A800908005D86F2978D0702940F0628140E07C
:1033B800752903D0782940F05C8141E00A22022B6C
:1033C8000D9207D1073424F0070303F10804D3E969
:1033D800000117E020680AA94FE00A22022B0D928B
:1033E80012D1073424F00703D3E9000103F10804DC
:1033F800002871F1000305DA2D23404261EB4101F9
:103408008DF830300AAA33E0012B206804F1040853
:1034180007D1002803DA2D2340428DF830300AA95D
:103428002FE0002803DA2D2340428DF830300AA916
:103438002AE09DF8283043F002038DF82830002355
:103448001022B1F1580EDEF100019DF828000D920E
:1034580051EB0E011AAA61F38200022B02F8400D0B
:1034680009D1073424F00703D3E9000103F1080464
:10347800FFF7C8FD0BE020681146012B04F1040892
:1034880002D1FFF715FE01E0FFF73DFE444628464E
:1034980031460AAAFFF762FEEBE0082320680D9385
:1034A8000AA9FFF730FE284631460AAA04F10408A3
:1034B800FFF754FE10E02846217804F10408B047CD
:1034C8000AE023680AAA284631460E93FFF746FE0B
:1034D80004AA04F104080E924446CAE02846B047FC
:1034E800C7E0073424F0070303F1080493E8040451
:1034F80000921046514600220023FDF7CFFA38B15A
:103508000B9B013B0B930AF1004A4FF0010B09E0BA
:103518009DF830302BB10B9B013B0B934FF0020B06
:1035280000E09B4651460098FDF7E0FA0022019022
:1035380080460A2108E098FBF1F010AB01FB1088E7
:1035480043F8228001328046B8F1000FF3D102F12E
:10355800FF3912B90B9A013A0B929DF82820D0072F
:103568001BD5BBF1010F02D128462D2107E0BBF185
:10357800020F05D128462B2101E028463021B0470B
:103588009DF83C200B9B4A440232591E93420B91F2
:10359800F3DC17E028462021B0479DF83C100B9A31
:1035A80049440231501E8A420B90F3DCBBF1010FF3
:1035B80002D128462D2104E0BBF1020F02D1284692
:1035C8002B21B047B9F1FF3F02D12846302107E04F
:1035D80010AB284653F82910303109F1FF39C9B228
:1035E800B047B9F1FF3FF3D128462E21B0474FF03D
:1035F80001091DE00A23019803FB09F9FCF776FF8E
:1036080002460B4600985146FCF722FECDE902011E
:103618004846FCF76BFF02460B46DDE90201FCF762
:10362800CBFFFDF763FA804610B928463021B04732
:103638009DF83C305A1E8DF83C20002BDAD10A2226
:1036480008E098FBF2F110A802FB118840F82380EB
:1036580001338846B8F1000FF3D1984606E010AB65
:10366800284653F828103031C9B2B04718F1FF384E
:10367800F5D217F8011B00297FF4F2AD03E00A2BFD
:103688007FF732AE4CE61BB0BDE8F08F0FB407B53C
:10369800064904AB0868064953F8042B09680193E6
:1036A800FFF7D4FDBDE80E4004B07047F0040020D9
:1036B800EC04002037B50D461346009000246846F8
:1036C8002A4604490194FFF7C1FD9DE80C00D45433
:1036D80001983EBD493202080EB403B503AA52F858
:1036E800041B0192FFF7E6FFBDE80C4003B07047EA
:1036F80001230B707047704710B50C46FEF7D4F9DC
:10370800207010BD10B50C46FEF7CEF9207010BD24
:1037180010B50C46FEF7C8F9207010BD10B50C4660
:10372800FEF7C2F9207010BD10B50C46FEF7BCF9C3
:10373800207010BD10B50C46FEF7B6F9207010BD0C
:1037480010B50C46FEF7B0F9207010BD10B50C4648
:10375800FEF7AAF9207010BD01230B7070470123F2
:103768000B70704701230B70704700007FB504464B
:1037780003A80E4608F05CF803980C4B0C4DB0FB00
:10378800F3F203FB1200B0FBF5F305FB130041F263
:1037980070710390B0FBF1F0009006492046FFF7E6
:1037A8009BFF2046FEF780F930707FBD00D683006E
:1037B800407E0500B9FB020870B5074C0546204657
:1037C8000E46FEF771F90246307021462846D2B2FD
:1037D800BDE87040FEF720BA30C2002070B5074C33
:1037E800054620460E46FEF75FF902463070214630
:1037F8002846D2B2BDE87040FEF70EBAEEC20020ED
:1038080070B5074C054620460E46FEF74DF90246B0
:10381800307021462846D2B2BDE87040FEF7FCB9A8
:10382800D4FB020870B5074C054620460E46FEF745
:103838003BF90246307021462846D2B2BDE87040B6
:10384800FEF7EAB916C3002070B5074C05462046B6
:103858000E46FEF729F90246307021462846D2B2B4
:10386800BDE87040FEF7D8B928C3002070B5074CF2
:10387800054620460E46FEF717F9024630702146E7
:103888002846D2B2BDE87040FEF7C6B9FEC1002096
:1038980070B5074C054620460E46FEF705F9024668
:1038A800307021462846D2B2BDE87040FEF7B4B960
:1038B80044C2002070B5074C054620460E46FEF768
:1038C800F3F80246307021462846D2B2BDE870406F
:1038D800FEF7A2B938C30020084A38B592F8CE32AC
:1038E8000C46054606490BB1303200E00232FFF7BC
:1038F800F3FE2846FEF7D8F8207038BDD8C000205F
:10390800D8FB0208084A38B592F8CE320C4605466C
:1039180006490BB13F3200E01132FFF7DDFE2846C1
:10392800FEF7C2F8207038BDD8C00020D8FB0208C6
:10393800084A38B592F8CE320C46054606490BB10E
:103948004E3200E02032FFF7C7FE2846FEF7ACF8FB
:10395800207038BDD8C00020D8FB0208084B93F867
:10396800CE2212B193F85D3001E093F82F300BB1FD
:10397800312300E03023037001230B70704700BF30
:10398800D8C0002038B5054A05460C460449FFF75B
:10399800A3FE2846FEF788F8207038BDD6C100205F
:1039A800D8FB020838B5054A05460C460449FFF716
:1039B80093FE2846FEF778F8207038BDEAC100204B
:1039C800D8FB020838B5054A05460C460449FFF7F6
:1039D80083FE2846FEF768F8207038BDB2C2002082
:1039E800D8FB020838B5054A05460C460449FFF7D6
:1039F80073FE2846FEF758F8207038BDC6C200206E
:103A0800D8FB020838B5054A05460C460449FFF7B5
:103A180063FE2846FEF748F8207038BDDAC2002059
:103A2800D8FB020810B5044A0C460449FFF754FEB7
:103A38000123237010BD00BFFFFB0208D8FB02085A
:103A480010B5044A0C460449FFF746FE01232370CB
:103A580010BD00BFFFFB0208D8FB020838B5084BB1
:103A680093F8CE320C46054606490BB1064A00E0EB
:103A7800064AFFF731FE2846FEF716F8207038BDD3
:103A8800D8C00020D8FB0208DBFB0208E0FB0208D4
:103A9800014B01221A707047D8C00020014B83F8EF
:103AA800CE027047D8C00020014B01221A7070471F
:103AB800F404002001460148FDF798BF08C1002022
:103AC80001460148FDF792BF17C100200146014891
:103AD800FDF78CBF26C1002008B506490222FEF773
:103AE80045F8054B08B9012200E0002283F85D2063
:103AF80008BD00BFE6FB0208D8C000200146014807
:103B0800FDF774BFD6C1002001460148FDF76EBF1E
:103B1800EAC1002010B5054C01462046FDF766FFB6
:103B28002046BDE810400BF0FDBA00BFB2C200202D
:103B380010B5054C01462046FDF758FF2046BDE864
:103B480010400BF0EFBA00BFC6C2002010B5054CFC
:103B580001462046FDF74AFF2046BDE810400BF01D
:103B6800E1BA00BFDAC2002010B5064C0146204673
:103B7800FDF73CFF20460BF0B9FABDE810400BF00A
:103B880081BA00BFFEC1002010B5054C0146204691
:103B9800FDF72CFF2046BDE810400BF0B5BA00BF7A
:103BA80044C2002001460148FDF720BF38C3002069
:103BB800024B00221A705A70704700BFD8C000200C
:103BC80070B5194C194D1A4E29462046FDF70EFFBF
:103BD800314604F1A000FDF709FF314604F1B400B5
:103BE800FDF704FF294604F1C800FDF7FFFE04F1C4
:103BF800FA001049FDF7FAFE29460F4D04F58770C3
:103C0800FDF7F4FE294604F5BE70FDF7EFFE2946E0
:103C180004F5C870FDF7EAFE04F5D2702946BDE840
:103C28007040FDF7E3BE00BF36C10020FF66030801
:103C38000FFC020816FC02081EFC020808B5FFF774
:103C4800B7FFFFF7BDFF044B002283F8CE22034ADB
:103C5800C3F8E02208BD00BFD8C0002015CD5B071F
:103C6800002306E003F1006202F580421268C254A4
:103C780001338B42F6D1704720200221FEF7F4BCB5
:103C880008B5FEF75BFC0348B921BDE80840FEF71C
:103C98005BBC00BFD8C000202DE9F74F0E46074691
:103CA800FFF7EEFF8246FEF75FFC1A4D1A4C4FF005
:103CB80003094FF00008FFF7DFFF04EB060B7B1941
:103CC80006E0195D01932046FEF794FC019B013440
:103CD8005C45F6D151461148FEF7A8FCFEF752FCA8
:103CE8000F484FF43971FFF7BBFFFFF7C9FF504585
:103CF800374409D009F1FF3919F0FF09C6EB05056A
:103D08004FF00108D7D102E0B8F1000F00D0FEE76C
:103D1800BDE8FE8F00C0FFF7004000089C7F000848
:103D2800D8C0002002484FF43971FFF7B5BF00BF73
:103D3800D8C0002008B504484FF43971FFF790FF48
:103D4800BDE80840FFF79CBFD8C0002073B50B4EF4
:103D5800451E002404F50E7189190631022201A8B6
:103D6800FDF75AFF0021102201A8FEF7C7FA033415
:103D7800122C05F8010FEDD17CBD00BFD8C0002082
:103D880070B5074C06460D46282200212046FDF74F
:103D9800B3FC204631462A46BDE87040FDF7F2BB29
:103DA800EEC2002000F1080343604FF0FF32C36009
:103DB800036100238260036070470023036170473A
:103DC800436808619A684B608A609A6899600368DA
:103DD80051600133036070470A68531C30B501D144
:103DE800036907E000F1080300E023465C682568E2
:103DF8009542FAD95A6808614A60916059608B60A7
:103E080003680133036030BD4168826803698A60D2
:103E1800826851605968814208BF5A600022026175
:103E28001868013818607047026C30B503466AB1EB
:103E3800C4684568A418AC42C46024BF0468C46060
:103E48000846D968BDE83040FDF79CBB30BD38B5A1
:103E5800044604F1240500F06BFF0AE0636A5BB1D5
:103E6800284600F00BFE08B100F082FEA36C013B6F
:103E7800A364A36C002BF1DC4FF0FF33A36400F0C4
:103E880083FF04F1100500F053FF0AE023695BB1DA
:103E9800284600F0F3FD08B100F06AFE636C013BB0
:103EA8006364636C002BF1DC4FF0FF336364BDE89F
:103EB800384000F069BF38B51546026C04463AB977
:103EC800056805B128E0406800F0A4FE656024E0BC
:103ED8006DB98068FDF756FBA268236CD318626839
:103EE800A360934218D323682846A36015E0C068EE
:103EF800FDF748FB236CE26821685B42D2188A42CE
:103F0800E26002D26268D318E360022D04D1A36B89
:103F180013B1A36B013BA3630020A36B0133A3631D
:103F280038BD38B50D46044610B900F0F9FEFEE775
:103F380000F0FEFE2368E06B226CA36000FB0231F8
:103F4800013802FB00336160E36000214FF0FF336A
:103F5800A1636364A36455B9236983B104F11000B4
:103F680000F08CFD01280AD100F0CEFE07E004F134
:103F78001000FFF717FF04F12400FFF713FF00F00C
:103F880003FF012038BDF8B50D461746064610B99F
:103F980000F0C6FEFEE711B14843013000E00846D4
:103FA800543000F0D3FF044638B10DB9206007E063
:103FB80000F15403036003E0FEE700F0B1FEFBE705
:103FC800E663256420460121FFF7ABFF84F85070B3
:103FD8002046F8BD10B50C4610B900F0A1FEFEE76A
:103FE800814202D900F09CFEFEE700210222FFF781
:103FF800CAFF10B1846310BDFEE700F091FEFBE735
:104008002DE9F04385B00F4601921D46044610B9CC
:1040180000F086FEFEE7002977D1036C002B74D0F0
:1040280070E0FEE7E36B012B72D102E0FEE70126A8
:1040380002E000264FF0000800F07AFEA26BE36B66
:104048009A4201D3022D15D1204639462A46FFF758
:1040580032FF636A43B104F1240000F00FFD012828
:1040680004D100F051FE01E00028FAD100F08CFEE6
:10407800012050E0DDF80490B9F1000F02D100F002
:1040880083FE3DE016B902A800F034FD00F07CFE86
:1040980000F024FB00F04CFE636C013308BFC4F849
:1040A8004480A36C013308BFC4F8488000F06CFE5C
:1040B80002A801A900F02EFDE8B900F039FED4F8F5
:1040C8003890E66B00F060FEB1450ED104F11000A7
:1040D800019900F09FFC2046FFF7B9FE00F09AFB1B
:1040E8000028A4D100F010FEA1E72046FFF7AFFE9C
:1040F80000F090FB9BE72046FFF7A9FE00F08AFB43
:10410800002008E000F00CFE8BE7022D91D189E732
:1041180000F006FE8AE705B0BDE8F08370B50646F4
:10412800542000F013FF044608B103E0FEE700F056
:10413800F7FDFBE701230025C3634FF0FF338563D9
:1041480045604364056083648560C560056480F8E4
:1041580050601030FFF726FE04F12400FFF722FE1E
:10416800204629462A462B46FFF74AFF204670BDBF
:104178002DE9F0410F4616461D46044610B900F0D9
:10418800CFFDFEE741BB036C33B322E0FEE7E36BF0
:10419800012B24D126E0FEE7022D18D1204639460E
:1041A8002A46FFF788FEA36C01330BD1636A03B973
:1041B8000BE004F1240000F061FC30B12EB10124C1
:1041C800346019E0A36C0133A364012414E00024D3
:1041D80012E000F0A5FDD9E7022D03D1D7E700F0E2
:1041E8009FFDD8E700F06CFE00F09AFDA26BE36B30
:1041F8009A428046D0D2D1E7404600F0C1FD204621
:10420800BDE8F081F8B50D46044610B900F088FD08
:10421800FEE7066C16B100F083FDFEE700F050FEE5
:1042280000F07EFDA26BE36B9A42074616D2A36BA1
:104238000133A363A36C01330BD1636A03B90BE0A9
:1042480004F1240000F01AFC30B12DB101242C60D7
:1042580005E0A36C0133A364012400E0344638462A
:1042680000F08EFD2046F8BD2DE9F04385B00D46DF
:1042780001929946044610B900F052FDFEE729B9AB
:10428800036C2BB17EE0FEE7012603E0002600E088
:104298000E46002700F04CFDA36B3BB32046294691
:1042A800E668FFF7C1FDB9F1000F12D1A36B013B1E
:1042B800A363236813B900F0EBFC606023698BB13A
:1042C80004F1100000F0DAFB01280BD100F01CFD0E
:1042D80008E0636AE6602BB104F1240000F0CEFB2D
:1042E8000028F3D100F050FD01204EE0DDF80480F5
:1042F800B8F1000F02D100F047FD41E016B902A85D
:1043080000F0F8FB00F040FD00F0E8F900F010FDC7
:10431800636C013308BF6764A36C013308BFA764EB
:1043280000F032FD02A801A900F0F4FB18BB00F070
:10433800FFFCA66B00F028FDBEB9236833B900F076
:10434800F7FC606800F01AFC00F01EFD04F1240080
:10435800019900F05FFB2046FFF779FD00F05AFA5B
:10436800002891D100F0D0FC8EE72046FFF76FFDC2
:1043780000F050FA88E72046FFF769FD00F04AFA96
:10438800002002E000F0CCFC7DE705B0BDE8F0833A
:1043980010B5044610B900F0C3FCFEE700F0C8FCF5
:1043A800A36BE46BE41A00F0EFFC204610BD00009C
:1043B800064A13681968064B11B94FF0FF3203E03B
:1043C8001268D268D26852681A607047FC040020EC
:1043D800AC0100200E4B1A6810B550600D4A1268E7
:1043E8009042044607D20C4A106819680431BDE8A7
:1043F8001040FFF7F1BC094A106819680431FFF74B
:10440800EBFC074B1A68944238BF1C6010BD00BF14
:10441800AC050020C8050020CC050020FC040020C5
:10442800AC0100202DE9F84F0A9DDDF82C800C9E88
:104438000F4693469A46814610B900F071FCFEE794
:10444800042D02D900F06CFCFEE736B9900000F0AC
:104458007DFD0646002800F09E805C2000F076FD79
:10446800044678B106634FEA8B023046A521FDF772
:1044780043F9236B0BF1FF3B03EB8B0B2BF0070B83
:10448800002603E0304600F0E7FD84E0A319BA5D9A
:1044980083F83420BB5D13B10136102EF6D1002607
:1044A800271D384684F84360E562E5642665FFF712
:1044B80084FC04F11800FFF780FCC5F1050366656C
:1044C8002461A361646284F858605846494652469C
:1044D80000F0FAFB2060B8F1000F01D0C8F80040E6
:1044E80000F026FC2E4A1368013313602D4B1E681A
:1044F80036BB1C601368012B2AD1DFF8D0804FF03F
:10450800140909FB06800136FFF74CFC052EF8D18B
:10451800DFF8BC80244E4046FFF744FC3046FFF7E6
:1045280041FC2248FFF73EFC2148FFF73BFC2148AD
:10453800FFF738FC204BC3F80080204B1E6007E0D3
:104548001F4A126822B91A68D26AAA4298BF1C6028
:104558001C4A1368013313601B4A6364E36A1168D9
:10456800012404FA03F001431160184A142000FBE7
:1045780003203946FFF724FC00F006FC104B1B68AB
:1045880033B1084B1B68DB6AAB4201D200F0BCFBBD
:104598002046BDE8F88F4FF0FF30BDE8F88F00BF28
:1045A800D4050020AC0500201C050020B005002023
:1045B80098050020D8050020FC040020CC05002028
:1045C80000050020D0050020EC050020340500205F
:1045D8000805002038B5044600F0AAFB0CB9224BA8
:1045E8001C68251D2846FFF70FFC68B9E26A1F49B9
:1045F80014235343CB583BB91D4B0120196800FACB
:1046080002F221EA02021A60A36A1BB104F118003F
:10461800FFF7FAFB17482946FFF7D2FB164B1A6833
:1046280001321A60154B1A6801321A6000F0ACFBAF
:10463800134B1B68002B15D00B4B1B689C4209D1F0
:10464800104B1B6813B100F06BFBFEE7BDE8384068
:1046580000F05ABB00F06CFBFFF7AAFEBDE838403B
:1046680000F092BB38BD00BFAC0500203405002027
:10467800EC0500209805002004050020D005002046
:1046880000050020C405002030B585B00024802234
:1046980000940194029403940C480D492346FFF7B3
:1046A800C1FE012805460AD100F03AFB094B1D60FE
:1046B800094B1C6005B0BDE8304000F0BDBB10B927
:1046C80000F02EFBFEE705B030BD00BFF54802083C
:1046D80054FC020800050020C8050020024B1A6897
:1046E80001321A60704700BFC4050020014B1868EA
:1046F800704700BFC80500203B4B1B682DE9F047F9
:10470800002B5BD1394B1A6801321A601E688EB9CA
:10471800374B1A68126812B100F002FBFEE7354AFF
:10472800196810681860344B11601A6801321A60F1
:10473800FFF73EFE314B1B6800249E4200D232E058
:104748002B4FDFF8CC80DFF8BCA03B681B68002B40
:104758003AD12A4B4FF0FF321A6024E0274A1360FF
:1047680021E005F104094846FFF74EFBAB6A1BB18F
:1047780005F11800FFF748FBEB6AD8F80010012292
:1047880002FA03F214200A4300FB03A04946C8F8C2
:104798000020FFF715FB1A4BEA6A1B68DB6A9A428E
:1047A80028BF0124D1E7164B1B68DB6A1422534348
:1047B800144AD358012B88BF01240CE0124B1A6805
:1047C80001321A60002406E03B68DB68DD686B682C
:1047D8009E42C6D2C2E70D4B1B68002B18BF0124AE
:1047E8002046BDE8F08700BFC4050020C8050020AA
:1047F800FC040020CC050020F8040020AC010020B7
:10480800AC0500203405002030050020F00500200C
:10481800EC0500202DE9F8432C4C236813B900F06F
:104828007FFAFEE700F084FA2368013B23602368DF
:104838000BB1002444E0264B1B680BBBF9E7F36877
:10484800DC6804F1040804F11800FFF7DDFA4046BB
:10485800FFF7DAFAE36A2A68012707FA03F1142056
:104868000A4300FB039041462A60FFF7A9FA194B57
:10487800E26A1B68DB6A9A4206D3174B1F6003E0A3
:10488800164E174DDFF860903368002BD7D1154CC2
:1048980023686BB9104B1C68012CCAD10EE0FFF7D6
:1048A8002BFF08B1012333602B68013B2B6001E02B
:1048B800094E25462368002BF1D1EBE700F024FAD6
:1048C80000F062FA2046BDE8F88300BFC405002066
:1048D800D4050020AC050020F0050020B00500201C
:1048E800EC0500203005002034050020F8B5144CF4
:1048F800144E154F2368E3B1FFF7F0FE3568FFF754
:1049080089FF002DF6D000F013FAF368DD68281D42
:10491800FFF77AFA3B68013B3B602368013B236061
:1049280000F032FA286B00F097FB284600F094FB61
:10493800E0E7064B1B68012BDCD900F0E5F9D9E765
:104948000405002098050020D40500203405002027
:1049580038B5044618B9BDE8384000F0D5B9114B50
:104968001B6813B100F0DCF9FEE7FFF7B7FE0E4B4A
:104978001D6865190D4C20680430FFF745FA48B9E1
:104988000B4B19682268D26A012000FA02F221EA68
:1049980002021A602846FFF71DFDFFF73BFF0028BB
:1049A800D9D038BDC4050020C8050020AC050020BA
:1049B800EC05002008B5124B1A68124B0AB1012207
:1049C8001CE01A60104B1A68B2FA82F2D2B21423B1
:1049D800C2F11F020D495A438B188A5812B900F0C8
:1049E8009FF9FEE75A68526803F108018A425A6043
:1049F80004BF52685A605B68DA68054B1A6008BDE4
:104A0800C4050020F0050020EC0500203405002036
:104A1800AC05002038B50D4610B900F081F9FEE765
:104A2800124C21681831FFF7D7F920680430FFF7D6
:104A3800EBF948B90E4B19682268D26A012000FACE
:104A480002F221EA02021A60691C07D1074B0948E1
:104A580019680431BDE83840FFF7B2B9064B186849
:104A68002818BDE83840FFF7B5BC00BFAC050020EA
:104A7800EC050020D8050020C805002038B5C3681B
:104A8800DC6814B900F04CF9FEE704F11805284673
:104A9800FFF7BAF9114B1B6883B9251D2846FFF7A4
:104AA800B3F90F4AE36A1068012101FA03F10143DF
:104AB80011600C4A142000FB032000E00A48294634
:104AC800FFF77EF9094BE26A1B68DB6A9A4203D951
:104AD800074B0120186038BD002038BDC4050020F0
:104AE800EC05002034050020B0050020AC050020AE
:104AF800F005002008B510B900F012F9FEE7034BE5
:104B08001B680360024B1B68436008BDF804002063
:104B1800C805002038B50D46044610B900F000F964
:104B2800FEE711B900F0FCF8FEE700F001F90E4BC2
:104B38001A682B68591C10D00C49086821688842EB
:104B4800616801D08A420AD2501A984207D28A1A5A
:104B5800D3182B602046FFF7CDFF002400E0012486
:104B680000F012F9204638BDC8050020F8040020DE
:104B7800014B01221A607047F0050020F8B5044681
:104B8800002840D0204AC36A1168C96A8B423AD2C9
:104B98008169002904DB1268D26AC2F105028261C8
:104BA8001A4E6269142707FB03639A4227D11FE054
:104BB800E26A5743F3593BB9154B0120196800FACB
:104BC80002F221EA02021A600F4B114A1B681068B0
:104BD800DB6A012101FA03F1014311600B4AE36228
:104BE800142000FB03202946BDE8F840FFF7E8B889
:104BF800251D2846FFF708F90028D9D0E4E7024B1D
:104C08001B68DB6AE362F8BDAC05002034050020B0
:104C1800EC05002038B5044608B9002038BD036DFE
:104C280013B900F07DF8FEE7C16AC26C013B9142FE
:104C38000365F2D0002BF0D1051D2846FFF7E4F8F4
:104C480068B9E26A104914235343CB583BB90F4B58
:104C58000120196800FA02F221EA02021A60E36CE4
:104C6800C3F10502A261094AE3621168012404FA4A
:104C780003F001431160044A142000FB0320294675
:104C8800FFF79EF8204638BD34050020EC050020CB
:104C9800044B1A681AB11A68116D01311165186848
:104CA800704700BFAC05002006480068006880F324
:104CB800088862B661B6BFF34F8FBFF36F8F00DF0E
:104CC80000BF000008ED00E04FF0807300E90A0023
:104CD800034B40F8202C40F80C3C4038704700BF8C
:104CE8006D4D0208074B19680868B0E8F00F80F3AB
:104CF8000988BFF36F8F4FF0000080F311884EF0E2
:104D08000D0E7047AC050020044B4FF080521A601E
:104D1800BFF34F8FBFF36F8F704700BF04ED00E004
:104D2800EFF311804FF0500181F311887047002094
:104D380008B5FFF7F5FF094A136801331360BFF39D
:104D48004F8FBFF36F8F012B07D1054B1B6813F0F3
:104D5800FF0F02D0FFF7E4FFFEE708BDB001002017
:104D680004ED00E008B5054B1B68013302D0FFF7DE
:104D7800D7FFFEE7FFF7D4FFFEE700BFB001002032
:104D880080F311887047000008B5074B186810B900
:104D9800FFF7C6FFFEE70138186018B9BDE80840FC
:104DA800FFF7EEBF08BD00BFB0010020EFF3098098
:104DB800BFF36F8F0D4B1A6820E9F00F10602DE9D3
:104DC80008404FF0500080F31188FFF7F3FD4FF0D3
:104DD800000080F31188BDE8084019680868B0E849
:104DE800F00F80F30988BFF36F8F7047AC05002080
:104DF80008B5FFF795FFFFF77FFC18B1044B4FF09C
:104E080080521A600020BDE80840FFF7B9BF00BF14
:104E180004ED00E0064B1A684FF47A73B2FBF3F224
:104E2800044B013A1A60072243F8042C704700BF6C
:104E38000801002014E000E007B51D4B1A78019224
:104E4800FF221A701B788DF803309DF80320194B48
:104E580002F050021A70184A0723136005E09DF803
:104E680003305B008DF803300B469DF80320591E74
:104E78001206F4D4104A1B0203F4E06313600C4BCF
:104E8800019A1A70D3F8202942F47002C3F8202935
:104E9800D3F8202942F07042C3F82029FFF7BAFF5F
:104EA800064B00221A60FFF7FFFEFFF75BFF00BF0B
:104EB80000E400E0F4050020F8050020B00100201F
:104EC80008B5EFF305830F2B08D90A4A9B5C0A4AF9
:104ED80012789A4202D9FFF723FFFEE7074B1A68B8
:104EE800074B1B6802F4E0629A4202D9FFF718FFE9
:104EF800FEE708BDF0E300E0F40500200CED00E05B
:104F0800F805002010B50F4B00E013461A688242DE
:104F1800FBD359685C18844203D140684118596032
:104F2800184641684418944206D1074C2468A242A6
:104F380002D014CA611841608342026018BF186029
:104F480010BD00BF0406002000060020F8B5054685
:104F5800FFF7C4FB3A4B1B681BBB3A4A560707D0FE
:104F6800D31D23F0070302F57042D11A1A4601E057
:104F78004FF470415118083921F0070132480023D5
:104F880080E80C000B604B608B1A82E80A002F4AFD
:104F98002B4813602E4A016013602E4B4FF00042DD
:104FA8001A602C4B1E68354240D1002D3FD005F1C8
:104FB800080358071CBF23F007030833002B33D01E
:104FC800234A1768BB4231D81F4A146801E02246B9
:104FD80004466168994204D319480068844204D1A0
:104FE80024E020680028F2D1F6E7206815681060F0
:104FF800CA1A0835102A09D9E018410702D0FFF764
:105008008FFEFEE742606360FFF77CFF626810492D
:10501800BB1A0B600D490868834238BF0B60164302
:10502800002384E8480002E01D4600E00025FFF761
:10503800F1FB6B0702D0FFF773FEFEE72846F8BDC9
:105048000006002000000010040600200C060020C6
:10505800FC0500201006002010B5044610B3124AC3
:1050680050F8043C12681A4202D1FFF759FEFEE7D5
:1050780050F8081C11B1FFF753FEFEE723EA0203BC
:1050880040F8043CFFF72AFB084B54F8041C1A6844
:10509800A4F108008A181A60FFF734FFBDE8104031
:1050A800FFF7B8BB10BD00BF10060020FC050020AC
:1050B80070B5094C06460D4630466168FCF7A8FBFA
:1050C80028B9A3682B60E36801206B6070BD246871
:1050D800002CF1D1204670BDDC2F030838B508201C
:1050E8000C4601F009FF0146A0B1002505604560A6
:1050F800204602F06FFB2046084902F06DFB20466F
:10510800074902F06DFB204606490A2202F06DFBB2
:10511800284600E0FF2040B238BD00BF795602089B
:10512800735102085B51020838B54B68B0F86650F5
:105138009D4228BF9DB20C462A460968002303F009
:10514800AEFE28B923685B19236063685D1B656040
:1051580038BD08B50346084613B902F0D9FD02E088
:105168001946FFF7E1FF002008BD01F0FDBD38B585
:1051780004460D46002102F02DFB2046002102F0D6
:105188002DFB2046002102F027FB284601F0ECFD0C
:105198002046BDE8384002F0BBBD08B503460846C6
:1051A8005A68194612B1FFF7BFFF01E0FFF7DFFFAA
:1051B800002008BD10B502F0D9FE50220446064969
:1051C80002F036FAFF21204602F06AFA0349BDE8E8
:1051D800104002F008BB00BF64690308E5500208EC
:1051E80038B54FF4FA620C46084600211D46FCF714
:1051F80083FA204600F00CFE2046FCF755FC288078
:1052080038BD00002DE9F04190461F46FCF7CCFE62
:105218000546E0B10F49FCF731FD0F49064628461F
:10522800FCF72CFD044620B928460C49FCF726FD5E
:105238000446A51B013D4046711C2A46FCF7ECFCC0
:1052480030232370012033703D70BDE8F081387041
:10525800BDE8F081472E0308F52D0308F72D030854
:1052680030B5024695B00C4607A8114632221D46B5
:10527800FCF7D2FC0021142202A8FCF73DFA07A88B
:105288000B4902AA0DF10703FFF7BCFF70B10948EB
:1052980002A9FCF7BDFA28B931232370012000F0D8
:1052A800FBFD01E03023237001232B8015B030BDB6
:1052B800F92D0308032E030810B508490446FCF726
:1052C80073FE48B1021B92B2C2F5BB6200210332E1
:1052D800BDE81040FCF710BA10BD00BF0C2E030843
:1052E80030B587B0002405468DF80340FFF7E4FF8A
:1052F8002146142201A8FCF7FFF90DF103035649D2
:1053080001AA2846FFF77EFF01A8FEF7F7FB214612
:10531800142201A8FCF7F0F90DF103034F4901AA83
:105328002846FFF76FFF01A8FEF7EEFB214614227F
:1053380001A8FCF7E1F90DF10303494901AA284640
:10534800FFF760FF01A8FEF7E5FB2146142201A83C
:10535800FCF7D2F90DF10303424901AA2846FFF7E9
:1053680051FF01A8FEF7E4FB2146142201A8FCF72F
:10537800C3F90DF103033C4901AA2846FFF742FF90
:1053880001A8FEF7E3FB2146142201A8FCF7B4F9B3
:10539800364901AA0DF103032846FFF733FF01A898
:1053A800FEF79AFB01A832490222FCF7DFFB00282E
:1053B80031D02146142201A8FCF79EF90DF1030310
:1053C8002C4901AA2846FFF71DFF01A8FEF772FB2A
:1053D8002146142201A8FCF78FF90DF10303264991
:1053E80001AA2846FFF70EFF01A8FEF769FB214630
:1053F800142201A8FCF780F9204901AA0DF1030342
:105408002846FFF7FFFE01A8FEF760FB01A821462A
:105418001422FCF771F90021142201A8FCF76CF999
:1054280009F02CFDA0B10120FEF738FB00F02BFDA0
:1054380040F2F230FFF78CFABFF34F8F104A114B4E
:10544800D16801F4E0610B43D360BFF34F8FFEE7EF
:1054580000F019FD07B030BD112E0308212E0308F6
:10546800322E03083D2E0308492E0308552E030843
:10547800E6FB02085B2E0308632E0308672E030869
:1054880000ED00E00400FA052DE9F041064688B079
:105498000C46904631461E2268461F46FCF7BCFB68
:1054A80068460E49FCF7EAFB054670B929464FF4F1
:1054B800FA622046FCF720F9204600F031FB20462E
:1054C800FCF7F2FA3880284604E030464146FFF7F8
:1054D80007FF012008B0BDE8F08100BF6D2E03086A
:1054E800F0B5002587B006460C464FF4FA62084628
:1054F80029461F468DF80350FCF7FEF83046FFF7A3
:10550800DBFE2946142201A8FCF7F6F801AA0DF1E2
:1055180003030B493046FFF775FE9DF8031001A8F9
:10552800FEF72EFC01A8FDF73DFC06492046FCF7D6
:105538005DFA2046FCF7B8FA388007B0F0BD00BF26
:105548006F2E0308782E030870B504460D461646DC
:10555800FCF7AAFA234680B205E013F8012BAA4209
:1055680008BF03F8016C1A1B92B28242F5D370BDD2
:1055780030B59FB0002405468DF80740FFF79CFE24
:1055880021466E2202A8FCF7B7F80DF1070302AA1C
:1055980028461E49FFF736FE2B21202202A8FFF7D6
:1055A800D3FF02A8FEF7E0FA21466E2202A8FCF714
:1055B800A3F80DF1070302AA28461549FFF722FEB2
:1055C8002B21202202A8FFF7BFFF02A8FEF7DCFA72
:1055D80021466E2202A8FCF78FF80DF1070302AAF4
:1055E80028460C49FFF70EFE2B21202202A8FFF7C0
:1055F800ABFF02A8FEF7D6FA21466E2202A8FCF7F6
:105608007BF800F040FC1FB030BD00BFA82E030897
:10561800AF2E0308BC2E03082DE9F041064688B0DA
:105628000C46904631461E2268461F46FCF7F4FA9F
:1056380068460E49FCF722FB054670B929464FF427
:10564800FA622046FCF758F8204600F025FB204671
:10565800FCF72AFA3880284604E030464146FFF72E
:1056680087FF012008B0BDE8F08100BF6D2E030858
:105678002DE9F3411746002204460D460092019297
:10568800002B40F0E7800846002F00F0E0803989C1
:1056980002F06EF82368002B40F0D5807E683A89C6
:1056A8006E4B6F481A803146FBF76CFF30466D49E8
:1056B8000D22FCF75BFA08B96B48B5E030466B4938
:1056C8000E22FCF753FA08B96948ADE0304669493B
:1056D8001022FCF74BFA08B96748A5E0304667493D
:1056E8000C22FCF743FA08B965489DE03046654945
:1056F8001222FCF73BFA00B949E0304662490E2213
:10570800FCF734FA00B936E0304660491022FCF75D
:105718002DFA48B95E4E304600F0FCF82660304657
:10572800FCF7C2F9606086E030465A491122FCF75E
:105738001DFA70B9584BDFF85881584E4848022274
:105748001A70464B41461A883346FFF79DFEF0B95A
:1057580065E0304652490D22FCF708FA68B93F4B1C
:10576800DFF82C814D4E1A883D4841463346FFF7F5
:1057780053FF00B953E04B4856E030464A490E22E1
:10578800FCF7F4F928B900F077FB00F07CFB4748F8
:105798004AE0304646490F22FCF7E8F910B900F014
:1057A80074FB50E0304643491022FCF7DFF920B97A
:1057B800FEF774F9FEF778F935E030463E491222D3
:1057C800FCF7D4F950B9DFF8C880344E234B24488D
:1057D8001A8841463346FFF743FD20E030463749F3
:1057E8001322FCF7C3F950B9DFF8A4802B4E1B4BEA
:1057F8001B481A8841463346FFF772FE0FE03046D1
:105808002F490F22FCF7B2F968B9144BDFF88080F2
:10581800224E1A88124841463346FFF7E1FCC4F885
:105828000080338806E027486946FFF741FC009B63
:105838002360019B636028462146FFF775FC2846D4
:10584800214901F0CBFF384601F000FD28462146EA
:10585800FFF78DFC0020BDE8FC8100BF1606002084
:105868008CCB0020C52E0308C92E0308D32E0308AD
:10587800D72E0308E22E0308E62E0308F32E0308AA
:10588800F72E0308002F0308132F0308222F0308FD
:10589800BCC30020332F030814060020180600207C
:1058A800452F0308172F0308532F0308042F030855
:1058B800622F0308722F03088F2F0308A22F0308F3
:1058C800B62F0308832F0308A3510208BFF34F8F95
:1058D800044A054BD16801F4E0610B43D360BFF380
:1058E8004F8FFEE700ED00E00400FA0508B50378E5
:1058F80033B1FEF7CDF8FEF715FA012009F0A2FB47
:105908004FF47A70FFF724F840F2F230FFF720F8EE
:10591800FFF7DCFF10B54FF47A728CB00446002113
:10592800FBF7EAFE20466E49FCF760F802A80DF185
:105938000701FDF7EDFE20466A49FBF743FF9DF896
:10594800072002A92046FCF7DFF802A80DF107019D
:10595800FDF7E4FE20466449FBF734FF9DF8072075
:1059680002A92046FCF7D0F802A80DF10701FDF7BF
:10597800C3FE20465D49FBF725FF9DF8072002A9D5
:105988002046FCF7C1F802A80DF10701FDF7BAFEA1
:1059980020465749FBF716FF9DF8072002A9204625
:1059A800FCF7B2F802A80DF10701FDF7BDFE20468D
:1059B8005049FBF707FF9DF8072002A92046FCF78E
:1059C800A3F802A80DF10701FDF792FE20464A4907
:1059D800FBF7F8FE9DF8072002A92046FCF794F88B
:1059E80002A80DF10701FDF786FE20464349FBF7A3
:1059F800E9FE9DF8072002A92046FCF785F802A8D1
:105A08000DF10701FDF796FE20463D49FBF7DAFE4A
:105A18009DF8072002A92046FCF776F802A80DF1A8
:105A28000701FDF793FE20463649FBF7CBFE9DF8AC
:105A3800072002A92046FCF767F802A80DF1070124
:105A4800FDF77EFE20463049FBF7BCFE9DF8072097
:105A580002A92046FCF758F802A80DF10701FDF746
:105A68007BFE20462949FBF7ADFE9DF8072002A9D9
:105A78002046FCF749F802A80DF10701FDF76FFE73
:105A880020462349FBF79EFE9DF8072002A92046E1
:105A9800FCF73AF802A80DF10701FDF763FE20466E
:105AA8001C49FBF78FFE9DF8072002A92046FCF74A
:105AB8002BF802A80DF10701FDF7D0FF2046164983
:105AC800FBF780FE02A99DF807202046FCF71CF88A
:105AD800204612490222FCF717F80CB010BD00BF8F
:105AE800D4660308006703080867030811670308FA
:105AF8001F6703082E67030838670308476703080A
:105B0800576703086467030875670308896703080C
:105B18009B670308AC670308C7680308C0670308E6
:105B280010B551498AB00446FBF760FF02A80DF191
:105B38000701FDF727FF20464C49FBF743FE9DF878
:105B4800072002A92046FBF7DFFF02A80DF1070195
:105B5800FDF728FF20464649FBF734FE9DF807204D
:105B680002A92046FBF7D0FF02A80DF10701FDF7B7
:105B780029FF20463F49FBF725FE9DF8072002A98B
:105B88002046FBF7C1FF02A80DF10701FDF72AFF28
:105B980020463949FBF716FE9DF8072002A9204642
:105BA800FBF7B2FF02A80DF10701FDF72BFF204616
:105BB8003249FBF707FE9DF8072002A92046FBF7AC
:105BC800A3FF02A80DF10701FDF786FE20462C4928
:105BD800FBF7F8FD9DF8072002A92046FBF794FF84
:105BE80002A80DF10701FDF78DFE20462549FBF7B8
:105BF800E9FD9DF8072002A92046FBF785FF02A8CA
:105C08000DF10701FDF794FE20461F49FBF7DAFD69
:105C18009DF8072002A92046FBF776FF02A80DF1A0
:105C28000701FDF79BFE20461849FBF7CBFD9DF8C1
:105C3800072002A92046FBF767FF02A80DF107011C
:105C4800FDF70CFF20461249FBF7BCFD02A99DF8A1
:105C580007202046FBF758FF20460E490222FBF793
:105C680053FF0AB010BD00BFD4660308C36703081A
:105C7800D7670308ED670308FD6703080E68030884
:105C88001F6803082C680308356803084068030880
:105C9800C7680308C067030810B551498CB00446AB
:105CA800FBF7A4FE02A80DF10701FDF75FFD2046F2
:105CB8004C49FBF787FD9DF8072002A92046FBF712
:105CC80023FF02A80DF10701FDF776FD204646499E
:105CD800FBF778FD9DF8072002A92046FBF714FF83
:105CE80002A80DF10701FDF779FD20463F49FBF7B2
:105CF80069FD9DF8072002A92046FBF705FF02A8C9
:105D08000DF10701FDF77CFD20463949FBF75AFDE7
:105D18009DF8072002A92046FBF7F6FE02A80DF120
:105D28000701FDF77FFD20463249FBF74BFD9DF843
:105D3800072002A92046FBF7E7FE02A80DF107019C
:105D4800FDF782FD20462C49FBF73CFD9DF8072016
:105D580002A92046FBF7D8FE02A80DF10701FDF7BE
:105D680085FD20462549FBF72DFD9DF8072002A952
:105D78002046FBF7C9FE02A80DF10701FDF788FDD3
:105D880020461F49FBF71EFD9DF8072002A9204663
:105D9800FBF7BAFE02A80DF10701FDF78BFD2046BF
:105DA8001849FBF70FFD9DF8072002A92046FBF7CD
:105DB800ABFE02A80DF10701FDF750FE204612497F
:105DC800FBF700FD02A99DF807202046FBF79CFE83
:105DD80020460E490222FBF797FE0CB010BD00BF0B
:105DE800D46603084A68030856680308626803080B
:105DF80070680308806803088E6803089A680308B7
:105E0800A6680308B8680308C6680308C0670308DB
:105E180010B5154986B00446FBF7E8FD134920463E
:105E2800FBF7D0FC684605F003FD009B6422B3FB3A
:105E3800F2F30021142201A80093FBF75DFC009AFD
:105E48000B4901A8FDF748FC01A8FBF72DFE01A9A5
:105E580002462046FBF758FE204606490222FBF779
:105E680053FE06B010BD00BFD46603084A68030895
:105E7800E0680308C067030808B5FDF7DFFEBDE862
:105E88000840FDF74FBFFDF74DBF08B540F2F230AF
:105E9800FEF75EFDFFF71AFD1FB5074B074918709F
:105EA8000022009201920292039205488022FEF796
:105EB800B9FA05B000BD00BF1A060020E368030860
:105EC800F55802081E4B1B6807B513B11D4A106828
:105ED80098471D4801A903F00DFD019B1A78052A72
:105EE800F7D8DFE802F00307151B20289868036835
:105EF8000430EDE7D968986891F82D2012F0600F0A
:105F080002D008F051FB01E004F04EF908200EE041
:105F180003F1080007C803F01FFC07E0D8681969F7
:105F280003F0C4FC02E09A68D868904707200199FA
:105F380001F082F8CDE79A68D8689047C9E700BFB2
:105F480024060020200600201C060020F8B50E4D6F
:105F58002B6806460F4693B1082001F057F804460F
:105F680078B1012303708660C7602146284608F08F
:105F780069FD38B10820214601F05EF801E0FA20F9
:105F880000E0FF2040B2F8BD1C06002037B50446EB
:105F98000D4600F0B3FE094B09481C60094B32213D
:105FA8001D6008F041FD03230093074907480022BC
:105FB8004FF4C87308F0B7FD3EBD00BF24060020AB
:105FC8001C06002020060020CD5E0208EE680308AB
:105FD800030A43EA002080B27047030A43EA00201C
:105FE80080B2704700BA7047FFF7FCBF037B8B4253
:105FF80003D000230173437343837047038B10B5A9
:106008004469E41884F8F01041695C1C11FA84F1C1
:10601800023381F8F020038310BD038B4269D21844
:10602800013382F8F01003837047038B4269D2185A
:1060380010B50C0A82F8F04042695C1C12FA84F22E
:10604800023382F8F010038310BD038B4269D21823
:1060580010B50C0E82F8F04042695C1C12FA84F20A
:10606800C1F3074482F8F04042699C1C12FA84F29A
:10607800C1F3072482F8F0404269DC1C12FA84F26A
:10608800043382F8F010038310BD90B1038B42698A
:10609800D218FF21013382F8F0100383002105E0B4
:1060A8004269D218013382F8F0100383038B432B23
:1060B800F6D970472DE9F0410C46174606460028E8
:1060C80000F08E80002900F08D8000204FF49A7136
:1060D800024601F008F92061002800F08580627B03
:1060E800434B12B91A6801321A601B684268236070
:1060F80001236261137062695370636996F8262000
:106108009A7063690025DD702068D4F81480FFF761
:1061180069FFC8F804006369082F1D725D729D72DB
:10612800DD721D735D739D73DD7307D0042F05D079
:10613800032F05D1227B043A012A01D87268DA605C
:1061480000251D745D749D74DD741D755D759D75E8
:10615800DD751D765D769D76DD7696F8261062698A
:10616800ABB2994288BF73192A448CBF93F8273081
:1061780000230135102D1377EFD1002319466269EA
:10618800D2180133402B82F82C10F8D10022104687
:106198006369991801320023802A81F86C00F7D1CD
:1061A80062696FF07D00632182F8ED00532082F868
:1061B800EC1082F8EE0082F8EF1023836269D2189F
:1061C80082F8F0300133442BF8D1204635210122E2
:1061D800FFF714FF20463946FFF71FFF002004E0B1
:1061E800F22002E0FA2000E0FF2040B2BDE8F08192
:1061F800B401002010B5044630B1006908B101F0BF
:1062080025F800232361636110BD000073B5046A9B
:1062180000230546636220460621FFF7E7FE28466D
:1062280021460122FFF746FF0646002830D1022208
:1062380020463921FFF7E2FE2046A98CFFF7F5FE3C
:10624800042220463721FFF7D9FE20460121FFF717
:10625800E4FE20460321FFF7E0FE20461C21FFF75D
:10626800DCFE06212046FFF7D8FE2046FFF70DFF8B
:10627800218B2069F03189B201F00FF80095606830
:1062880021690F4A432303F081FC2046FFF7B2FF40
:10629800637B0133DBB2052B98BF4FF47A726373CB
:1062A8009ABF02FA03F39BB24EF660234FF4FA72D8
:1062B80003F2F31393FBF2F3638330467CBD00BF14
:1062C8006069030873B5046A054604212046FFF790
:1062D8008DFE284621460322FFF7ECFE0646D8B974
:1062E800022220463921FFF789FEA98C2046FFF7B4
:1062F8009CFE2046FFF7C9FE218B2069F03189B248
:1063080000F0CBFF0095606821690E4A432303F033
:106318003DFC2046FFF76EFF637B0133DBB2092BA0
:10632800637304D84FF47A7253439BB201E042F28C
:1063380010734FF4FA7203F2F31393FBF2F36383CF
:1063480030467CBD6069030873B5046A05460321BD
:106358002046FFF74BFE284621460322FFF7AAFEF8
:10636800064640BB022220463921FFF747FE204659
:106378004FF41071FFF759FE042232212046FFF72F
:106388003DFE606AFFF730FE01462046FFF75DFEDE
:106398002046FFF77AFE218B2069F03189B200F0A0
:1063A8007CFF0095606821690E4A432303F0EEFBE9
:1063B8002046FFF71FFF637B0133DBB2092B6373B2
:1063C80004D84FF47A7253439BB201E042F210733F
:1063D8004FF4FA7203F2F31393FBF2F3638330463C
:1063E8007CBD00BF6069030873B5046A05460121D6
:1063F8002046FFF7FBFD284621460322FFF75AFEF9
:106408000646002848D1022220463921FFF7F6FD2A
:106418002046A98CFFF709FE042232212046FFF707
:10642800EDFD606AFFF7E0FD01462046FFF70DFE2F
:10643800042236212046FFF7E1FD206AFFF7D4FD4C
:1064480001462046FFF701FE042220463721FFF7C8
:10645800D5FD20460121FFF7E0FD20460321FFF787
:10646800DCFD20461C21FFF7D8FD06212046FFF75A
:10647800D4FD2046FFF709FE218B2069F03189B24F
:1064880000F00BFF0095606821690F4A432303F071
:106498007DFB2046FFF7AEFE637B0133DBB2052BA5
:1064A80098BF4FF47A7263739ABF02FA03F39BB2F0
:1064B8004EF660234FF4FA7203F2F31393FBF2F3F0
:1064C800638330467CBD00BF6069030838B5046A41
:1064D800054608212046FFF789FD284604F12401D6
:1064E800002207F041FF637B013363730123638359
:1064F80038BD37B50546002859D0046A002C56D057
:10650800636B581C0DD03C221E33B3FBF2F34FF6DD
:10651800FF72934228BF13469BB2A3830BB9012392
:10652800A383A36B591C0DD03C221E33B3FBF2F39B
:106538004FF6FF72934228BF13469BB2E3830BB911
:106548000123E383E38BA28B9A4202D30BB100238E
:10655800A383A37B0BB1A36A0BE094F824301A063B
:1065680001D4FF2305E0BF2B8CBF6FF07F434FF6AC
:10657800FF730093E36A01932BB9636A009A13408F
:1065880043F080730193284604F1240100F06AFD6A
:106598002846694600F0A6FD01A9284600F09EFDA0
:1065A800284600F0F5FD20460A21FFF71FFD3EBDF5
:1065B8002DE9F04F92468BB0BAF80A30D0F8208017
:1065C80052682B2B054640F2B8811378022B40F015
:1065D800B48190F82610002308E0E8180133D41895
:1065E80090F82700E47E844240F0A781D8B2884220
:1065F800F3D35068FFF7F8FCD8F80030984240F021
:106608009C8100210A229D48FBF776F8BAF80A30E7
:106618002B2B40F29281DAF80430BAF80890C8F8C7
:1066280008304FF0000BF02204E04FF0000B4FF061
:106638006C092C22574609E03F68D21AC3EB0909B6
:1066480092B21FFA89F9002F00F077817B899A426C
:10665800F2D278680390DBE07B89501C984203DA19
:10666800039883185B7803E03B680BB15B681B7881
:10667800332938D007D8012919D011D303291DD0BF
:10668800062955D121E036293DD004D8342931D006
:1066980035294DD135E03A293CD03B2948D140E055
:1066A800511E002389B24FF0FF341E4644E0042BEC
:1066B80040F043811E46114606243DE0032B40F27C
:1066C8003C8111460724042636E0990740F03581BD
:1066D800082B34BF1E460826F6B2B342C0F02D81FF
:1066E8001146082428E0042B40F027811E46114655
:1066F800032421E0012B40F020811E46114600248E
:106708001AE0012B07E0042B40F017811E461146C2
:10671800022411E0042B40F010811E4611461C464D
:106728000AE0042B40F009811E461146052403E0C7
:1067380011464FF0FF340026023113FA81F39BB261
:106748000193002E4FD0023292B20AA9059200237B
:106758004B4A41F8043D02EB8402049106920293ED
:1067680005980299454A43184448A2180792225CA2
:10677800C1EB060C9BB25FFA8CFC002A33D1BCF14A
:10678800030F94BF6246042238460499CDF800C02E
:1067980000F0AAFEDDF800C0BCF1040F0FD91CF010
:1067A800030F40F0CA800799099801220A70FFF781
:1067B80019FC029B06990134C8500433CFE704D171
:1067C8000998FFF711FC099006E0BCF1010F40F0B1
:1067D800B4809DF824300993284A29480123135589
:1067E800099B40F824307B89019999420FD3CA1A32
:1067F800C3EB090992B21FFA89F94A45019203D3FA
:106808001E4A137863B99FE03F687B680393019A37
:106818000398815CFF29F3D04A45FFF41DAFEFE7E9
:10682800174B16491B680022012B0A7000F0938051
:10683800022B3FF4FAAE032B40F0868089E0104A21
:106848001179052940D198F80C10012935D12C6A05
:10685800DB78C4F828B0C4F82CB00BB1D368236334
:10686800064B1A7912B1064A126901E0226B5208E6
:106878005B79626333B1024B5B6904E068D1002045
:1068880074D10020236BA363A368394A1B69636230
:10689800937916462BB1374B9869FFF7A3FB012371
:1068A800A062A373F37923B1324BD869FFF79AFB3F
:1068B800E0622846FFF70AFE3FE0033902293CD888
:1068C8002846FFF716FE38E0062921D198F80C3043
:1068D800052B32D898F90C304FF0B8429A402CD595
:1068E80028462C6A00F06EFC2846234900F0BAFBC3
:1068F8002846214900F0F2FB28461F4900F0F2FB28
:1069080020460C21FFF772FB2846FFF77FFC14E0B6
:10691800022912D198F80C1006290ED19B78A8F8F4
:106928001AB02C6A4BB19068FFF75CFBA368206231
:106938001B6928466362FFF757FD0023C8F8083033
:10694800504600F083FC10E0BBF1000F7FF46DAE01
:1069580005E04FF0010B4FF0EC096C226AE6044B9E
:106968005A78002A7FF46BAFE7E70BB0BDE8F08FE9
:1069780068D1002074D100206469030837B5054642
:10698800002837D0046A002C34D0237B082B31D15F
:106998000A68636A9A422DD120460C21FFF726FB2C
:1069A800284621460422FFF785FBF0B9042232214C
:1069B8002046FFF723FB606AFFF716FB01462046D7
:1069C800FFF743FB2046FFF760FB218B2069F0317E
:1069D80089B200F062FC009560682169064A432389
:1069E80003F0D4F82046FFF705FC637B013363739B
:1069F800142363833EBD00BF6069030873B5046A4E
:106A0800054605212046FFF7F1FA284621460322CC
:106A1800FFF750FB0646E0B9022220463921FFF76E
:106A2800EDFAA98C2046FFF700FB2046FFF72DFB67
:106A3800218B2069F03189B200F02FFC0095606845
:106A4800216904F12002432303F0A0F82046FFF750
:106A5800D1FB637B0133DBB2092B637304D84FF49A
:106A6800FA6253439BB201E044F620634FF4FA7292
:106A780003F2F31393FBF2F3638330467CBD00000B
:106A880038B5154B154D1C6823E0236A03B3DA8B20
:106A9800511E012AD9830BD11A7B0A2A18D893F9D7
:106AA8000C3015FA03F313D52046FFF70BFC0FE063
:106AB8009A8B511E012A99830AD11A7B0A2A07D870
:106AC80093F90C3015FA03F302D52046FFF796FF29
:106AD8002468002CD9D138BDB0E50020000020443E
:106AE80073B5046A054600212046FFF77FFA0023A4
:106AF80023626362A362E362A3636363236328463A
:106B080021460722FFF7D6FA064698B92046FFF72E
:106B1800BCFA218B2069F03189B200F0BEFB0095E8
:106B28006068216904F12002432303F02FF820460E
:106B3800FFF760FB637B0133DBB2092B637304D877
:106B48004FF47A7253439BB201E042F210734FF450
:106B5800FA7203F2F31393FBF2F36383284600F00F
:106B680031FB2846064900F07DFA2846044900F022
:106B7800B5FA2846024900F0B5FA30467CBD00BF98
:106B88006469030838B5264B00251C6844E0236A6D
:106B9800002B40D05A8B012A02D9013A5A833AE095
:106BA80039D11A7B5D830C2A28D0062A00D125E02A
:106BB800012A06D15B7B052B20461DD8FFF714FC64
:106BC80029E0082A09D15B7B012B204602D8FFF770
:106BD8007DFC20E0FFF78DFC1DE0052A03D120464F
:106BE800FFF70CFF17E0042A0AD15B7B082B20462D
:106BF80002D8FFF767FB0EE0FFF772FF204608E0B8
:106C0800032A08D15B7B012B204602D8FFF79CFBA7
:106C180001E0FFF7FBFA2468002CB8D138BD00BFAB
:106C2800B0E5002010B598B190F82D30046A23F033
:106C3800080380F82D305CB1606818B103F052F891
:106C48000023636020460021BDE81040FFF7CEB95D
:106C580010BD000038B5044608B9F22047E090F8A6
:106C68002D30056A23F0080203F02003DBB280F818
:106C78002D20002BF1D0838CB3F5107F00D22EE0AD
:106C880035B93C2000F038F9054640B3206203E0EE
:106C9800686808B103F026F800213C222846FAF774
:106CA8002BFD03F03BF86860C8B1037A114943F043
:106CB800200303724422686802F018FF0D496868CF
:106CC800432202F0DDFF68680B49224603F006F80C
:106CD8002046FFF79BFA20B12046FFF7A3FFFF20CD
:106CE80005E094F82D3043F0080384F82D3040B2C5
:106CF80038BD00BF64690308B965020808B507F024
:106D08000FFF00F00FF800F05BF900F0A9F902F0AE
:106D180027FE00F08BFC05F0C5FDBDE8084002F039
:106D280049BD00000B4B0C4A0C4823F003031360C9
:106D38004FF4A05100225A801A715A18026001209B
:106D480010715180198006481180064A136007F0B7
:106D5800C9BE00BF9FD10020340600202C060020A9
:106D6800300600202806002070B5044600284CD0C4
:106D7800264B1B68984203D3254B1B68984205D3C2
:106D880007F0E8FEBDE8704007F0EEBE214807F0C6
:106D9800B5FE002304F8043C1F4B34F8080C1968AE
:106DA800A4F108028A4238BF1A60184B1B681918E8
:106DB8008A4211D00D797DB9154D2D68A9420BD0A5
:106DC800154D2E688E42195A08BF2A6024F8081CEF
:106DD800195A5918D01A488034F8060C19189142D3
:106DE8000ED00D7965B90C4D2E68964234F8082CF2
:106DF80008BF29601A5234F8082C9A18CB1A538005
:106E08000448BDE8704007F085BE70BD3406002018
:106E18002C06002030060020280600202DE9F0412D
:106E280003314FF6FC750D400B2D044603D9B5F51B
:106E3800A05F01D953E00C25DFF8B880D8F80030FE
:106E48009C4203D3284A1268944204D307F082FE76
:106E580007F08AFE44E0A4F1080634F8087CF61A24
:106E6800083FB6B2BF1BBFB2BD4238D838D01F48A2
:106E780007F044FED8F8003034F8081C5A18107986
:106E880078B95F5A06F108016D1819490868ADB25A
:106E9800904203EB050208BF0A60002111715F539D
:106EA80010E005F11402BA4215D8114806F108029B
:106EB800AD180768ADB25A19BA4238BF02605953C3
:106EC80000201071568024F8085C5A5BB2F5A05F68
:106ED8001CBF9B185D80054807F01CFE00E00024DD
:106EE8002046BDE8F08100BF2C06002030060020B7
:106EF8002806002034060020F8B5002856D00330B4
:106F08004FF6FC7404400B2C03D9B4F5A05F01D9EB
:106F18004BE00C24264807F0F1FD264B1968264B58
:106F28001A688B1A9BB2C4F5A05E39E0D5182F7980
:106F3800002F34D1D65AA6F10800C01AA0422ED389
:106F480004F1140E704510D308341C19A4B210199A
:106F5800165343802C80012307712B71135BB3F503
:106F6800A05F04D0D218548001E001232B718D4218
:106F78000FD1124B1A68104B19682B4601E01B8879
:106F8800CB18187910B90B4A136002E09342F6D176
:106F9800F9E7074807F0BEFD05F10800F8BD2B88A2
:106FA8007345C3DB024807F0B5FD0020F8BD00BFFC
:106FB8003006002028060020340600202C06002079
:106FC8000E4A0F49F0B500230E4E0F4F22F0030270
:106FD8001D4641F8045B33F806C0002008E051F86C
:106FE800044C1460DC5B41F8042C0130121980B2A7
:106FF8006045F4D10233202BEBD1F0BD3B060020D5
:1070080078BC0020FC6803081C6903080F2838B501
:1070180005460BD807F09EFD064B53F8254014B1E2
:10702800226843F8252007F09FFD00E00024204651
:1070380038BD00BF78BC002038B505460C4659B1AC
:1070480007F088FD054B53F82520226043F82540BA
:10705800BDE8384007F088BD38BD00BF78BC0020C7
:107068007047000070B504460D4641B9204604F04B
:1070780099FD0020214604F02BFEFDB91FE00A68A7
:1070880043689A42F2D0134B186807E002686368B5
:10709800C6689A4201D100F089FD30460028F5D132
:1070A8000D4B1B6807E01A6822B161688A4204BF69
:1070B8002A681A60DB68002BF5D1D7E72D682046CF
:1070C800656004F02DFD00202146BDE8704004F005
:1070D800B3BD00BFBCE50020C4E5002001B10968CC
:1070E800C160704738B504460D460020214604F0BB
:1070F800EFFD05B12D6800202146A560BDE83840A8
:1071080004F09ABD70B5054616461C46FFF7AAFF5F
:1071180028463146FFF7E6FF04B12468EC6070BDED
:10712800F8B5069EC661104E377880F83070013782
:107138003770089E0025044645608560C56080F864
:107148002D5005620661FFF7DDFF2046079B984733
:1071580030B9064B1A6822601C6004F0C5FB00E0D9
:107168002C462046F8BD00BFB8BC0020B0E5002082
:1071780010B504462146012014B904F0A9FD01E028
:1071880004F05AFD014B1C6010BD00BFB4E500209F
:1071980010B590F82D30DA07044612D443F00103F5
:1071A80080F82D30383004F043FB94F82D3003F08C
:1071B8003003302B05D12046211DBDE8104007F0D3
:1071C8007DB810BD10B590F82D30D907044611D5FB
:1071D80023F0010380F82D30383004F029FB94F8AF
:1071E8002D3003F02003DBB223B12046BDE8104068
:1071F80007F034B810BD10B521B330B3002905DA53
:107208004B4242899BB29A4201D21DE08BB2027B6B
:1072180044680AB1032A05D1641A00F110039C429C
:1072280012D308E0013A012A0ED800290CDA428963
:107238009A4209D3641A43894460CB18438103896D
:10724800C9180181002010BD012010BD70B5044689
:1072580000B3002507F07EFCE689013EB6B2E68160
:1072680007F082FCBEB9237B2668032B01D10F20CF
:1072780003E0013B012B04D80E202146FFF7DCFE7A
:1072880002E02046FFF770FD0135EDB23446002ECE
:10729800E0D100E00546284670BD38B5038999421B
:1072A80020D2CA1A0D46044605E0ED1A2389D318E0
:1072B80023812468ADB263899D42F6D8227B4AB9FE
:1072C8009D4207D063681B1BE918204689B2FFF767
:1072D800A5FD044620686581258108B1FFF7B6FF42
:1072E8000023236038BD2DE9F0470D4617460328D3
:1072F8007CD8DFE800F002080406362604E00E26F3
:1073080002E0002600E02226032F6FD8DFE807F00E
:10731800465E5E020F20FFF779FE044600B965E07D
:107328008219033626F003061332C6F5C066032316
:1073380022F003020436AE42A8BF2E460373426011
:1073480000230122468103600581C281AE1B0746E6
:10735800984640F2036940F2046A1CE00F20FFF7E8
:1073680055FE054618B92046FFF770FF3EE0032397
:1073780000F110020373B3B2038142604B4588BF2A
:1073880053460122C0F8008080F80D8038604381A0
:10739800C281F61A0746002EE0DC22E006F113004F
:1073A800EB1C23F0030320F00300C01880B2FFF7A2
:1073B800A3FD0446D0B186191336002326F0030630
:1073C800466005814581036003730AE00E20FFF7DC
:1073D8001DFE044650B100234360058145810360CA
:1073E80007730123E3810023637300E00024204630
:1073F800BDE8F0870346002002E001301B68C0B2F8
:10740800002BFAD1704710B5044640B107F0A2FB33
:10741800E3890133E381BDE8104007F0A5BB10BD47
:1074280010B568B161B103E004891B1903811046E6
:1074380002680B89002AF7D1028901609B18038131
:1074480010BD10B50C46FFF7EBFF2046BDE8104015
:10745800FFF7D9BF2DE9F0410C46054608B9F220DF
:107468003FE00029FBD002890B899A42F7D3002616
:107478003746B4F80A806B8961686868C6EB080803
:10748800DB1B4345B4BF1FFA83F81FFA88F8C019FD
:1074980089194246FAF776F846446389B6B2B34288
:1074A80047446B8998BF2468BFB298BF0026BB4287
:1074B80005D12D6815B9002CD1D10FE000272CB1CA
:1074C800628923899A4201D123684BB96A892B8939
:1074D8009A4201D12B681BB9002CCAD1204600E082
:1074E800FA2040B2BDE8F0812DE9F84388461646F7
:1074F80028B331B300240546A1461CE02BB16A89A4
:10750800934202D39B1A9BB214E06F896968FF1AF1
:10751800BFB2B74228BF374608EB0900C9183A4638
:107528003C19B944F61BFAF72DF8A4B21FFA89F9E9
:10753800B6B200232D682EB1002DDFD102E004463B
:1075480000E00C462046BDE8F88300002DE9F0472E
:107558004368DFF874A093F80990194B06461C6835
:107568000025984623E0237C4B4518D123681BB19E
:10757800DAF80020934212D1676987B1A069114BEC
:1075880021463246B84750B15DB1E368EB60D8F8A0
:107598000030C8F80040E3600026012303E0002320
:1075A80001E001232E46E26825462BB91446002C3B
:1075B800D9D12046BDE8F0870120BDE8F08700BF9B
:1075C800BCBC0020DCE50020E4E500206FF00900E9
:1075D80070470000134B70B51888134D4FF4804264
:1075E8004FF6FF74A04202D0013080B201E04FF4A0
:1075F80040400023595909680BE04E8B864207D159
:10760800013A92B2002AEDD1064B1880104670BD9F
:10761800C9680029F1D10433102BEBD1014B188034
:1076280070BD00BFBC0100203C6903087047000022
:10763800F8B5037E04460D4633BB1AB9FFF7CAFFF7
:10764800024618B3144F0021CB591B680AE0588B27
:10765800904206D11E68DEB1D5B12868C0B1864215
:1076680016D0DB68002BF2D104311029ECD115B10A
:107678002B6803B12360094B62831A681C60E260BF
:1076880002F0DEF8002004E0FA2002E0FE2000E02C
:10769800F82040B2F8BD00BF3C690308CCE50020E3
:1076A80038B5037E04460BB1002038BD0320FFF730
:1076B800ADFC05460028F7D023690361638B43833B
:1076C80001230376637E4376237A43F00203037231
:1076D800A37A8372637A437223680360638BABB1C6
:1076E800114A1368A34201D1E3680CE00F4A136002
:1076F80007E0D968A14203D11360E268DA6003E0C9
:107708000B46002BF5D113600023E36002202146CD
:10771800FFF792FC064B6B61064B1A681D60EA6026
:1077280002F08EF8284638BDCCE50020C8E50020D8
:10773800D5750208C4E5002030B5016B848DC58E6F
:10774800826A034640F66830854228BF0546601ABB
:107758008018451B002D01DBDC8530BD501A002840
:107768004FF0000001DDD88530BD8A1ADA8530BDBA
:10777800838DC91889B241F2D063994210B58CBF84
:10778800838581850446FFF7D7FF40F2B3539842BB
:1077980008DDA37F204643F00203A377BDE810402D
:1077A80001F090BD10BD10B5044648B1406808B15D
:1077B800FFF74CFD04202146BDE81040FFF73CBC14
:1077C80010BD10B503E00468FFF7EDFF2046002860
:1077D800F9D110BD01617047C16770478167704773
:1077E800C0F88810704741617047C0F8841080F86D
:1077F80020207047037E10B50446BBB10A2B15D074
:10780800012B13D0406F18B1FFF720FD00236367E9
:107818004FF6FF73A386E06EFFF7D3FF206FFFF7E5
:10782800D0FF0023E3662367A4F86A3010BD000088
:107838009C4B2DE9F74F1A68DFF8848201321A60F1
:10784800994B1A7801321A70C146984BDFF858A242
:107858001C680026FFE09AF8003094F821209A422C
:1078680001D1E768F6E0217E84F82130022994F8F6
:10787800462001D1062A51D00C2A4FD094F89130D5
:10788800C3B18B4994F89020C918013211F8011C32
:10789800D2B2914284F8902000D93DE00022062B14
:1078A80084F8902002D8013384F89130204601F002
:1078B80004FF31E0A38E180401D40133A386236F9B
:1078C80053B3B4F93400B4F94430984224DB0229A4
:1078D8000BD0B4F94010B4F9423003EBE103754919
:1078E8008A5C03FA02F3A4F844300023B4F84C107D
:1078F800A386B4F86030994228BF1946E38E490838
:107908005A009142A4F84E10A4F84C30B8BFA4F81D
:107918004E20204601F040FE002500E00125237E90
:10792800062B0CD1A27F02F01002D2B23AB15D4A06
:107938001168626A8A1A282A01D90135EDB2277AB4
:1079480007F00807FFB24FB3042B01D0072B24D14F
:10795800544BD4F88C001A68636AD21A00F52423B1
:1079680003F6B8434FF4FA71B3FBF1F39A4203D923
:107978000135EDB2012711E094F892304E4F07FB24
:107988000300B0FBF1F18A4207D9204601F076FEE8
:1079980094F89230013384F892300027237E032B29
:1079A80008D1404B1A68636AD31A282B0AD90135C3
:1079B800EDB207E0092B05D13A4B1A68636AD31A6E
:1079C800F02B00D845B32046FFF714FFE3680EB14B
:1079D800F36001E0354A13604FB1638B0093A38BCA
:1079E8000193206DA16A2246231D01F08FFDD4F872
:1079F8008850D4F810B0E76802202146FFF71CFB36
:107A0800002388F800301DB158466FF00901A847D7
:107A180099F80030F3B118E7E37F94F82020E7687D
:107A28000133DBB29A42E37713D8D4F88430E57790
:107A380088F800501BB120692146984700E0284685
:107A480099F80030002B7FF400AF10B9204601F000
:107A580039FC26463C46002C7FF4FDAE174B114EF0
:107A68001D681F460FE032686B6AD31AF02B10D8D6
:107A78000CE0E26000E03A6029460220D5F80C806C
:107A8800FFF7DAFA4546002DEDD109E02C46ED68FE
:107A9800F9E72846FFF7AEFEEA68002CE9D1EAE7E5
:107AA800BDE8FE8FC0E50020C1BC0020BCE5002079
:107AB800596903084C690308F8240100D0E500203F
:107AC800B8E5002003688B4210B50C4602D1CB689C
:107AD80003600DE0114A136007E0D968A14203D1A1
:107AE8001360E268DA6003E00B46002BF5D11360FF
:107AF8000023E3602046FFF77DFE237E0A2B0AD091
:107B0800012B08D0A37FDA0705D543F00203A3773A
:107B1800204601F0D7FB0023237610BDC8E50020DE
:107B2800037E0A2B2DE9F743044689460AD12146EC
:107B38001B48FFF7C7FF0220214603B0BDE8F0430A
:107B4800FFF77ABAD0F85080876AD0F8885006696B
:107B580014482146FFF7B6FF134B206F01221A7015
:107B680008B1FFF72EFEE06E08B1FFF72AFEB9F163
:107B7800000F09D0638B0093A38B404601933946CD
:107B88002246231D01F0C2FC02202146FFF754FAC9
:107B98001DB130466FF00901A84703B0BDE8F08376
:107BA800D0E50020BCE50020B8E500200121FFF762
:107BB800B7BF000037B50446002943D0037E042B25
:107BC80001D0072B3ED1636F23B9A28D41F2D06358
:107BD8009A4237D0638B206D0093A38BA16A0193DF
:107BE8002246231D01F092FC2046FFF703FE424A7D
:107BF8001368A34201D1E3680CE0404A136007E030
:107C0800D968A14203D11360E268DA6003E00B4649
:107C1800002BF5D113603A4B01221A70237E002500
:107C2800042BE56008D10A232376364B1A681C60BA
:107C3800E26001F005FE03E002202146FFF7FCF9AF
:107C4800284651E0237E072B53D8DFE803F0041EB3
:107C580027353C525244638BABB12B4A1368A3427D
:107C680001D1E3680CE0254A136007E0D968A14216
:107C780003D11360E268DA6003E00B46002BF5D10C
:107C880013600023E360022004E020482146FFF748
:107C980019FF03202146FFF7CFF92AE021461648AD
:107CA800FFF710FF164B0122022021461A70FFF73A
:107CB800C3F904F093F81CE0204601F0BEFA98B925
:107CC80004F08CF805E0204601F0B7FA60B904F03A
:107CD8008DF8052306E0204601F0AFFA20B904F03C
:107CE80085F80923237601E040B204E0204601F03C
:107CF800E9FA0020F8E73EBDBCE50020C8E5002011
:107D0800B8E50020D0E50020CCE50020C4E500203F
:107D1800037E012B03D0837F43F010038377012177
:107D2800FFF748BF10B50846144632B11189FFF76E
:107D38001FFD2046FFF78AFA04E01BB9BDE8104092
:107D4800FFF7E6BF002010BDF8B5456FC66F6F7B23
:107D580000230446436726B121462A460069B047F6
:107D680005E0304621462A463346FFF7DBFFB0B927
:107D780007F02007FFB2BFB1A38D41F2D062934252
:107D880001D00133A385E56F05B90CE00022206915
:107D980021461346A8470A3005D1F62004E040B230
:107DA8000A30FAD06567002040B2F8BD2DE9F843E3
:107DB800184B194F1A7801321A7098463C68174DBB
:107DC800002622E098F8002094F82130934220D031
:107DD80084F82120A27FD10709D542F00202A277B8
:107DE800204601F06FFAA37F23F00303A377636FA4
:107DF800D4F80C900BB94C4607E020462E70FFF7DC
:107E0800A3FF2B78002BD9D1F5E7002CDAD1BDE8F8
:107E1800F883FEE7C1BC0020BCE50020B8E50020DF
:107E280008B5FFF7C3FF064A13780133DBB2D8075A
:107E3800137003D5BDE80840FFF7FABC08BD00BFC2
:107E4800C0BC0020034B044A10681A6880181860E8
:107E5800704700BFB8010020C0E50020F8B505460E
:107E68000220FFF7D3F80446002836D1394B3A4AA6
:107E78001B68116807E05A6A8A1AA24234BF224670
:107E88001846DB681446002BF5D108B1FFF78EFEC3
:107E98000220FFF7BBF80446F8B92F4A2F4B1768A2
:107EA8001B687F2022460CE0597EA94208D88142EF
:107EB80006D85E6ABE1BA64202D3084634461A4656
:107EC800DB68002BF0D112B11046FFF76FFE0220DD
:107ED800FFF79CF80446002839D000219422204658
:107EE800F9F70AFC41F2D06246F2A863A4F86630BA
:107EF800A2850023E285FF226576A4F868301D4636
:107F08006372A272A4F840304FF406724FF6FF7302
:107F1800E286A38606220123A4F84C30A4F8442064
:107F2800A4F84220FFF78EFF0B4BA0651B68206565
:107F380063620B4BA0641B78E06584F82130094B21
:107F4800E577E367084B84F89250C4F88C302046F4
:107F5800F8BD00BFD0E50020C0E50020BCE500204A
:107F6800C1BC00202D7D020800DD6D004020FFF718
:107F780075BF10B50446084602F0F2F830B1838C9C
:107F880023B1283B9BB29C4228BF1C46204610BD0B
:107F9800F8B51E4D2C680646A089FEF71EF8C0F3FA
:107FA8000F30052831D92B689889FEF716F8000B91
:107FB800411F8900143489B2002340F2B35040F2C3
:107FC800B45520E0E25C012A05D01ED3022A04EB56
:107FD800030214D101E0013314E05778042F14D1BF
:107FE800DF1C8F4211DA9778D27842EA0722571EAF
:107FF800BFB2874288BF2A46F286043302E052782D
:108008001AB1D3189BB28B42DCD3F8BDC4BC002094
:108018002DE9F041A04B1B7803F01003DBB20446B6
:10802800002B00F06B819D4A436D1268B0F86050D8
:10803800816D981A00280EDB9342994B03D118687A
:10804800081A002807DB1B6899421FD1954B1B684B
:10805800DB89AB421AD9934BB4F862601B68D889A4
:1080680062658F4AA4F8600012688642A26538BF2C
:10807800A4F8620094F8912020B93AB984F89000E5
:10808800012301E012B1002384F89130844BA26CE3
:108098001B68981A002834DC0020A4F86400824881
:1080A8000088002840F0F481B4F86060A06D691879
:1080B8003018884240F0EC81B4F934100029C0F23D
:1080C800E7819A4240F0E48194F84720531CDBB2E0
:1080D800934288BF84F8473094F84730032B0AD975
:1080E800B4F84C20E38ED3189BB2934240F2B2808E
:1080F800A4F84C30AEE040F0AD80204601F092FA92
:10810800A8E0D143D9427ED4216D591A00297ADCDE
:10811800A17F01F00400C0B230B121F00401A177C1
:10812800B4F84E10A4F84C10B4F94050B4F842001A
:10813800A36400EBE5009A1AA4F84400237EB4F87F
:108148006600A4F8642000211218032B84F8461056
:10815800A4F8662084F8471031D9B4F84E20B4F852
:108168004C309A42E28E00D902E0524392FBF3F27D
:108178009A1892B29A4222D9A4F84C201FE0256F8F
:108188002B6868682367FFF735F9B4F8643053B192
:10819800EB689889FDF721FFC30704D5B4F864306C
:1081A800013BA4F864306868B4F86870FFF722F9F6
:1081B800381AA4F868002846FFF7F5FA00E0384EA8
:1081C800236F1BB9226F0023D2B915E0DB6858680A
:1081D800FDF70AFF236F1D89DB6807469889FDF7BD
:1081E800FCFE336810F0030018BF0120FB1A2818A2
:1081F8001B18002BC3DDE5E74FF6FF72A28600E0EF
:10820800A386E37726E00023A4F8643022E0E56E35
:108218002B68E3660BB9A4F86A306868FFF7EAF8D8
:10822800B4F8643053B1EB689889FDF7D6FEC707F8
:1082380004D5B4F86430013BA4F864306868B4F835
:108248006870FFF7D7F8381AA4F868002846FFF7CF
:10825800AAFA00E0124EE36E13B9A36B33BB4DE0EC
:10826800DB6835685868FDF7BFFEE36E1F89DB6879
:1082780080469889FDF7B1FE10F0030018BF012071
:10828800C8EB050538182D1A002DE6DB3268236D7A
:10829800D31A002BBBDDE0E7D4BC0020C8BC00200B
:1082A800D0BC0020C4BC0020CCBC00207B49E26BC1
:1082B8000968521A002A21DA794AB4F8401012687B
:1082C80041F3CC00D21A121A92B293B2511889B261
:1082D8001804A4F8401001D553429BB2B4F84220C8
:1082E80042F38D00121AD3189BB241F3CC01A4F8C3
:1082F80042305B18A4F844300023A363694B6A4AF0
:108308001888002800F0B380237E062B00F2AF8087
:108318001168A36ACA43DA4225D45A1C521A101AA1
:10832800002820DC591A614B586843898B420ADAC5
:1083380002890025521A03E0028145810068C91AA2
:1083480043898B42F8DB494209B2FEF754FF574A8A
:10835800554915890868A36A4019C01A1081D2685E
:108368000B60536006E0C91A002903DAA37F43F0C3
:108378000203A3774C4BA26A1B68991A002971DB88
:10838800591CA08D891A091A00296BDC9A4269D1F7
:10839800464DEB682E899889FDF71FFE10F0030003
:1083A80018BF01203F4B301880B21880A38D83423C
:1083B80030D2EB689889FDF710FEC0070CD5ED6840
:1083C800AE893046FDF709FE00F03E00FDF700FEDD
:1083D80026F47C563043A881A38D344D2B81EB685D
:1083E8009889FDF7FAFD00F0020080B210B12B89E0
:1083F800013B2B8168682989FEF74FFFEB682E89BE
:108408009889FDF7EAFD10F0030018BF0120254BFD
:1084180030181880234B244A1B8812689A18A262C5
:10842800A28DD31AA3852046FFF786F91F4B5A68F9
:10843800118919B11E490A6000225A60DB689889BF
:10844800FDF7CBFDC10704D51A4B1A7842F020027C
:108458001A70A37FDA0702D523F0010313E043F073
:10846800010312E02046BDE8F04100F009BF1268A0
:10847800A36AD11A002905DB0132A18DD31A5B1A30
:10848800002B09DDA37F43F00203A377BDE8F08149
:10849800002384F84730DDE6BDE8F081D0BC002039
:1084A800C0E50020CCBC0020C8BC0020E0BC0020F7
:1084B800D8BC0020D5BC00202DE9F74F06460F4652
:1084C80003F09CFC7368A74AA74C13601A7802F063
:1084D8000F02910003EB8203304649422360FEF706
:1084E8008AFE002840F0CE833389132B40F2CA83DA
:1084F8009E4D3946286801F043FD002840F0C283AC
:108508002B6803F0F003E02B00F0BC832368988904
:10851800FDF763FD6FF00301C0F30733594330469D
:10852800FEF769FE8346002840F0AC832768388848
:10853800FDF753FD388027687888FDF74EFD788071
:1085480027687868FDF750FD894B786027681860C0
:10855800B868FDF749FD874BB86027681860F88947
:10856800FDF73BFDF88123689889FDF736FD824BBE
:10857800B6F80880276810F0030C00F03F0118BF18
:108588004FF0010C1970C4447C4B29681FFA8CFC0D
:10859800A3F800C07A4BD3F800A07A4B0246D3F870
:1085A80000905446584619E0A58B3B889D4213D14C
:1085B800658B7B889D420FD163684B450CD123683E
:1085C8008B4209D1002800F08283E368C3606C4BBA
:1085D800C4F80CA01C607AE32046E468002CE3D1C0
:1085E80072E3988B3C88844230D1588B7D888542D1
:1085F8002CD15868484529D11868884226D102F0FC
:108608000401C9B2002940F03F8302F00201C9B257
:1086180059B1574A11689A6A8A1A0BD4988D121A56
:10862800002A07DC0095019441E0D20702D5564A9A
:1086380012685A62BCF1000F00F026839A7F42F05C
:1086480002029A77184600F03DFE1DE3DB68002B16
:10865800C7D14E48046825460FE0688BB7F80280FA
:10866800804508D1D5F80080884500F04283B8F1EC
:10867800000F00F03E832B46ED68002DEDD13CE362
:10868800E968D960414BEC601D6002F00403DBB27D
:10869800002B40F0F98202F010085FFA88F8B8F170
:1086A800000F0CD0324B196800903B880193314B76
:1086B800186861442D4A334B00F028FFE4E202F0C9
:1086C8000202D2B2002A00F0DF82687EFFF7C6FB02
:1086D8000446002800F0D882244B1B6803606B8B8B
:1086E8004383284B1B6843601F4B1B6859781A78D3
:1086F80042EA01228283032202761D4A1268511C33
:1087080081620163DB89A0F86030A0F86230A0F8CC
:108718004E302B6903616B69013A426543612B7ADC
:1087280023F073030372164B1A681860C26001F0D5
:1087380087F8174B012220461A70FFF729FC211DE4
:10874800E08EFFF716FCE08603F040FB204612217E
:1087580000F028FD20B120464146FFF7E1F993E2F9
:10876800204670E7DCBC0020C4BC0020E4E5002003
:10877800C8BC0020D0BC0020D4BC0020CCBC002049
:10878800BCE50020DCE50020C0E50020C4E50020B1
:10879800B8E50020737B43F001037373636F63B123
:1087A8002046FFF7D1FA0A3004D0636F2BB19F4BF4
:1087B8001B8813B103F03AFB49E29D4B1C609D4BAB
:1087C8001B7803F00402D2B2AAB1237E022B06D191
:1087D800994B1A68236D9A4240F0A18296E2974B12
:1087E8001A68A36AD31A00F19A82A18D5B1A002B2A
:1087F80000F395828AE203F00203DBB223B1237E01
:10880800023B012B00D96BE0A37F03F01003DBB21E
:1088180013B98B4B1B686362002384F8923020469F
:10882800FFF7B6FB237E023B072B00F27882DFE8D6
:1088380013F008007700C900DA003001C9005201BE
:1088480086017C4B1B7803F01203122B53D1236F44
:10885800794DDB682E685868FDF7C6FB0130864203
:1088680049D1B4F86630E08E0133A4F86630734B12
:108878001B685A1CA26222632A68A264714A1268A1
:10888800013BD289636504232376E118A4F86020AC
:10889800A4F86220FFF76DFB0A234343A4F84E3087
:1088A800B4F84C30E086012B01D1400080B2B4F816
:1088B8006830A4F84C00206F013BA4F868300368C6
:1088C8002367FEF770FF236F1BB94FF6FF73A3866C
:1088D80003E00023A38684F84630D4F880301BB91F
:1088E800A37F43F0020319E200222069214698473A
:1088F8000A30F5D1ABE14F4B1B7803F01003DBB224
:10890800002B00F00C824F4B484A1B68118858888E
:108918004A4A126800901B880193474B18683AE04E
:10892800444B1B7803F01002D2B2002A39D0424BD4
:108938001868A36CDB43C34223D4236DC31A002BEE
:108948001FDC04232376636903B947E120692146C4
:108958000022984718B10A3040F0408177E120465C
:10896800B4F84C50FFF754FBB4F8643013B1013B32
:10897800A4F86430E38E012D08BF5B00A4F84C30E6
:1089880023E0304B294A1B6811885D882B4A1268FE
:1089980000951B88019389182B4B2C4A00F0B6FDD3
:1089A800BDE103F00203DBB2002B00F0B881234ADB
:1089B800A36A1268013B9A4240F0B181204600F058
:1089C80003FEACE12046FFF723FB214B1B7803F0A5
:1089D8002003DBB2002B00F0A281A37F43F0020347
:1089E800A377072353E02046FFF712FB184B1A78AA
:1089F800104B1B7802F0200203F01003D2B2DBB256
:108A0800002A3AD0002B32D00B4B1A68236D9A42B9
:108A18002DD1A37F43F00203A3772046FEF7EAFE99
:108A28000C4A1368A34217D16DE000BFCCBC0020EC
:108A3800D4E50020D4BC0020D0BC0020C8BC002055
:108A4800C0E50020C4BC0020DCE50020E4E50020EF
:108A5800D5BC0020BCE500208E4A136004E0D9682C
:108A6800A14200D157E00B46002BF8D15AE0A37F72
:108A780043F00203A377082309E0002B00F04F819D
:108A8800854B1A68236D9A4240F049810623237664
:108A980045E12046FFF7BCFA804B1B7803F0200322
:108AA800DBB2002B00F03B81A37F43F00203A377E6
:108AB8002046FEF79FFE7A4A1368A34200D122E0BF
:108AC800744A136004E0D968A14200D123E00B4640
:108AD800002BF8D126E02046FFF79AFA714B1B7855
:108AE80003F01003DBB2002B00F019816A4B1A68FF
:108AF800236D9A4240F013812046FEF77BFE684AB8
:108B08001368A34201D1E3680CE0624A136007E0EE
:108B1800D968A14203D11360E268DA6003E00B462A
:108B2800002BF5D11360604B01221A700A232376BB
:108B38005E4B1A681C60E26000F082FEEFE020469F
:108B4800FFF766FA574B1B7803F01003DBB2002BD4
:108B580000F0E580504B1A68236D9A4240F0DF80A0
:108B68004E4B1A7842F010021A70D8E0D4F88830C8
:108B78009BB120696FF00A010EE003F01003DBB22D
:108B8800A3B1A37F03F01003DBB233B9D4F8883064
:108B98001BB120696FF00B01984721464048FEF74A
:108BA80091FF02202146FEF747FA50E0B4F864200E
:108BB8001AB93F4B1A684AB926E0A36F002BF8D0C0
:108BC8002069214698470A30F3D140E0A37F03F09B
:108BD8001003DBB233B11046FEF738FB2046FEF730
:108BE800E5FF34E0E56F1DB120692146A84704E0A0
:108BF800284621462B46FFF795F843B20A3326D07C
:108C080010B12B4B1B686367244B1B7803F02003C0
:108C1800DBB2B3B1636F23B15A7B42F020025A73BF
:108C28000FE0A38D41F2D062934201D00133A385B6
:108C3800E56F35B10022206921461346A8470A305E
:108C480005D01C4B002220461A6000F03BFB194B54
:108C5800194D00241C606868154B1C60002867D0FB
:108C6800FEF7F4FA6C6063E0144B154A1B68118830
:108C78005888144A126800901B880193064B89187B
:108C8800186817E503F0D2F8304603B0BDE8F04F96
:108C9800FEF7DCBAC8E50020D0BC0020D5BC002017
:108CA800BCE50020D4BC0020B8E50020D0E50020B9
:108CB800D8BC0020D4E50020E0BC0020C4BC0020C3
:108CC800CCBC0020C8BC00201B4B1B68BFE41B4B5E
:108CD80000211960A3F808805E60DF60184B02F07D
:108CE80008021960174BD2B21970002A7FF452ADEE
:108CF80054E5002B7FF4C4ACC7E4B889FDF76DF9DF
:108D080000F0040080B20028BED1ADE70D4B1A7800
:108D180042F008021A70A37F23F00103A377094BDE
:108D28001B7803F00802D2B2002A7FF41FAF24E7B1
:108D380003B0BDE8F08F00BFD0E50020E0BC002004
:108D4800D8BC0020D5BC002070B591420C461E4608
:108D5800049D1AD29DF8143003F00203DBB25BB90C
:108D6800AB7F03F04003DBB27BB99DF818301BB131
:108D7800E96E09B92B6F43B104F2B75121F0030131
:108D88009142A8BF114689B200E021460022FEF7B1
:108D9800AAFA20B143891B1B33800481448170BD2A
:108DA8002DE9F0479DF8206006F0020716F0010F44
:108DB800FFB280469A460CBF00230423002F14BF3D
:108DC8000C27002704200D469146FF18FEF71EF9D0
:108DD800044618B92846FEF739FA30E086722B891E
:108DE8004560DB1B00260660038114212846FEF738
:108DF80002FA054620B12046FEF7D5FC34461EE0AF
:108E08006368B8F81A005E68E660FDF7E1F830803C
:108E1800B8F81C00E668FDF7DBF870805046E66895
:108E2800FDF7E0F8BF02706007F5A04040EA0900CE
:108E3800E668FDF7CDF8B081E3689D74DD742046DF
:108E4800BDE8F0871431F8B589B205461746012008
:108E58000022FEF748FA0646F8B14468688BFDF729
:108E6800B7F82080A88BFDF7B3F867606080A86A20
:108E7800FDF7B8F8A06045F21000FDF7A9F8A08149
:108E8800E88DFDF7A5F80023E08123746374A374CB
:108E9800E374EA8DAB6AD3182B633046F8BD2DE92D
:108EA800F04F8FB0914607930023ADF83630044653
:108EB800B0F86220C38E0691002900F06881017E17
:108EC800072900F2668190F918104FF06450884025
:108ED80040F15F81B9F1000F0DD0B4F86610494533
:108EE80000D203E0B4F86810472904D9A37F63F0DF
:108EF8007F03A37751E15208E66EB4F868B09A424E
:108F080028BF1A460A920EB966E01E463368002B3F
:108F1800FBD1B37A37890A98B4F86A5013F0010F75
:108F280003F002030CBF00210421DBB2C21B002B9B
:108F380014BF0C230023521AD21A92B21DB9ADF8ED
:108F480036502B460AE0A94534BF4B462B46ED1A4E
:108F5800D21AADF8365092B21D4633464D453FD22F
:108F6800002A3DD0002F3ED00799C5EB090A92454B
:108F7800A8BF9246CB071FFA8AF814D5012301919E
:108F880002930094032041460DF13603FFF7DCFEFF
:108F98000746002800F0E980069A406851194246C1
:108FA800F8F7F0FA0BE0032041460122FEF79BF99F
:108FB8000746002800F0D980069843197B60384698
:108FC800FEF718FAA8441FFA88F85844AA461FFA68
:108FD80080FB4546334607E0B2463546334600E057
:108FE800AA46002700E0AA4607994FF0000801F0BA
:108FF8000101CDF82C80089168E0C5EB09030A9AB5
:109008009BB2934238BF1A46089B0992DBB1D8F14C
:1090180001030798009438BF00230190029311467A
:1090280000200A9A0DF13603FFF78EFE84460028C9
:1090380000F09E80069A4068CDF814C05119099A2C
:10904800F8F7A0FA19E0089809990122FEF74BF9F8
:109058000346002800F08C800698421908985A6048
:10906800014602460593FEF73EF9059B08B91846E6
:1090780013E019460590FEF7D3F9DDF814C06046F1
:10908800CDF814C0FEF7B6F958441FFA80FBBBF1BF
:10909800480FDDF814C003D96046FEF7D7F867E03B
:1090A800E36D0022EB18009220466146FFF778FE38
:1090B800034600285CD0B8F1000F02D00B99086075
:1090C80000E08046099A0B935519ADB24D4594D3EB
:1090D800BAF1000F19D0756811E02A8952442A8123
:1090E8002A685AB96A686889069905931018524619
:1090F800F8F748FA6A89059B52446A812D68002D61
:10910800EBD132899244A6F808A0BDF83620A4F81D
:109118006A2057B1706805933946FEF781F9398995
:109128003289059B8A18328103E016B9C4F86C802D
:1091380001E0C6F80080E26DA4F868B04A44E26530
:10914800B4F86620C9EB0209A4F8669033B3DC686A
:109158000CB3079B03F00205EDB2E5B90820A68918
:10916800FCF736FF3043A08115E04FF00008474672
:10917800A37F63F07F03A37717B13846FEF766F83D
:10918800B8F1000F09D04046FEF71BFB05E0F223BB
:1091980004E0F32302E0002300E0FF2358B20FB0FD
:1091A800BDE8F08FB0F86830472B73B504460D461C
:1091B80000D914E0B0F86630C1F34006B100002BC6
:1091C80038D000200246FEF78EF8014600B906E0C6
:1091D800009620462A46E36DFFF7E2FD20B9A37FFB
:1091E80063F07F03A37725E0E36E13B9E06604E03C
:1091F80013461A68002AFBD118600023A907A4F8AF
:109208006A3007D0E36D0133E365B4F86630013B9B
:10921800A4F86630EA0703D5A37F43F02003A377B9
:109228004068B4F86850FEF7E5F84019A4F86800FB
:10923800002000E0FF2040B27CBDF8B5C46E0546B2
:109248000CB90AE01C462368002BFBD1E368988917
:10925800FCF7C3FE10F0070605D028460121BDE83B
:10926800F840FFF79FBFE4680120A789FCF7B0FE2C
:109278003843A081AB7F43F02003AB773046F8BD7D
:1092880037B50446006DFCF7ADFE002102462046C6
:10929800FFF7D8FD054688B1A37F627A23F0030360
:1092A80000920622A3770192A37A2146221D01F09B
:1092B800ABF82846FDF7CAFF002000E0FE2040B2C8
:1092C8003EBD00008F4B1B6883422DE9F74F0446D3
:1092D80000F01381B0F84C30B0F86090C56E994535
:1092E80028BF9946837F03F00203DBB283B12DB90F
:1092F800204603B0BDE8F04FFFF7C2BFEB685868DF
:10930800FCF772FE2A89A36CD31A18184845EFD8BF
:10931800266F0EB9D1E01E463368002BFBD1CCE096
:10932800EB689889FCF759FE236F9BB1A27F12F076
:10933800440F0FD1E36E2BB1196859B91989E38E1F
:10934800994207D2B4F8663023B1B4F86830472B95
:1093580040F2CE802B68E366237E022B0CD0EF68A8
:109368001020B7F80CB0FCF733FE40EA0B00B881C8
:10937800A37F23F00303A37702F048FDA06AEF68F8
:10938800FCF730FEB860E08DEF68FCF721FEF8814D
:10939800E28DA36AEF68D3182363AB7AD80709D59F
:1093A800414640F2B450FEF7E4FD40F00170FCF78E
:1093B80019FE7861B4F93430013301D10023A38652
:1093C80023682BB9404600F0CBFE10B343682360F6
:1093D800A36B3BB9DAF80030A363EB685868FCF775
:1093E80003FEE0636868EB684268418943609A1A43
:1093F800891A418101898A1A028100221A745A74D1
:10940800627AA37A0092062201922146424600F02F
:10941800FBFFEB685868FCF7E7FDEA68B5F808B0A9
:1094280007469089FCF7D9FD10F0030018BF01200A
:10943800226D0BEB0003DB19D21A002AB8BF236593
:10944800EB682F899889FCF7C8FD10F0030018BF56
:109458000120381860B300232B60236F0BB92567F0
:1094680024E0EB685868FCF7BFFDF36807465868C6
:10947800FCF7BAFD381A002817DA04F1700700E083
:109488003F683B681BB93B682B603D6013E0DB68B5
:109498005868FCF7A9FDEB6883465868FCF7A4FDFB
:1094A800C0EB0B000028EBDBEDE735602E4602E051
:1094B8002846FEF778F9E56E03E0DFF84CA004F1E2
:1094C800040815B9E36E73B90BE0EB685868FCF74C
:1094D8008BFD2A89A36CD31A181848457FF620AF4C
:1094E800F0E7A4F86A30A37F03F07F03A37704E0D2
:1094F80012F0A00F7FF42EAFE4E7002003B0BDE820
:10950800F08F00BFD4E50020C0E500202DE9F74F1B
:1095180081460D4690460120142100221F46BDF8C1
:1095280030B0BDF834A0FDF7DEFE0646002830D086
:1095380044685846FCF74CFD20805046FCF748FD2F
:1095480060804846FCF74EFD60602846FCF74AFDFF
:10955800A06045F21400FCF73BFD16230025A37319
:109568006FF02F03A081E37325746574A574E57407
:1095780002F064FC062301930095304641463A46C2
:10958800FF2300F041FF304603B0BDE8F04FFDF780
:109598005DBE03B0BDE8F08F026F10B59AB11146F9
:1095A80000E019460B68002BFBD1C46E0C60C26644
:1095B80090F846200367013280F846208363BDE8AF
:1095C8001040FFF77FBE10BDF8B5056F0446002DAB
:1095D80027D02B6800F16C06036700E03668336813
:1095E8002BB933682B6035602B687BB90CE0DB68DE
:1095F8005868FCF7F9FCEB6807465868FCF7F4FC78
:10960800381A0028EADBECE7A4F86A3094F8463008
:10961800013384F846300023A363BDE8F84002F024
:10962800FDBBF8BD036F10B5044633B3837F03F069
:109638000403DBB20BBBFFF7C7FFB4F84C30B4F838
:109648006020934203D95208A4F84E2002E05B0838
:10965800A4F84E30E38EB4F84E105A009142B8BFC9
:10966800A4F84E20B4F84E20032101FB0323A4F8EC
:109678004C30A37F43F00403A37710BD37B50446ED
:10968800006D0138FCF7AEFC002102462046FFF7CA
:10969800D9FB054678B100224FF0060E8DE804404C
:1096A800A37A2146221D00F0AFFE284603B0BDE88C
:1096B8003040FDF7CBBD03B030BD2DE9F341046F59
:1096C800054614B9C46E002C42D0E3689889FCF7AB
:1096D80084FC10F0010005D02189D1F1010138BFC7
:1096E800002100E00146E3685FFA81F8284681F02E
:1096F80001015A68FFF7A6FB0646002828D04768EC
:10970800B8F1000F09D0BC891120FCF761FC24F4E2
:109718007C54A4B22043B88109E060682389028997
:10972800D31A07F1140101229BB2FDF7DDFE0022D6
:109738004FF0060C8DE80410AB7A304629462A1DF6
:1097480000F062FE304602B0BDE8F041FDF77EBD94
:1097580002B0BDE8F081000070B5044609200D464E
:109768001646FDF753FC034608B31149002280E86A
:1097780074000A6802B905E05068A0420CD9041BBD
:1097880054601A600B6070BD4C6884420CD80A465D
:1097980002E01960136070BD51685868401A11687A
:1097A80058600029F0D1F4E7201A4860F1E770BD4D
:1097B800F4BC002008B5002241F288300849FFF7C0
:1097C800CBFF00224EF660200649FFF7C5FF064989
:1097D8004FF4FA700022BDE80840FFF7BDBF00BF94
:1097E8002D98020811980208F597020808B5FDF7A8
:1097F800C9F904494FF4FA700022BDE80840FFF7A0
:10980800ABBF00BFF597020808B5FDF739F9044961
:109818004EF660200022BDE80840FFF79DBF00BF5C
:109828001198020808B504F0FBFC044941F288309D
:109838000022BDE80840FFF78FBF00BF2D9802083F
:10984800084B1B686BB9084B1B6813B9074B1B689F
:109858003BB1044B064901221A60FA200022FFF7A7
:109868007BBF7047F0BC0020BCE50020D0E500209D
:109878007D98020808B5FEF7D3FA084B1B6813B9A0
:10988800074B1B6833B10749FA200022BDE808409E
:10989800FFF762BF044A136008BD00BFBCE50020A3
:1098A800D0E500207D980208F0BC0020104B1B6812
:1098B80010B5E3B1002200E023469C68844212D12F
:1098C800DC688C420FD1196802B9094A11601A681C
:1098D8001AB1506859684118516009201946BDE805
:1098E8001040FDF7A9BB1C681A46002CE4D110BD36
:1098F800F4BC00202DE9F843184E04460D463746BF
:1099080032682AB920462946BDE8F84305F0B4B8BC
:1099180052686AB939680A68D1F808803A6009203B
:10992800D1F80C90FDF788FBB8F1000FE8D006E0FD
:109938002046294605F0A0F8431CEBD002E0484633
:10994800C047DDE7054B1B685968884234BFC0EB48
:10995800010200225A60BDE8F88300BFF4BC002071
:10996800704700002DE9F04FD0F8049003890E46A7
:1099780099F8001001F00F018A1CB3EB820F85B033
:10998800054605DB89004942FDF735FC834610B1E1
:1099980002F06CFA96E0DFF850A16C68DAF8000083
:1099A800314600F0EDFA80462088FCF716FB0746A2
:1099B8006088FCF712FB44280FD1432F4FD1336A3C
:1099C800002B4CD05C68002C49D06368002B4ED02B
:1099D800434A1268934242D149E0424BDAF800A068
:1099E800D3F800C03E4B1B686446039359465B4658
:1099F80032E0628A82422DD12268B8F1000F00D18C
:109A08005AB1524509D0B8F1000F23D02AB18AEAD9
:109A1800020BB2681BEA020F1CD1002B58D1237C21
:109A280003F00403DBB2002B0CBF234600234FE0F6
:109A3800D4F804B0BBF1000F01D121B917E0039AA3
:109A4800934507D1F9E7E368CB60264BC4F80CC00F
:109A58001C600CE02146E468002CCAD133B9224BC3
:109A680072681B689A422DD1002400E01C462846E3
:109A78006FF00701FDF7BFFB002889D154B102F050
:109A8800E5F9A669F6B10097E069154B21462A4623
:109A9800B04721E0B8F1000F12D1134B1B6803F057
:109AA800F003E02B0CD099F8001001F00F010231FF
:109AB80089002846FDF79FFB2846032100F0D2F9CC
:109AC80002F0CCF9284605B0BDE8F04FFDF7BEBB63
:109AD800A28ABA42BED1ABE705B0BDE8F08F00BF9D
:109AE800DCE50020D8E50020E4E50020F8B5254BAA
:109AF800044618680025034612E09C420ED05E8A90
:109B080096420CD11F680FB9F82039E00029FBD024
:109B18000E68002EF8D0B74201D1F5E70125DB68C1
:109B2800002BEAD101B109682160FAB9164B1A88ED
:109B38004FF480414FF6FF76B24202D0013292B222
:109B480001E04FF4404203460AE05F8A974206D19B
:109B5800013989B20029EFD10B4B1A80D4E7DB68B1
:109B6800002BF2D1084B1A80002ACDD06282204601
:109B780002F08CF91DB9034B1A681C60E2600020E2
:109B880040B2F8BDD8E50020BE0100202DE9FF470E
:109B98009246428ADDF8308005460E46994632B133
:109BA80030460821FDF727FB40B9344613E001464B
:109BB800FFF79CFF07460028F2D044E00120082167
:109BC8000022FDF790FB0446002839D0338913B1F1
:109BD8003146FDF736FC688A6768FCF7F9F9388082
:109BE8004846FCF7F5F900237880BB71FB712B68B8
:109BF80013B908F104090AE0D8F80420934205D003
:109C0800B4421FD02046FDF721FB1BE0A94620895E
:109C1800FCF7DEF9B8806A7AAB7A009211220192D9
:109C280049465246CDF80880204600F09DFB07467D
:109C380002F024F9B44206D02046FDF707FB02E003
:109C4800FF2700E0FA2778B204B0BDE8F087F7B53F
:109C5800054610460F4614461E4600F081FA38B1F4
:109C680000903946284622463346FFF78FFF00E02A
:109C7800FC2040B2FEBD838A021DFFF7E8BF00004A
:109C880070B51646428A04460D460AB135B906E053
:109C98000146FFF72BFF0028F8D013E02D68237C3E
:109CA800094A656043F0040323741368A6821846C2
:109CB80002E0844205D0C0680028FAD1E36014604D
:109CC80000E0002040B270BDD8E5002000234360CA
:109CD8008382037C23F00403037470478161C261AB
:109CE8007047000010B5044602F014F90A4A1368D8
:109CF800A34209D1E368136008E0DA681AB1A24206
:109D080004BFE268DA60DB68002BF6D10120214647
:109D1800BDE81040FDF790B9D8E5002010B5012046
:109D2800FDF774F9044628B100212022F7F7E4FC76
:109D3800FF23A372204610BD2DE9F043044685B0E9
:109D48000F4602F01BF8656895F8008008F00F08C8
:109D58004FEA8808C8F1000920460FFA89F1FDF793
:109D68004AFA002872D12389032B6FD963681B78BC
:109D7800082B65D1394B1E683946304600F000F98A
:109D880000285DD106F0F006E02E00D158E02389C6
:109D9800072B5BD9204600F0CFF800B156E02046EB
:109DA80022211FFA88F8FDF726FAF8B12046414625
:109DB800FDF721FA0246002848D102202189FDF743
:109DC80092FA0646002841D02146FDF743FB0028B9
:109DD8003CD130460FFA89F17568FDF70CFA002876
:109DE80034D12046FDF732FA344606E020466FF0BB
:109DF8002101FDF700FA002828D1DFF86090636898
:109E0800D9F80020EA60164A1268FF262A61002263
:109E18001A709A70DA70AA72EA722E7201F0BEFF96
:109E280001F0CCFF20464146FDF7E5F9024638B976
:109E380001238DE8890020464946334600F094FA0C
:109E4800204605B0BDE8F043FDF700BA2046FDF70F
:109E5800FDF905B0BDE8F04301F098BFE4E5002046
:109E6800DCE500202DE9FF4107460D4601202421AD
:109E78000022FDF738FA064658B34468D7F804803C
:109E8800657003230025237025716571A571E5713F
:109E9800406879681C220830F7F774FBA570E570F4
:109EA8007189204600F042F8608001F077FF01F0E8
:109EB8007DFFD8F80C3004AA304642F8043D01234F
:109EC800019300952946FF2300F09EFA3046FDF7DE
:109ED800BDF9BDE8FF8113B5002310F00102ADF80C
:109EE800063006D0994204DD10F8013B01398DF89F
:109EF8000730002303E030F8024B02391B1901290F
:109F0800F9DC04BF01788DF80610BDF806001B18AF
:109F180098B200EB134398B200EB134022B103064A
:109F2800C0F3072040EA134080B21CBD08B5FFF714
:109F3800D2FFC04380B208BD70B50026054634463E
:109F480013E069896868FFF7C6FF6B89001984B256
:109F5800D90704EB104407D52306C6F10106C4F35C
:109F68000724F6B244EA13442D68002DE9D126B13E
:109F78002306C4F3072444EA1344E04380B270BDC7
:109F8800431E033311D891F82D3003F00203DBB2DE
:109F98006BB14A6890420AD08B6842401A4200D09E
:109FA80005E0DB431840984201D1012070470020AA
:109FB8007047F0B5037885B00E46002400AAA718AC
:109FC800A3F13002092A6DD8302B0BD14378782BB6
:109FD80004D0582B02D00130082504E083781025DE
:109FE800023000E00A250246002000E00132A3F119
:109FF8003001092903D805FB0030303813E0102D53
:10A0080013D1A3F16101C9B2052904D9A3F1410C07
:10A01800BCF1050F09D80A3319298CBF41216121E8
:10A028005B1A43EA00105378E0E72E2B07D10C2C7B
:10A0380038D04DF804005378501C0434BEE70D2B7B
:10A0480003D8092B03D213B12CE0202B2AD16B465D
:10A05800FB1A9B100133042B1FD8DFE803F0231EE3
:10A06800030A1300B0F1807F1CD2009B40EA036012
:10A0780013E0B0F5803F15D2009B1A06019B42EA17
:10A08800034309E0FF280DD8009B1A06019B42EA0A
:10A098000342029B42EA032318432EB1FBF7A2FFB7
:10A0A800306001E0002000E0012005B0F0BD07B5F8
:10A0B80001A9FFF77EFF08B1019801E04FF0FF30DA
:10A0C8000EBD2DE9F74F036802A80DF1070840F807
:10A0D800043D0C46013800274FF00A0C4FF02E09BA
:10A0E80043780025B3FBFCF60DF1080B0CFB163A80
:10A0F8000BEB05030AF1300A013503F808AC16F03A
:10A10800FF03EDB2EED1013DE61B00F8013FEDB2D1
:10A118003B4637460BE06C1E9342E4B216DA0DF16B
:10A12800080A554415F8085CFD5401332546FF2DEF
:10A1380006EB0304EFD15F1C934207DA404504F8AD
:10A14800019BCDD1002304F8013C00E00021084622
:10A15800BDE8FE8F01491022FFF7B3BFF8BC00200D
:10A168000F4B10B51C680AE094F82D30D90705D5B7
:10A17800036862685A40A3681A420ED02468002C0B
:10A18800F2D1084B1B682BB193F82D20D20748BF9A
:10A198001C4602D401F0BCFCFFE7204610BD00BFFE
:10A1A800B0E50020B4E500202DE9F84F04460F463D
:10A1B80001F06EFC666896F800804FEA1813042BCD
:10A1C80005D02046FDF742F801F06AFCBEE0708831
:10A1D800FBF703FF08F00F0863894FEA8808434537
:10A1E8000146204602D323898B4202D2FDF72EF87E
:10A1F80045E0FDF752F83269564BDFF868B11A604E
:10A20800F168554A3D4611604FF001099A4695F8A4
:10A218002D30D80703D4B9F1000F0ED110E06B68C8
:10A22800002BF8D0DAF80000984200F08880294620
:10A23800FFF7A6FE0028EED081E0DBF8005000E032
:10A248002D68BD4208BF2D684FF00009002DDED1F2
:10A2580072E006EB08035B88B3F5884F6FD111E015
:10A268003946FFF78DFE28B9D8F8003003F0F0031F
:10A27800E02B08D12046FCF7E9FF01F019FC01F0BA
:10A2880027FC63E03D463DB901F012FC01F020FCDB
:10A298002046FCF7DBFF59E0F38823F0C0039BB2AC
:10A2A8002BB12046FCF7D2FF01F00AFC4EE02B4B05
:10A2B8001F602B4B204639461E60FDF747F988BBC7
:10A2C800737A062B0BD0112B02D0012B15D10DE080
:10A2D80001F006FC20463946FFF744FB22E001F076
:10A2E800FFFB20463946FEF7E7F81BE001F0F8FBD4
:10A2F80020463946FFF720FD14E0164D39462868F8
:10A30800FFF73EFE48B92B6803F0F003E02B04D0BA
:10A31800666020460221FFF7A5FD2046FCF796FF60
:10A3280001F0CEFB0D4A002313600D4A13600A4A60
:10A338001360084A136009E0737A112B89D0DFF89B
:10A348001880D8F8000000289DD089E70020BDE8D3
:10A35800F88F00BFE4E50020DCE50020E0E5002000
:10A36800E8E50020B0E500202DE9F347154606464C
:10A3780089469A460C9F01F0BBFBB5B330461421C1
:10A38800FCF739FF804618B101F0BAFBFE2036E031
:10A3980074689DF82C3084F808A063722B682361D8
:10A3A800452323709DF8283063703089FBF710FE31
:10A3B80084F8068084F80780DFF848806080B8F861
:10A3C8000000FBF705FEA080B8F800300133A8F8BC
:10A3D8000030B9F1000F02D0D9F8003003B97B681A
:10A3E800E3600023A372E37204E0736802AD1B69A3
:10A3F80045F8043D7B69384631462A46984740B2BD
:10A40800BDE8FC8708BD0020F0B5054685B01046BC
:10A418000F4614461E46FFF7A3FE68B19DF8283084
:10A42800029000939DF82C30284601933946224625
:10A438003346FFF799FF00E0FC2040B205B0F0BDBD
:10A4480010B500230CE044891C19A4B2A14205D21E
:10A458004068CB1AC35C0020137004E000682346F0
:10A468000028F0D1F22040B210BDF0B5002579E007
:10A4780044892C19A4B2A14272D2D0F804C04F1B4F
:10A488000CEB07051CF8076016F0800F05D10121B9
:10A4980011701CF807201A805AE0802E2AD1002655
:10A4A8001E8022E0B3F800C0013189B20CF1010C22
:10A4B800A142A3F800C008D3006800B94EE0B0F884
:10A4C8000AC045686444A4B200E0013595F800C0AC
:10A4D800BCF1000F04D10136F6B2022E01D107E01B
:10A4E8000026B942DED1022E02D08F1CBFB2D9E7B6
:10A4F80001232CE0812E0CD1013189B2A14203D372
:10A50800016859B34D6800E00135297819800223A4
:10A518001DE0822E1ED14E1CB6B2A64201D20135D4
:10A5280005E00068D0B146894568A419A4B22E7820
:10A53800023189B23602A1421E8001D2013502E001
:10A54800016859B14D6829780E431E8003231370A2
:10A5580000200AE006F07F0601361670F22004E0BB
:10A5680000682546002883D1F8E740B2F0BD2DE900
:10A57800F041002549E044892C19A4B2A14242D2F5
:10A58800561ED0F804C0B6B24F1B042E0CEB0705BC
:10A5980001D9F2203CE04FF00008C3F800801CF815
:10A5A800077017F0800FF4D1012A0ED06FB901316E
:10A5B80089B2A142324607D300680028E9D046890B
:10A5C8004568A419A4B200E001354E1C8A18B6B239
:10A5D80092B210E029780F433F02A6421F6007D3CA
:10A5E80000680028D5D0418945686418A4B200E005
:10A5F80001350136B6B296421F68EBD12A78174367
:10A608001F60002004E0006825460028B3D1C0E799
:10A6180040B2BDE8F0812DE9F04100254EE04489C3
:10A628002C19A4B2A14247D2476802F1FF3C4E1B45
:10A63800BCF1030F07EB060501D9F22041E0BE5734
:10A64800002E0BDA4FF0FF361E60012601F1010CD7
:10A6580052181FFA8CFC92B2FF2122E000261E60DD
:10A66800F4E795F800803EB108EA07071F701F68F5
:10A678003F021F60197005E048EA07071F701F684E
:10A688003F021F60A44507D300680028D5D047893A
:10A698004568E419A4B200E001350CF1010C1FFA79
:10A6A8008CFC94451F78DCD12A781EB117401F70A6
:10A6B800002006E01743FAE7006825460028AED1D7
:10A6C800BBE740B2BDE8F0812DE9F04100268DE0FE
:10A6D80044893419A4B2A14280F086804FF0000862
:10A6E800476883F800800AB9002083E08E1BBD19F3
:10A6F80017F806C0BCF12B0F03D101265E600326B4
:10A7080016E0BCF1270F03D8C3F80480BE5D0FE044
:10A71800BCF14F0F06D84FF0010CC3F804C0BE5D62
:10A72800283E05E04FF0020CC3F804C0BE5D503E61
:10A73800013A022792B29E601F7003F10C06002AAC
:10A748004BD0013189B2A14208D3006808B9F22080
:10A7580050E047894568E419A4B23EE001353CE081
:10A768002F7817F0800F23D014E0013189B2013A15
:10A778002CF0800CA14292B20CEBC71708D30068EA
:10A788000028E4D0B0F80AC045686444A4B202E0E6
:10A79800013500E0002795F800C01CF0800F2CD090
:10A7A800012AE2D109E0013A92B20CEBC71701E0A5
:10A7B800013A92B246F8047C62B1013189B2A142F1
:10A7C80007D300680028C2D047894568E419A4B2B5
:10A7D80000E001351F7801371F700436002A83D046
:10A7E8001F781F2FBCD9B2E70068264600287FF4DF
:10A7F8006FAFACE740B2BDE8F081002AD3D1E9E7FA
:10A80800F0B5002A2DD127E044893419A4B2A14219
:10A8180024D247688D1B93423D4405D3059B9EB2C5
:10A82800B21892B2891B11E0F2201EE02E7803F8CC
:10A83800016BCE18B6B2A64207D300680028F3D041
:10A8480046894568A419A4B200E00135D71ABFB2F9
:10A85800012FEBD82A781A70002006E000682646F7
:10A8680000E000260028CFD1DEE740B2F0BD7F2807
:10A8780001D8012304E0FF2801D8022300E00323C4
:10A888000B7070477F2801D801230EE0B0F5004F08
:10A8980001D2022309E0B0F5000F01D2032304E03E
:10A8A800002801DB042300E005230B807047C34325
:10A8B8008342A8BF18467F2801DC01230AE0B0F5CF
:10A8C800004F01DA022305E0B0F5000F01DA032397
:10A8D80000E004230B807047012810B504D9023822
:10A8E800C0B20831012300E00023043908E0013830
:10A8F80051F8044FC0B2E4110133002CDBB2FADC8A
:10A908000028F4D1138010BD10B500230BE0448952
:10A918001C19A4B2A14204D24068CB1AC254002028
:10A9280004E0006823460028F1D1F22040B210BDAF
:10A93800F0B500243FE04389E3189BB2994238D22E
:10A9480045680C1B7F2A05EB040601D82A552EE022
:10A95800FF2A01F101070DD8BFB281219F42295575
:10A9680005D303680BB9F22028E05E6800E00136E1
:10A9780032701CE0BFB24FF0820C9F4205F804C051
:10A9880001D2741C06E000680028ECD045894468B0
:10A998005B199BB2023189B2150A9942257001D21E
:10A9A800013403E00368002BDDD05C6822700020CE
:10A9B80004E000681C460028BDD1D4E740B2F0BDD1
:10A9C800F0B5002537E044892C19A4B2A14230D251
:10A9D80047684E1B052A07EB060510D1013189B2DD
:10A9E8000022A142BA5508D3006808B9F22025E030
:10A9F80042894568A418A4B200E001350422511820
:10AA080012E0013A92B2D60023FA06F62E708E1A98
:10AA1800B6B2A64207D300680028E7D04689456841
:10AA2800A419A4B200E00135012AEAD82B7000204D
:10AA380004E0006825460028C5D1D7E740B2F0BD3C
:10AA4800F0B5002624E044893419A4B2A1421DD2ED
:10AA580047688D1B7D19511813E0013A92B2D60050
:10AA680043FA06F62E708E1AB6B2A64208D30068CC
:10AA780008B9F2200FE046894568A419A4B200E09D
:10AA88000135012AE9D82B70002004E00068264629
:10AA98000028D8D1EDE740B2F0BD2DE9F0430025FC
:10AAA80068E044892C19A4B2A14261D246684D1BC2
:10AAB800012A06EB050801D8F2205EE0D3F800C0B1
:10AAC800BCF1010F05D15F68032F02D12B27775501
:10AAD80006E05F684FF0280909FB0C7C06F805C002
:10AAE800013189B2A14207D300680028E4D0468921
:10AAF8004568A419A4B201E008F10105023AD2B2EE
:10AB0800043331E0013A53F804CFD2B21C260027AF
:10AB18004CFA06F818F0FF0F00D18FB1013189B255
:10AB280048F08008A14285F8008007D30068002813
:10AB3800C2D047894568E419A4B200E0013501276D
:10AB4800073EE5D10CF07F0C85F800C072B10131E9
:10AB580089B2A14207D300680028ADD0468945686C
:10AB6800A419A4B200E00135002ACBD1002004E0EA
:10AB780000682546002894D19EE740B2BDE8F083DE
:10AB8800F0B5002625E044893419A4B2A1421ED2AA
:10AB980047688D1B7D19511812E0013A13F8016BB3
:10ABA80092B22E708E1AB6B2A64208D3006808B9BF
:10ABB800F22012E046894568A419A4B200E00135E4
:10ABC800012AEAD842B11B7800202B7005E0006802
:10ABD80026460028D7D1EBE7104640B2F0BD002347
:10ABE800137070477047002070477047012845D19F
:10ABF80002200B1F9071936011F8043C013B062B57
:10AC08003CD8DFE803F0040B141A222A340001238D
:10AC180013705370042393701A4B25E001231370AB
:10AC2800537006239370184B1B789B0024E0012374
:10AC380013705370432393701DE001231370032393
:10AC4800537004239370114B0EE0012313700323F8
:10AC58005370042393700E4B06E0012313700323F3
:10AC68005370042393700B4B1B681B7804E001237B
:10AC780013705370907004239380704700231370EF
:10AC8800704700BFDC0300208C020020380200203F
:10AC98003402002020040020012809D102239371E6
:10ACA800043993700423916010705070938070473A
:10ACB800002313707047000083681B68012B02D1C2
:10ACC800014B9B8B136070476C02002083681B78D4
:10ACD800013B162B36D8DFE803F00C0E10121416C1
:10ACE800181A1C1E20222426282A2C2E30353535E9
:10ACF8003200022325E0FF2323E0134B20E0134B0F
:10AD08001EE0134B1CE0134B1AE0134B18E0134BD7
:10AD180016E0134B14E0134B12E0134B10E0134BE7
:10AD28000EE000230DE0124B0AE0124B08E0124B34
:10AD380006E0124B04E0124B02E0124B00E0124B0B
:10AD48001B681360704700BFB8BD002040BD0020DD
:10AD580024BD002040BE002080BD00200CBE002085
:10AD680044BE00202CBE0020D0BD002050BE0020D4
:10AD7800A0BD00204CBD002000BE002010BD00205A
:10AD88007CBD00201CBE002008BE002083681B7804
:10AD9800012B02D0022B09D102E01068022801E041
:10ADA8001068FF2814BF002001207047002070475A
:10ADB80001282CD105239371A1F11003936011F898
:10ADC800103C013B0C2B22D8DFE803F0070D0D0DDA
:10ADD8000D0D070D110D070D180002231370032325
:10ADE8005370402307E002231370032102E002237B
:10ADF8001370012151709370042306E0022313702D
:10AE0800012353700623937008239380704700230F
:10AE180013707047012810D151F8043C002B0CDD49
:10AE28001A2B0ADC022393714123043993700423FB
:10AE380091601070507093807047002313707047B2
:10AE480083681B78013B192B43D8DFE803F00D0F0B
:10AE580011131517191B1D1F21232527292B2D2FEA
:10AE680031333537393B3D3F1A4B30E01A4B2EE032
:10AE78001A4B2CE01A4B2AE01A4B28E01A4B26E012
:10AE88001A4B24E01A4B22E01A4B20E01A4B1EE022
:10AE98001A4B1CE01A4B1AE01A4B18E01A4B16E032
:10AEA8001A4B14E01A4B12E01A4B10E01A4B0EE042
:10AEB8001A4B0CE01A4B0AE01A4B08E01A4B06E052
:10AEC8001A4B04E01A4B02E01A4B00E01A4B1B68BD
:10AED8001360704748BD002044BD002020BD0020FD
:10AEE80004BE002038BE002030BD00205CBD00201C
:10AEF800FCBD002074BD002064BD0020A4BD00205E
:10AF08003CBE0020D8BD0020C8BD00204CBE00209B
:10AF1800E0BD002094BD002058BD0020ACBD00203D
:10AF280068BD002048BE0020E8BD0020B4BD002058
:10AF380098BD002060BD0020C0BD002083681B783C
:10AF4800013B0E2B36D8DFE803F0080A0D10121467
:10AF580016181A2A2C2E35303200042329E04FF413
:10AF68007A7326E04EF6602323E00C2321E0124B8F
:10AF78001EE0124B1CE0124B1AE0124B18E0124B69
:10AF880000211B6807E0187E042801D0072801D19A
:10AF9800013189B2DB68002BF5D1116070470B4B8A
:10AFA80006E00B4B04E00B4B02E00B4B00E00B4BB5
:10AFB8001B681360704700BF3CBD002070BD0020B7
:10AFC800BCBD002050BD0020BCE50020CCBD002049
:10AFD80018BE0020ECBD002078BD0020DCBD00209C
:10AFE800012810D151F8043C002B0CDD052B0ADC9C
:10AFF80002239371412304399370042391601070E4
:10B0080050709380704700231370704783681B78D3
:10B01800013B032B0CD8DFE803F002040608054BBC
:10B0280004E0054B02E0054B00E0054B1B6813608C
:10B03800704700BFF8BD0020B0BD002020BE002032
:10B04800A8BD002083681B78013B1D2B4BD8DFE887
:10B0580003F00F11131517194A1B1D1F212325274C
:10B06800292B2D2F313335374A393B3D3F41434654
:10B078001D4B32E01D4B30E01D4B2EE01D4B2CE0EC
:10B088001D4B2AE01D4B28E01D4B26E01D4B24E0FC
:10B098001D4B22E01D4B20E01D4B1EE01D4B1CE00C
:10B0A8001D4B1AE01D4B18E01D4B16E01D4B14E01C
:10B0B8001D4B12E01D4B10E01D4B0EE01D4B0CE02C
:10B0C8001D4B0AE01D4B08E01D4B06E01D4B04E03C
:10B0D8001D4B02E01D4B00E01D4B1B6802E01D4BA1
:10B0E8001B681B781360704754BD002024BE0020E5
:10B0F80010BE002028BD00202CBD002014BE00205A
:10B10800D4BD002054BE0020F0BD0020C4BD0020E6
:10B118009CBD0020F4BD002034BD002088BD002067
:10B128000CBD002030BE002084BD00201CBD0020C6
:10B138006CBD002038BD002018BD002058BE00207E
:10B1480090BD002028BE002034BE002014BD002081
:10B158008CBD00203803002083681B781E2B03D188
:10B16800024B12781B681A70704700BF3803002022
:10B17800012813B5144649D1022393710A1FA2600E
:10B1880011F8042C013A152A40D8DFE802F00B0E1A
:10B198000B0B1419270B2B30303030303030303057
:10B1A80030301437237001221AE001226270042221
:10B1B8002370A27028E023700123637042231AE0F1
:10B1C800086801A901F000F80223237001236370C5
:10B1D8000423A370019B93F8263015E02370032203
:10B1E800627008E0237001236370432303E0237037
:10B1F800012363704123A370042305E02370012316
:10B2080063700623A3700823A38001E00023237042
:10B218001CBD000037B50446806801A904301546F6
:10B2280000F0F0FFA1680C4B8A8A1B68019800E0C7
:10B23800DB687BB11C688442FAD15C8A9442F7D1FE
:10B2480003E0286006E02A6004E00B78012BF8D0C0
:10B25800022BF8D03EBD00BFD8E5002073B50646E6
:10B268008068184B01A904301C68154600F0CAFF15
:10B278000199002302E0013324689BB204B3626899
:10B288009142F8D10AE0636806E0013304E0A3685C
:10B2980002E0012300E000232B6011E0B26812787D
:10B2A800013A042A0CD801A151F822F08FB2020801
:10B2B80093B2020897B202089BB202089FB2020832
:10B2C8007CBD00BFB0E5002030B5836885B0054679
:10B2D80003A95868144600F077FFA86802A9083047
:10B2E80000F090FF039802A96A4601AB02F0CAFF7A
:10B2F800002815DBAB681A78013A032A10D8DFE872
:10B3080002F002040A0D5B6809E0009B1A682260DB
:10B318009B88A38004E0019B1B6800E00323236053
:10B3280005B030BD30B5836885B0054603A95868B7
:10B33800144600F049FFA86802A9083000F062FF2F
:10B34800039802A96A4601AB02F09CFF002812DBB1
:10B35800AA681378022B05D0032B09D0012B0AD138
:10B36800536807E0009B1A6822609B88A38002E06C
:10B37800019B1B68236005B030BD000083681B7803
:10B38800052B07D0062B0FD0042B11D1094B1A68B7
:10B39800094B02E0094B1A68094B9A4208D0FF2969
:10B3A8008CBF002001207047064B1A68064BF4E753
:10B3B80000207047B4030020646D03084003002098
:10B3C8007C6A0308CC040020AC6A0308012820D159
:10B3D8000620A1F114039071936051F8143C022BDC
:10B3E80008D0032B0DD0012B13D102230321137096
:10B3F80051700AE0137003235370042393709080F4
:10B408007047022153701170402393700423938076
:10B418007047002313707047012810B521D102240A
:10B428000B1F9471936011F8043C172B19D80E491F
:10B4380099400BD44FF4802199400CD44FF0C0416F
:10B4480099400ED503231070537006E04123107005
:10B458005070937002E010705070947004239380C1
:10B4680010BD0023137010BD00F1FB1F01281CD173
:10B4780005239371A1F11003936011F8103C052B7B
:10B4880013D84FF03051994008D44FF0A04199405B
:10B498000BD5022313705070402302E0022313706F
:10B4A8005070937004239380704700231370704783
:10B4B800012823D106239371A1F11403936011F895
:10B4C800143C013B032B19D8DFE803F002070F02F5
:10B4D80002230321137051700CE00223137003231D
:10B4E800537004239370062306E00223137003238A
:10B4F8005370402393700423938070470023137084
:10B5080070470000012810B521D102240B1F947147
:10B51800936011F8043C0F2B19D80E4999400BD4AD
:10B528004FF4800199400BD44FF0F04199400ED56B
:10B5380010705070947007E010705070412302E052
:10B5480014705070422393700423938010BD00231D
:10B55800137010BD0000BB07012816D10623937194
:10B56800A1F11403936051F8143C012B02D0022B73
:10B578000BD104E0022153701170402301E01370D5
:10B5880050709370042393807047002313707047A2
:10B59800012810B519D1022393710C1F11F8041C4E
:10B5A80094601E2911D80A4C8C4003D413FA01F177
:10B5B80004D40AE010705070412302E00321107097
:10B5C800517093700423938010BD0023137010BD35
:10B5D800FCFEFF7E83681B781E2B0FD1084B10687A
:10B5E8001968084B994205D0013801288CBF002002
:10B5F80001207047831E5842584170470020704709
:10B6080038030020606B030810B5002302E0CC5C0F
:10B61800C45401339CB2A242F9D110BD83681B788F
:10B62800052B10B50C4611460AD0062B0FD0042B5B
:10B6380015D10B4B22461868FFF7E6FF094B0CE0C3
:10B64800094B22461868FFF7DFFF084B05E0084B57
:10B6580022461868FFF7D8FF064B1B681C7010BD00
:10B66800B4030020380200204003002034020020E8
:10B67800CC04002020040020043905E051F8043FE0
:10B68800013A40F8043BD2B2002AF7D170470000D3
:10B6980073B5836806460D46586801A9144600F03C
:10B6A80093FDB3681A78013A152A5CD8DFE802F0EE
:10B6B8000B0D1115181B222E373A3D4043525246A6
:10B6C800494C4F5252555B6845E0019920462E314E
:10B6D8000CE0019B93F831303DE0019B9B8C3AE0F4
:10B6E800019B5B6B37E00199204627312A46FFF71B
:10B6F8008BFF38E0019B93F82D30D9070DD503F067
:10B708001003DBB203B106E0072324E0019B93F8A2
:10B718002D30DA0701D501231DE002231BE0019B30
:10B728009B6B18E0019BDB6B15E0019B1B6C12E027
:10B73800019B5B6C0FE0019B9B6C0CE0019BDB6C3D
:10B7480009E0019B1B6D06E0019B5B6D03E0019B1B
:10B758009B6D00E00023236005E020460249C5F305
:10B768008702FFF789FF7CBDE86B0308F7B585689A
:10B778000F46281D01A9144600F044FD019B1BB982
:10B78800234A106860B941E0224A106800E0006866
:10B7980000283BD0466883EA060286683242F6D122
:10B7A8002D78013D0C2D31D8DFE805F0070D111477
:10B7B8001414171C212325142A0003B91EE08268DB
:10B7C800436813401AE0214600F00CFD1EE083B9DF
:10B7D800012313E04FF0FF3310E00BB9C3680DE00D
:10B7E80043680BE00BB9042308E0032306E00223B7
:10B7F80004E0002302E003B900E08368236005E069
:10B8080020460549C7F38702FFF736FFFEBD00BF94
:10B81800B4E50020B0E50020FC69030818B1024B2C
:10B828001860024B1960704760030020DC03002099
:10B8380010B5044603F075F90A23034AB0FBF3F088
:10B848001060206010BD00BFE4BD00201346826870
:10B858001278013A10B50C46062A25D8DFE802F01E
:10B8680004070F14171A22001846104B14E0104949
:10B878001846C4F38702BDE81040FFF7FDBE18461E
:10B88800BDE81040FFF7D4BF18460A4B04E018463D
:10B89800094B01E01846094B19682246BDE81040DB
:10B8A800FFF7B2BE48221A6010BD00BF6003002037
:10B8B80090020020B403002040030020CC040020A4
:10B8C80018B1024B1860024B19607047B40300208E
:10B8D8003802002018B1024B1860024B19607047FB
:10B8E800CC0400202004002007B5064802AA818B5A
:10B8F800002342F8043D013100F0CCFC024B012248
:10B908005A820EBD6C020020E40300202DE9F047A6
:10B9180086B00C4601A900F065FC204602A900F09B
:10B928007EFCDFF8A08000251F4CDFF89C90DFF834
:10B938009CA0002D18BF444600260023009301ABAD
:10B94800204653F8261000AAF7B200F0A3FC042FF3
:10B958001DD0009BDBB1DC68CCB900F079FC009B02
:10B968000446D86020B90135EDB2022DDCD112E0D1
:10B97800032F0CD11DB90D4B03600D4B02E00D4B8D
:10B9880003600D4B6360C4F80890C4F80CA001363E
:10B99800052ED2D1E7E7094A01235382084A538288
:10B9A80006B0BDE8F08700BFB8030020D5B3020891
:10B9B8002DB30208B9B40208D1B20208DC01002094
:10B9C800C0010020A8040020EFAB0208F3AB020876
:10B9D800F0B591B00C460BA900F004FC20460CA968
:10B9E80000F01DFC0027264B264D0026002F08BF1F
:10B9F8001D4634460BAB2846F15800AA00F085FCDA
:10BA0800C0B298B101280BD110AB03EB8402009BA4
:10BA180042F83C5C013442F8283CE4B2DD6807E0B7
:10BA2800022805D1009B0024DD6801E00446054694
:10BA38000436142E11D0002DDCD10EE0013CE4B206
:10BA480010AA02EB840353F8281C53F83C0C00910D
:10BA580000F075FC08B100F019FC002CEED101379C
:10BA6800FFB2022FBFD1064B9B8B0BB9064B5C82F2
:10BA7800044B9B8B0BB9054A538211B0F0BD00BF34
:10BA8800B8030020A8040020DC010020C001002029
:10BA9800024B1A6801321A60704700BFB8BD002017
:10BAA800024B1A6801321A60704700BF40BD00207F
:10BAB800024B1A6801321A60704700BF24BD00208B
:10BAC800024B1A6801321A60704700BF80BD00201F
:10BAD800024B1A6801321A60704700BF0CBE002082
:10BAE800024B1A6801321A60704700BF44BE00203A
:10BAF800024B1A6801321A60704700BF2CBE002042
:10BB0800024B1A6801321A60704700BFD0BD00208E
:10BB1800024B1A6801321A60704700BF50BE0020FD
:10BB28002DE9F04186B0043002A900F078FB174CEB
:10BB3800174FDFF86C8000250023019302AB2046E5
:10BB480053F8251001AAEEB200F0A4FB032E15D07D
:10BB5800019B9BB1DC688CB900F07AFB019B044621
:10BB6800D86018B90B4B01225A820BE0022E05D17E
:10BB7800094B80E880018360084BC3600135042DC0
:10BB8800DAD1EFE706B0BDE8F08100BF140300206A
:10BB980075B4020898030020EFAB0208F3AB020863
:10BBA80065B2020870B58EB004300AA900F037FB00
:10BBB80000261F4D34460AAB2846F15801AA00F06A
:10BBC800A4FBC0B298B101280BD10EAB03EB8402E1
:10BBD800019B42F8305C013442F8203CE4B2DD6855
:10BBE80007E0022805D1019B0024DD6801E0044636
:10BBF80005460C2E12D00436002DDCD10EE0013C97
:10BC0800E4B20EAA02EB840353F8201C53F8300C5C
:10BC1800019100F094FB08B100F038FB002CEED144
:10BC2800034B9B8B0BB9034B5C820EB070BD00BFFE
:10BC380014030020980300202DE9F04186B010B1CC
:10BC4800002300932BE08A684B681340009333BBB2
:10BC580021E00023019302AB204653F8251001AAE6
:10BC6800EEB200F017FB032E12D0019B83B1DC6803
:10BC780074B900F0EDFA019B0446D86058B1022E61
:10BC880006D10D4BC0F8008083600C4B4760C36041
:10BC98000135042DDDD10A4B01225A8209E068469C
:10BCA80002A900F0BCFA0025064CDFF82080064FF8
:10BCB800CFE706B0BDE8F081EFAB0208F3AB0208AE
:10BCC800000400204402002075B70208B9AD02083C
:10BCD80070B58EB010B10023009341E08A684B68BC
:10BCE80013400093002B3BD134E00AAB2846F158AF
:10BCF80001AA00F00AFBC0B298B101280BD10EAB23
:10BD080003EB8402019B42F8305C013442F8203C8A
:10BD1800E4B2DD6807E0022805D1019B0024DD6854
:10BD280001E0044605460C2E12D00436002DDCD165
:10BD38000EE0013CE4B20EAA02EB840353F8201C87
:10BD480053F8300C019100F0FAFA08B100F09EFAAD
:10BD5800002CEED1074B9B8B53B9074A538207E05F
:10BD680068460AA9002600F05AFA3446014DBCE795
:10BD78000EB070BD4402002000040020024B1A6877
:10BD880001321A60704700BF48BD0020024B1A6894
:10BD980001321A60704700BF44BD0020024B1A6888
:10BDA80001321A60704700BFC8BD0020024B1A68F4
:10BDB80001321A60704700BF94BD0020024B1A6818
:10BDC80001321A60704700BFE8BD0020024B1A68B4
:10BDD80001321A60704700BF70BD0020024B1A681C
:10BDE80001321A60704700BFBCBD0020024B1A68C0
:10BDF80001321A60704700BF50BD0020024B1A681C
:10BE080001321A60704700BFCCBD0020024B1A688F
:10BE180001321A60704700BF18BE0020024B1A6832
:10BE280001321A60704700BFECBD0020024B1A684F
:10BE380001321A60704700BF78BD0020024B1A68B3
:10BE480001321A60704700BFDCBD0020024B1A683F
:10BE580001321A60704700BFF8BD0020024B1A6813
:10BE680001321A60704700BFB0BD0020024B1A684B
:10BE780001321A60704700BF20BE0020024B1A68CA
:10BE880001321A60704700BFA8BD00202DE9F041BB
:10BE9800044686B001A900F0C2F9638A174F184C0E
:10BEA800DFF86C80059300250023009301AB204642
:10BEB80053F825106A46EEB200F0ECF9042E15D0BE
:10BEC800009B9BB1DC688CB900F0C2F9009B04466A
:10BED800D86018B90B4B01225A820BE0032E05D10A
:10BEE800094B80E880018360084BC3600135052D4C
:10BEF800DAD1EFE706B0BDE8F08100BF61B502080E
:10BF080014020020F8010020EFAB0208F3AB02088E
:10BF18001DB2020870B5044690B00BA900F07FF975
:10BF2800618A2A4B0F911B68002209E01D6820686E
:10BF3800854204D1588A884201D10132D2B2DB68E5
:10BF4800002BF3D1012A04D0214B9B8B002B39D035
:10BF58003AE01F4D1E461C460BAB2846F1586A4670
:10BF680000F0D3F9C0B298B101280BD110AB03EBA4
:10BF78008402009B42F83C5C013442F8283CE4B25D
:10BF8800DD6807E0022805D1009B0024DD6801E098
:10BF980004460546102E12D00436002DDCD10EE0E2
:10BFA800013CE4B210AA02EB840353F8281C53F8AE
:10BFB8003C0C009100F0C3F908B100F067F9002CBF
:10BFC800EED1C1E7034A538210B070BDD8E5002016
:10BFD80014020020F8010020024B1A6801321A608E
:10BFE800704700BF54BD0020024B1A6801321A6026
:10BFF800704700BF24BE0020024B1A6801321A6045
:10C00800704700BF10BE0020024B1A6801321A6048
:10C01800704700BF28BD0020024B1A6801321A6021
:10C02800704700BF14BE0020024B1A6801321A6024
:10C03800704700BFD4BD0020024B1A6801321A6055
:10C04800704700BF54BE0020024B1A6801321A60C4
:10C05800704700BFF0BD0020024B1A6801321A6019
:10C06800704700BFC4BD0020024B1A6801321A6035
:10C07800704700BF9CBD0020024B1A6880181860EA
:10C08800704700BFF4BD0020024B1A688018186082
:10C09800704700BF34BD0020024B1A6801321A6095
:10C0A800704700BF88BD0020024B1A6801321A6031
:10C0B800704700BF0CBD0020024B1A6801321A609D
:10C0C800704700BF30BE0020024B1A6801321A6068
:10C0D800704700BF84BD0020024B1A6801321A6005
:10C0E800704700BF1CBD0020024B1A6801321A605D
:10C0F800704700BF6CBD0020024B1A6801321A60FD
:10C10800704700BF38BD0020024B1A6801321A6020
:10C11800704700BF18BD0020024B1A6801321A6030
:10C12800704700BF58BE0020024B1A6801321A60DF
:10C13800704700BF14BD0020024B1A6801321A6014
:10C14800704700BF8CBD0020014B0360704700BFE3
:10C1580024040020024B1B681B780370704700BF43
:10C168003803002030B5074D2B781F2B08D8064A16
:10C178000C2404FB032407C884E8070001332B7050
:10C1880030BD00BF5CBE002060BE0020D0B1037C83
:10C19800042B05D1838B03B909E043693BB110E057
:10C1A8009A1E012A05D8438A0BB1806904E0012050
:10C1B8007047052B05D1007ED0F1010038BF002063
:10C1C8007047002070470000054B01381B680022AB
:10C1D80001E01B6801320BB18242FADB0B60704749
:10C1E800B0E50020064B00221B6801E01B6892B2F4
:10C1F80001320BB90A6070478342F7D1FAE700BFF2
:10C20800B0E500200278C36842EA0363027A43EA91
:10C2180002434268120643EA12430B6070470378F0
:10C228000B6043784B6083788B60C378CB60704732
:10C2380010B504460B20FAF7E9FE20B1002303608D
:10C2480043608460C36010BD01460B20FAF7F4BE5A
:10C2580008B50A20FAF7DAFE70B1084B0360084BFC
:10C268004360084B8360084BC360042303740023B6
:10C27800438243618361838308BD00BFE7AB020843
:10C28800EDAB0208EFAB0208F3AB020801460A2047
:10C29800FAF7D2BEF8B5054616466C6908463CB9A9
:10C2A800FFF7C6FF50B36861A861306021E03C46E3
:10C2B800A368834202D13460022323E00ADA676864
:10C2C800002FF4D1FFF7B4FFD8B180E89000606088
:10C2D800A8610BE0FFF7ACFF98B1226880E8140072
:10C2E8000AB9686101E0226850602060306001236B
:10C2F80008E0AB8B0133AB83012300E0FF2358B286
:10C30800F8BDFF23012BFAD1F3E7436900E05B682E
:10C318006BB198688842FAD1D96861B1087C042861
:10C3280007D1888B012894BF0120022004E0184619
:10C3380002E0032000E00120136040B2704738B5E6
:10C34800838BCD68013B838343699942044605D1B9
:10C358004B6843617BB100221A600CE08369994203
:10C368000B6804D1836133B100225A6003E04A6844
:10C378005A604A6813600846FFF766FFA38B0BB93B
:10C388006361A361284638BD2DE9F04F044685B0A6
:10C398000D461E4602F104084FF0000B68E0237CAE
:10C3A8009A1E012A12D80DB900206AE0678A002374
:10C3B8009AB2BA42F8D29A006169885858F8041CAF
:10C3C80001338842F4D1A3699B5857E0042B0CD160
:10C3D800002DE9D0636900E05B68002BE4D0996820
:10C3E80058F8042C9142F7D147E0052B2ED1002DA7
:10C3F800DAD0E3696069594698474FF000098446E6
:10C4080003E009F101091FFA89F9E145CCD0606917
:10C4180058F8043C276ACDF804C059464A46B8473C
:10C42800DDF804C00028ECD1E145BDD2594603AB84
:10C43800676A60694A46B847237E0BF1010B9B4542
:10C4480000D10BE05FFA8BFB23460CE0012BABD14C
:10C45800012DA9D1DAF80030002BA5D13570C6F826
:10C4680004A020460DE0013DEDB208F104081C4689
:10C47800A8F1040A002C92D196E7DB68002BF2D1D0
:10C48800ECE705B0BDE8F08F2DE9F04F1D468BB005
:10C49800A44B4FF0000A08AF04460E46904683F8B6
:10C4A80000A005979CE1237C9A1E012A00F28F8048
:10C4B800678A0EB9B1466FE04FF0000C1FFA8CF294
:10C4C800BA4280F06881636953F82C10D8F80030BC
:10C4D80099424FEA8C090CF1010CEFDB2B7805EB44
:10C4E80083077960591C2970D4F818B05BF80900E3
:10C4F80098B9606950F80960D8F80000864200F3DE
:10C508007381608A2B700132824280F244816369B0
:10C5180053F82C3029707B6066E10132618A5FFA3A
:10C5280082FC00270CEB0703DBB28B421AD21BB24A
:10C538009A005BF823300491184603920293CDF8D1
:10C5480004C0FFF723FE01370499039A029BDDF824
:10C5580004C00028E6D1079363699B588DF824002E
:10C56800089301E00023079307A8FFF7FBFD636921
:10C5780053F80920D8F800309A4204D1013EF6B2A7
:10C5880008F1040800E00026A36953F8093040E1E7
:10C5980009F101095FFA89F9B94580F0FC800FFAC1
:10C5A80089F2A36953F822004FEA820BFFF7EEFDE8
:10C5B8000028EDD162692B7852F80B1005EB830245
:10C5C80001332B70A369516053F80B301FE1042B22
:10C5D8004CD16769002E40D000E07F68002F00F042
:10C5E800DA80BA68D8F800309A42F6DB2B7805EB87
:10C5F80083014A605A1C2A70F86878B9B868D8F874
:10C608000060B04200F3F08078682B70002800F0DA
:10C61800C2807B689B682A704B60E5E07C6800E01C
:10C628006468002C00F0E980D4F80C904846FFF7C5
:10C63800ADFD0028F4D1D9E007A8FFF793FDBA684B
:10C64800D8F800309A4204D1013EF6B208F1040845
:10C6580000E00026FB68DCE07F68002F00F09B808C
:10C66800F868FFF793FD0028F6D1C8E0052B40F0E5
:10C678008680002E6ED0E3696069514698474FF076
:10C688000009834603E009F101091FFA89F9D94530
:10C6980000F08180276A6069D8F8003051464A4620
:10C6A800B8470028EFDBD94575D251464A4606AB54
:10C6B800676A6069B8472B78069A05EB83010AF127
:10C6C800010C4A60591C2970217E8C4518D1D8F874
:10C6D80000108A4200F3888009F101025A450DDAF8
:10C6E80006AB666A6069514692B2B0472B78013B47
:10C6F800DBB205EB8305069B6B6075E02B704AE0A7
:10C7080009F10102D2B25A450ED207946069059B1D
:10C71800CDF804C05146676AB847DDF804C08DF803
:10C7280024C003E05CBE00200023079307A8FFF79E
:10C7380019FD276A6069D8F8003051464A46B8475B
:10C7480020B9013EF6B208F1040800E000260AF11B
:10C75800010A11E05146324606AB676A6069B8477C
:10C768002B78069A05EB830101334A602B70237EF0
:10C778000AF1010A9A4537D05FFA8AFA30E0012BAC
:10C7880001D0002047E036B92B7805EB830201334E
:10C7980056602B7028E021494FF0000A0B78204999
:10C7A800524654460C260BE0013BDBB206FB03F273
:10C7B80088188C5890F808A04268287801382870A2
:10C7C8001BB9164F3B7024B9DBE7002CECD013499A
:10C7D8000B702B7805EB830101334A602B70002620
:10C7E800002C7FF460AECCE7204614E0A368CDF8B7
:10C7F8001C9008938DF824001EE707941CE72B78FB
:10C80800BA6805EB830101332B70FB684A60002B83
:10C81800EAD01C46E4E70BB0BDE8F08F5CBE002010
:10C8280060BE002003280DD90B68012B0AD14B6884
:10C83800032B07D18B68062B04D1C868431E5842C6
:10C84800584170470020704700232DE9F041151D1D
:10C85800042834BF80464FF004081C46104F03E0FC
:10C868000134EE50E4B20433444505EB030C07EB06
:10C87800030601D100230CE0DE59C858B042EFDDB1
:10C888000020BDE8F081F15801344CF80310E4B2FF
:10C898000433032CF7D914700120BDE8F08100BFE0
:10C8A8007872030810B5FDF739FA0B4C206040B1D7
:10C8B8000A49A122FDF712FA20680949A122FDF7C9
:10C8C80015F9084B002283F85A205A611A61024B65
:10C8D8001A68054B1A6010BDECE5002059D402080F
:10C8E80064690308F0E5002028E700202DE9F843F3
:10C8F80080460C2089461746FAF788FB044600282C
:10C9080032D000230360436098F800500572ADB13F
:10C918000D20FAF77BFB0646E06028B921460C207B
:10C92800FAF78AFB34461FE0013DEDB208EB8503B8
:10C938005B6846F82530002DF6D100E0C56084F824
:10C94800109067747FB10D20FAF760FB606158B9E9
:10C95800E16811B10D20FAF76FFB21460C20FAF7B8
:10C968006BFB002400E067612046BDE8F88341695D
:10C9780010B5044611B10D20FAF75EFBE16811B15C
:10C988000D20FAF759FB0C202146BDE81040FAF7B4
:10C9980053BB38B50446406803E04568FFF7E7FF36
:10C9A80028460028F9D120722060606038BD70B533
:10C9B800044600220E46D0F80001D4F80C31114686
:10C9C80008E01D7A0572DD681972C560D9600068D3
:10C9D8001B68013294F8F850AA42F2DB04F5867518
:10C9E8002846FFF7D6FF04F5807393E80700002375
:10C9F800012EC4F80031C4F8043184F8083118BF96
:10CA080094F8F830266118BF013385E807006361A0
:10CA1800204601F073F82846FFF7BBFF002384F88F
:10CA28005A3070BD10B5044601F068F804F58070FE
:10CA3800FFF7AFFF04F58670FFF7ABFF002384F81C
:10CA48005A3010BD037A0BB9016002E043681960DF
:10CA58004B60037A41600133037270472DE9F0435C
:10CA68000546A7B0002840F09083B24CA67A012E64
:10CA780040F0D48094F85A30072B25D194F87420CC
:10CA8800D4F85C8004EB82023146743204F1680306
:10CA9800D8F83870B84794F8680048B1082384F883
:10CAA8005A30D8F82C30284604F168019847A6E097
:10CAB80094F87420D8F8483004EB82023146743276
:10CAC8009847204602212AE0082B40F0988004F17C
:10CAD800740094F86A1094F86C20D4F85C80FFF71E
:10CAE80005FF0746A0B17B69D8F83CC07A7C284688
:10CAF80004F16801E04704F586703946FFF7A2FFA4
:10CB080094F8F83084F85A60013384F8F83076E005
:10CB180004F16801D8F84C30984720463146FFF7B1
:10CB280046FF6CE013B9D4F8003102E0D4F8FC30C9
:10CB38001B68C4F8FC30D4F8FC3005AA187AD96808
:10CB4800FFF782FE002800F0FF82D4F8FC30197A43
:10CB5800032905D9DA6878480439C9B2103202E0E5
:10CB6800002175480A4605ABFFF78EFC05460028EC
:10CB780000F0EA82037C052B13D10723E06505A9A1
:10CB880084226E4884F85A30F4F7FCFC9DF814307F
:10CB9800AE6A686905AD0021012205EB8303B04741
:10CBA8002EE002239DF8141084F85A3005AF03686C
:10CBB80007EB8101012002AA984705A89DF80A10F1
:10CBC8009DF80C20FFF792FE0646A8B1032384F8CF
:10CBD8005A306B68BDF80C10726902A8984758481B
:10CBE8003146FFF72FFF012384F85A3094F8F830C4
:10CBF800013384F8F83003E04E480121A6E24D4C99
:10CC080094F85A30012B40F0C08294F8F83094F828
:10CC18000821934286D3A7E2464892E2002E40F0CC
:10CC2800268194F85A30072B22D1E56D94F860904C
:10CC3800D4F86480AF6B04F1680349464246B847AC
:10CC480094F8683063B194F86930DA0708D5082396
:10CC580084F85A30EB6A304604F168019847F7E0E7
:10CC680000204946AB6C424698473248022159E0B9
:10CC7800082B40F0ED800C20D4F85C80FAF7C6F958
:10CC88000546002847D006604660D4F8FC30DA68CC
:10CC98001B7AC2600372D4F8FC301E72DE6094F80E
:10CCA8006A30037494F86C704774EFB10D20FAF78A
:10CCB800ADF90346686138B1D8F83C706A7C3046F3
:10CCC80004F16801B84718E0D8F84C3004F168015D
:10CCD8009847D4F8FC30EA68DA602A7A0C201A728D
:10CCE8002946FAF7A9F91BE0D8F83C60384604F160
:10CCF80068013A463B46B0476F6104F5867029469D
:10CD0800FFF7A0FE012384F85A3094F8F830013375
:10CD180084F8F8309CE0D8F84C3004F16801984762
:10CD280020460121FFF743FE92E05BB9D4F80031B9
:10CD38000BE000BFF0E500209071030864E60020D6
:10CD4800FCE60020D4F8FC301B68C4F8FC30D4F8AA
:10CD5800FC30187AD968FFF765FD002873D0D4F83D
:10CD6800FC30A648197ADA680439C9B210326B4621
:10CD7800FFF70AFB0646002865D0037C052B10D177
:10CD8800E065072398E8030084F85A309C4B9DF827
:10CD9800002083E803000021B56A7069019BA84759
:10CDA80058E0022384F85A30036801999DF800007E
:10CDB80002AA98479DF80830002B44D09DF8093006
:10CDC800DB0700F1C6813EE000222A606A60D4F8E1
:10CDD800FC30D9681B7AE9602B72D4F8FC301A72DF
:10CDE800DA609DF80A302B749DF80C306B74BBB177
:10CDF8000D20FAF70BF90246686120B17768697C63
:10CE080002A8B8470DE0D4F8FC30E968D960297A5F
:10CE1800E8601972287229460C20FAF70DF90DE01E
:10CE28006B6178482946FFF70DFE012384F85A30D4
:10CE380094F8F830013384F8F83003E0724801219F
:10CE4800FFF7B5FD36B970480221FFF7B0FD01E0E4
:10CE58006D4CE84694F85A30012B40F0968194F8CE
:10CE6800F83094F808219342FFF45FAF7CE1032E79
:10CE780040F08B8194F85A30072B1BD1E66D94F85B
:10CE88006090D4F86480B76B4946424604F1680361
:10CE9800B84794F8680040B1092384F85A30336BD6
:10CEA800284604F168019847D5E0B36C49464246E4
:10CEB800984723E0092B24D194F86930E56D03F0F5
:10CEC8000203DBB2B3B1D4F8FC3094F86A101A7CD0
:10CED800914208D15A7C2E6C5B6904F16801B04715
:10CEE80008B1012340E0002048492B6D9847464887
:10CEF800032129E02B6D04F168019847204602219F
:10CF080022E00A2B23D1E66D94F86090D4F864806F
:10CF1800B76B4946424604F16803B84794F868007D
:10CF280060B10B2384F85A30D4F8FC30766B5A7C05
:10CF38005B69284604F16801B0478CE04946B36C48
:10CF48004246984720460521FFF731FD83E00B2B29
:10CF580040F08180D4F8FC30E26D04F16801556C32
:10CF68005A7C5B69A847062384F85A3094F8F8304D
:10CF7800013384F8F8306EE012B9D4F8003102E0D9
:10CF8800D4F8FC301B68C4F8FC30D4F8FC30187AAC
:10CF9800D968FFF747FC002858D0D4F8FC30174868
:10CFA800197ADA680439C9B210326B46FFF7ECF91E
:10CFB800054600284AD0037C052B10D1E0650723DD
:10CFC80096E8030084F85A300D4B9DF8002083E85A
:10CFD80003000021AF6A6869019BB8473DE002275A
:10CFE80084F85A70036801999DF8000002AA9847CE
:10CFF8009DF80830002B40F0B98027E090710308B5
:10D0080050E60020FCE60020F0E5002058E600206D
:10D01800D4F8FC309DF80A101A7C91420ED1AF6802
:10D02800597C5A6902A8B84740B1012384F85A309C
:10D0380094F8F830013384F8F83006E054480321B6
:10D0480001E053483946FFF7B2FC35B95048022190
:10D05800FFF7ADFC01E04E4C6E4694F85A204C4B5D
:10D06800012A51D194F8F82094F808118A4283D300
:10D0780088E0002283F8F820062283F85A2043E04B
:10D0880013B9D4F8003102E0D4F8FC301B68C4F8B6
:10D09800FC30D4F8FC303F48197ADA680439C9B250
:10D0A80010326B46FFF770F9054600282ED0037C36
:10D0B800052B10D1E0650A2396E8030084F85A305E
:10D0C800354B9DF8002083E803000021AF6A6869AA
:10D0D800019BB8471AE0052384F85A300368019980
:10D0E8009DF8000002AA9847062384F85A30D4F81D
:10D0F800FC30ED68597C5A6902A8A84794F8F830C2
:10D10800013384F8F83001E0214C6E4694F85A3027
:10D118001F4D062B39D194F8F83094F80821934222
:10D12800AED331E005F5807207CA05F5867383E84A
:10D1380007000023C5F80031C5F8043185F8083127
:10D148002846FFF76FFC20E011480221FFF72FFC6B
:10D1580056E503230C2084F85A30F9F757FF0546A3
:10D1680000287FF431AE69E60FD155E5042384F831
:10D178005A309DF8093003F00203DBB2002B7FF42C
:10D1880047AF5EE7C0D174E7CCD027B0BDE8F083E5
:10D19800F0E500209071030850E600202DE9F04FDB
:10D1A800C7B00DF10B078A4691463A4604461D461C
:10D1B8000DF10E06FDF744F90AF10101204689B286
:10D1C8000DF10A023346FDF750F910B93B78302BC0
:10D1D80002D0FEF721FF2BE09DF80A8085F80801B0
:10D1E80008F10108D0441FFA88F8C5F80001C5F80D
:10D1F800040118E141463A462046FDF721F908F1B5
:10D208000101204689B20DF10A0203ABFDF72DF9A1
:10D2180040B93B78302B05D1BDF80C2012B13388CA
:10D228009A4207D9FEF7F8FE05F58070FFF7B1FBC3
:10D23800F22009E19DF80A2090441FFA88F808F1C5
:10D24800010AD2431FFA8AFA9B1851463A462046E9
:10D258003380FDF7F5F808F10201204689B20DF197
:10D268000A0203ABFDF701F90028DBD13B78062B56
:10D27800D8D19DF80A10BDF80C2001315144204640
:10D2880089B204ABFDF720FA0028CBD19DF80A300B
:10D29800BDF80C2099188A441FFA8AFA31880AF1D5
:10D2A80001088A1A1FFA88F8DB43D31841463A4620
:10D2B80020463380FDF7C4F80AF10201204689B2FE
:10D2C8000DF10A0203ABFDF7D0F80028AAD139788E
:10D2D800062947D005D8042936D039D80229A1D142
:10D2E80009E0432904D8412919D240299AD169E093
:10D2F800442997D128E004A80422FFF7F7FA8346C7
:10D3080000288FD09DF80A10BDF80C20DBF81430E7
:10D3180001314144204689B2FDF77DF96BE004A84C
:10D328000422FFF7E3FA834600283FF47BAF9DF819
:10D338000A10BDF80C20DBF81430013141442046B6
:10D3480089B2FDF714F956E004A89DF80C203FE0D7
:10D35800052104A80022FFF7C9FA014600283FF476
:10D3680061AF2AE09DF80A10BDF80C200131414454
:10D37800204689B225ABFDF7A7F900287FF452AF04
:10D388009DF894203978920004A802F0FC02FFF777
:10D39800ADFA014600283FF445AF9DF89430406946
:10D3A80009E0013BDBB20DF58C7E0EEB830252F8EF
:10D3B800802C40F82320002BF3D105F58070FFF76F
:10D3C80041FB22E0BDF80C20042A7FF42BAF04A80F
:10D3D800FFF78CFA834600283FF424AF9DF80A1023
:10D3E800437C4069BDF80C2000900131414420463F
:10D3F80089B2FDF705FA8246594605F58070FFF7B0
:10D4080021FBBAF1000F7FF40DAFBDF80C209DF899
:10D418000A30511C591888443188DB438A1AD318BA
:10D428001FFA88F833803388002B7FF4E3AEAB7A99
:10D4380095F80801032B02D1FEF726FE01E0FEF75E
:10D448001BFEA9F80080002040B247B0BDE8F08F6D
:10D458002DE9F043A34D178995F85A6087B099468E
:10D46800002388461446ADF81030002E00F0AA813B
:10D478002046F9F7EBFED6E19DF80E60BDF81230B4
:10D48800751CEB189F4240F0C4809DF80F30302B7C
:10D4980000D0BEE0ADB229460DF10F022046FCF7E0
:10D4A800CFFF2046B11C0DF10E020DF11203FCF75F
:10D4B800DCFF002840F0AD809DF80F30022B40F0D3
:10D4C800A8809DF80E10BDF8122001312046691879
:10D4D80005ABFDF7A0F8002840F09B80059B13B131
:10D4E800FEF78AFDC4E79DF80E20BDF81230D31868
:10D4F800ED18ADB26E1CB6B231460DF10F022046E2
:10D50800FCF79EFFA91C204689B20DF10E020DF111
:10D518001203FCF7AAFF00287BD19DF80F30042BDB
:10D5280077D19DF80E10704DBDF81220009501318D
:10D538007118204689B24023FDF762F9002868D1A6
:10D54800BDF81230A5F11802402B28BF4023D1188E
:10D558009DF80E20ADF8123085F841309B18F6186A
:10D56800B6B206F101081FFA88F808760DF10F0225
:10D5780041462046FCF764FFB11C204689B20DF1F4
:10D588000E020DF11203FCF770FF002841D19DF83F
:10D598000F30A02B0FD15548F4F786FA29460246DA
:10D5A8005248F4F7E3FA20B1FEF72EFD00F07EFDB5
:10D5B8005EE74E480CE0A32B12D14D48F4F774FAFD
:10D5C800294602464A48F4F7D1FA0028ECD14848DF
:10D5D800F4F76AFA06462846F4F766FA8642E3D173
:10D5E8009DF80F30A03B042B13D8DFE803F00306A7
:10D5F800090C0F00FEF750FD00E1FEF755FDFDE0B8
:10D60800FEF762FD34E7FEF757FDF7E0FEF764FD2D
:10D618002EE7FEF701FD2BE731460DF10F022046FC
:10D62800FCF70EFF08F10201204689B20DF10E0247
:10D638000DF11203FCF719FF0028EAD19DF80F300D
:10D64800022BE6D19DF80E10BDF812200131711899
:10D65800204689B205F10C03FCF7DDFF0028D8D17C
:10D668009DF80E20BDF81230D318F618B6B2771C04
:10D67800BFB239460DF10F022046FCF7E1FEB11C9E
:10D68800204689B20DF10E020DF11203FCF7EDFEF2
:10D698000028BED19DF80F30022BBAD19DF80E108C
:10D6A800BDF8122001317918204689B205F110031E
:10D6B800FCF7B1FF0028ACD12B69013B042B1BD828
:10D6C800DFE803F00306090C1800FEF7ADFC13E0D1
:10D6D800FEF7B2FC10E0FEF7B7FC0DE0FEF7BCFC6D
:10D6E8000AE000BFF0E5002008E60020D6C10020CF
:10D6F800EAC10020FEF7B8FC9DF80E20BDF81230F4
:10D70800D318FF18BFB27D1CADB229460DF10F0228
:10D718002046FCF795FEB91C204689B20DF10E0291
:10D728000DF11203FCF7A1FE00287FF472AF9DF8FB
:10D738000F30022B7FF46DAF9DF80E10BDF812204C
:10D748003A4B01316918204689B2FCF764FF00287A
:10D758007FF45FAFBDF812309DF80E2001339B189F
:10D76800ED18334BADF810509A7A32B19A7A012AF3
:10D7780003D09A7A032A7FF47BAE1B692C4D002BC9
:10D788007FF476AE6B69002B7FF472AE06AA204652
:10D7980032F8081D2B46FFF701FD06462046F9F72B
:10D7A80055FD002E3FD195F80831002B3BD00123C1
:10D7B8002E6130466E6185F85A3085F8F860FFF7BB
:10D7C8004DF930E0FEF708FCD9F80030C5F80080C4
:10D7D8006B60BDF8383031462B810DF10F022046C1
:10D7E800FCF72EFE204601210DF10E020DF1120369
:10D7F800FCF73BFE00283FF43FAE0AE79DF80F30E8
:10D808000B4D03F01F03AB729DF80E3098441FFABE
:10D8180088F808F10106B6B2BDF81230BF1BBB424A
:10D828003FF4FAAEF5E607B0BDE8F08304E6002061
:10D83800F0E50020F8B50025064644682F4651E07B
:10D84800237C062B20D005D8022B0CD024D3042B04
:10D8580022D316E0432B03D8412B0BD2402B00E0F8
:10D86800442B19D10DE0636904F120011868FDF714
:10D878001EF812E0636904F120011868FDF702F848
:10D888000BE0637C238408E0607C6169800804F114
:10D898002002FDF721F800E02784208C04F11A010A
:10D8A800FCF7E5FF04F11E02207AE168FDF714F8A1
:10D8B800E08B04F11901FCF7DAFFE38B208CC01828
:10D8C800A37E0230C018637EC01880B2A08304F122
:10D8D8001801FCF7CCFFA38B227E646801339B18E8
:10D8E800ED18ADB2002CABD12846758106F10901BF
:10D8F800FCF7BDFF737A0133E81880B2F8BD000069
:10D908002DE9F047044600F58C750F46406904F58B
:10D918009071FCF7CCFFB4F820012946FCF7A7FF6B
:10D92800206994F81881B4F820A104F59171FCF7E6
:10D93800BEFF691CB4F82201FCF799FFB4F82291E4
:10D94800E06894F8196104F59271FCF7B0FFB4F837
:10D95800240104F58D71FCF78AFFD144B4F8243111
:10D9680009F10309994418FA89F894F81A314644D8
:10D97800F61817FA86F6B6B2E91C3046A4F82661FE
:10D98800FCF775FF94F8590094F81B81A4F8280156
:10D9980004F58E71FCF76BFF144B94F81C71186832
:10D9A800B4F8289104F59571FCF781FF691DB4F866
:10D9B8002A01FCF75CFFB4F82A5194F81D314D4454
:10D9C800033545447D19ED1816FA85F5ADB228469C
:10D9D800A4F82C5104F58F71FCF749FF94F81E3117
:10D9E8000133E81880B2BDE8F08700BF88720308E9
:10D9F80070B51646044601360D460846B6B21146BD
:10DA08003022FCF781FF284631466289FCF790FFF7
:10DA1800637A64E0314601363022B6B22846FCF714
:10DA280073FF3146A28B2846FCF782FF237EF61847
:10DA3800B6B2314601360622B6B22846FCF764FF74
:10DA48003146E28B2846FCF773FF637E227AF6188C
:10DA5800B6B23146E3682846FDF71FF8E38B227C0F
:10DA6800F618B6B231460136B6B22846FCF74CFF76
:10DA780031462846228CFCF75BFFA37EF618237CF0
:10DA8800402BB6B21CD006D8042B19D0062B1ED0BA
:10DA9800022B23D104E0432B0AD9442B1ED10FE0DB
:10DAA8006369228C1B6828463146FCF7C9FF15E0DC
:10DAB8006369228C1B6828463146FCF781FF0DE01C
:10DAC80028463146228C6369FDF75AF806E0627CE5
:10DAD8006369284631469208FCF7DFFF238C2468E7
:10DAE800F618B6B2002C95D1304670BD18B901B100
:10DAF8000968014B1960704720E70020F0B504461B
:10DB080085B00C22002101A804F58676F3F7F4FD10
:10DB18003046FFF78FFE01462046FFF7F1FE03224D
:10DB280001460020F9F7DFFB054690B90123236180
:10DB3800606101A8FFF77EFE01462046FFF7E0FE80
:10DB4800032201462846F9F7CEFB0546002800F0D7
:10DB5800DC80002130222846FCF7D6FE0121B4F8EB
:10DB68002C212846FCF7E4FE94F81E710222791C49
:10DB780028460237FCF7C8FE3946B4F82A21284659
:10DB8800FCF7D6FE94F81D31B4F82A21FF18614B32
:10DB980039461B682846FCF753FFB4F82A31FF18AA
:10DBA800BFB2394601370422BFB22846FCF7ACFEA3
:10DBB8003946B4F828212846FCF7BAFE94F81C31F7
:10DBC800B4F82821FF18BFB2394604F118032846D3
:10DBD800FCF7D6FFB4F82831FF18BFB23946013731
:10DBE800A222BFB22846FCF78FFE3946B4F8262198
:10DBF8002846FCF79DFE94F81B31FF18BFB2394642
:10DC080001370222BFB22846FCF77EFE3946B4F837
:10DC180024212846FCF78CFE94F81A31B4F8242104
:10DC2800FF18BFB23946E3682846FCF709FFB4F885
:10DC38002431FF18BFB2394601370222BFB2284645
:10DC4800FCF762FE3946B4F822212846FCF770FE3C
:10DC580094F81931B4F82221FF18BFB23946236964
:10DC68002846FCF7EDFEB4F82231FF18BFB239465A
:10DC780001370222BFB22846FCF746FE3946B4F8FF
:10DC880020212846FCF754FE94F81831B4F82021D6
:10DC9800FF18BFB2394663692846FCF7D1FEB4F8CD
:10DCA8002031FA183046294692B2FFF7A1FE2369BF
:10DCB800013B042B0FD8DFE803F00306090E0C0024
:10DCC800FEF712FA07E0FEF717FA04E0FEF71CFA6F
:10DCD80001E0FEF721FAFEF727FAFEF785F9228917
:10DCE8002068211DFBF7CCFF29462068FBF7C3FFFE
:10DCF800B0F1FF3F0CBF4FF0FF3600262068FBF75E
:10DD0800E5FF2846F9F7A2FA00E0FF2670B205B051
:10DD1800F0BD00BF887203082DE9F04F114B17467C
:10DD28001A7985B005460E46002A00F0B8811868B1
:10DD3800002800F0B4810C4C60601846FCF710FA1B
:10DD480043682561C3F3072223736273062DC3F367
:10DD58000742C3F30763A273E373676106D1A66042
:10DD680008E000BF20E7002028E7002004F10800B1
:10DD7800FEF7EAF9BB48BC4CFDF75AFDBB48FFF774
:10DD880059FD04F132010646A069FCF77BFD608E5F
:10DD980004F12801FCF76BFDB4F832C06069CDF8D6
:10DDA80004C004F1340194F82890FCF780FDA08E9B
:10DDB80004F12901FCF75BFDA38E2069029304F1AD
:10DDC800360194F829800425FCF771FDE08E04F1F2
:10DDD8002A01FCF74CFD284604F12B01B4F836B0B3
:10DDE80094F82A702587FCF742FD94F82B20A16847
:10DDF800039211F8040BB4F838A004F13A02FCF7C6
:10DE08006BFD608F04F12C01FCF731FDDDF804C0D7
:10DE1800029B628F634405339B44DA4412FA8AFA00
:10DE2800D144C844039B17FA88F7DF1994F82C30BB
:10DE3800FF1816FA87F6B6B2304604F12D01062708
:10DE4800A687FCF714FD384604F12E0194F82DA09E
:10DE5800E787FCF70CFD864B94F82E90D3F80080EA
:10DE6800B4F83EB0404604F14001FCF720FDB4F898
:10DE7800400004F12F01FCF7FAFCB4F840309B4451
:10DE88000BF1030B94F82F30DA44D144994416FA75
:10DE980089F6B6B2304604F13001A4F84260FCF7C6
:10DEA800E6FC94F830300133F118002089B20322DF
:10DEB800F9F719FA0646002800F0F380002130220D
:10DEC800FCF722FD0121B4F842203046FCF730FD72
:10DED80094F83090022209F10101304609F1020953
:10DEE800FCF712FD4946B4F840203046FCF720FD07
:10DEF80094F82F30B4F840209944494643463046B8
:10DF0800FCF79EFDB4F8403099441FFA89F92A4677
:10DF180009F101054946ADB23046FCF7F5FC294642
:10DF2800E28F3046FCF704FD94F82E30E28FED18AE
:10DF3800ADB229464F4B3046FCF722FEE38FED1871
:10DF4800ADB229460135A422ADB23046FCF7DCFC5F
:10DF58002946A28F3046FCF7EBFC94F82D30ED18DB
:10DF6800ADB2294601353A46ADB23046FCF7CCFC95
:10DF78002946628F3046FCF7DBFC94F82C30ED180C
:10DF8800A368ADB2294613F8042B3046FCF785FD8B
:10DF9800638FED18ADB2294601354022ADB2304647
:10DFA800FCF7B2FC2946228F3046FCF7C1FC94F8F6
:10DFB8002B30228FED18ADB2294604F10C03304600
:10DFC800FCF7DEFD238FED18ADB22946013502229C
:10DFD800ADB23046FCF798FC2946E28E3046FCF795
:10DFE800A7FC94F82A30E28EED18ADB229462369D1
:10DFF8003046FCF7E5FCE38EED18ADB22946013555
:10E008000222ADB23046FCF77FFC2946A28E30468C
:10E01800FCF78EFC94F82930A28EED18ADB2294693
:10E0280063693046FCF7CCFCA38EED18ADB22946E7
:10E0380001354322ADB23046FCF766FC2946628EB4
:10E048003046FCF775FC94F82830628EED18ADB2B6
:10E058002946A3693046FCF7B3FC638EEA183146BB
:10E068000AE000BF40E7002028E7002044E700203E
:10E07800887203088C72030892B204F11C00FFF73F
:10E08800B7FCFEF759F8FDF7AFFF2246314652F8C4
:10E09800040BA223FBF7DBFD3046F9F7D7F8002085
:10E0A80000E0FF2040B205B0BDE8F08F07B50DF1E4
:10E0B8000700FEF74FF89DF80730012B09D1002122
:10E0C800044B04200A46D961196283F82410FFF72B
:10E0D80023FE0EBD28E70020F8B54C6806460D461D
:10E0E8001746194606222046F3F74CFA3946A01D72
:10E0F8000622F3F747FA0823237300236373B369EF
:10E10800304629469847F8BD70B50B4D1424444352
:10E118002919064604314868FDF75AFC285918B1F0
:10E12800F9F794F800232B51142303FB0655002319
:10E13800AB74103570BD00BFE4BF00202DE9F74F68
:10E1480000250A24354A01910646A846AA462B46C8
:10E158002746A446A3460A2F92F8129004D1B9F193
:10E16800000F04D1DFB223E0B9F1000F20D02EB1A7
:10E1780030685168884201D118464BE0B9F1010F67
:10E188000ED1106892F8139020B1A94510D3DCB2D3
:10E198004D460DE0D1450BD35FFA83FBCA4607E035
:10E1A80006D992F81390C14524BF5FFA83FCC8468C
:10E1B8000133DBB214320A2BCDD1019A02F00203EB
:10E1C800DBB233BB0A2F02D1D30702D421E0FCB261
:10E1D80011E0BCF10A0F02D05FFA8CF408E0BBF141
:10E1E8000A0F02D05FFA8BF402E00A2C11D0E4B2D5
:10E1F8002046FFF789FF094B26B11422316802FB3C
:10E2080004325160142202FB04330022DA742046DF
:10E2180000E0FF2040B2BDE8FE8F00BFE4BF002051
:10E2280070B50D4C00250226A37C83B1E27C013237
:10E23800D2B2EF2AE27403D8012B05D1012A06D9FC
:10E248002846FFF761FF02E0032B08BFA6740135DB
:10E2580014340A2DE8D170BDE4BF002070B5084D14
:10E2680006460024AB7C2BB1AB68B34202D12046F2
:10E27800FFF74AFF013414350A2CF3D170BD00BFF3
:10E28800E4BF0020F8B50846022116461F46FFF7EE
:10E2980055FF00280CDB1424074D444329198B7CB7
:10E2A800012B05D90C460C3404313460396000E088
:10E2B800FF2040B2F8BD00BFE4BF00202DE9F843BD
:10E2C80000220646884600F1270700F104092A21A2
:10E2D8000320F9F708F8054600283CD044680120D7
:10E2E800F7F776FE3946A082062204F11600F3F706
:10E2F80049F9062204F120001949F3F743F90622E7
:10E3080020461849F3F73EF9A01D39460622F3F7CF
:10E3180039F94946042204F11C00F3F733F9414660
:10E32800042204F12600F3F72DF900230122A37338
:10E33800E27363740822062304212274E1742273B1
:10E34800A3746373B3693046294698470446284640
:10E35800F8F77CFF00E0FF2460B2BDE8F88300BF57
:10E3680099720308937203082DE9F04107460E4697
:10E37800086839461546FBF703FE002857D133686D
:10E3880003F0F002E02A52D0002B50D00121304691
:10E39800FFF7D4FE041E4FDB3149142202FB04139D
:10E3A8001033987808B90120987002FB0412937C06
:10E3B800012B00D035B938463146FFF77FFF0246BA
:10E3C8000DB936E0FF22142325496343C818807C21
:10E3D80001280BD9234ACB1814703846294607F16F
:10E3E80027020C33BDE8F041FFF776BE23D12B4658
:10E3F80003E01A7B012A28D11B68002BF9D11EE003
:10E408002946F9F727F820B13046F8F71FFF24E02E
:10E418002E461423124A03FB04F1154650581F4692
:10E4280008B1F8F713FF7C432E51002404E0F224CE
:10E4380002E0044600E0144660B2BDE8F0812846D8
:10E44800F8F7E1FF002DE3D107E003201989002246
:10E45800F8F749FF06460028D2D1FF24ECE700BFB1
:10E46800E4BF0020E0BF00202DE9F041104B154625
:10E4780014220E4602FB053107468A7C022A01F166
:10E48800100408D1CA7CE32A05D90431FFF716FF26
:10E4980008B90323A370064B142202FB0533384640
:10E4A800314607F127020C33BDE8F041FFF714BEEF
:10E4B800E4BF0020F7B504460E4608460E2115466F
:10E4C800F8F799FE002863D128682146FBF758FD24
:10E4D800002855D12B6803F0F002E02A14D101235B
:10E4E8008DF800305E238DF802306B788DF80100CE
:10E4F80003F07F038DF80330AB788DF80430EB78A8
:10E508008DF805306B463CE0626883EA0201A26838
:10E51800114209D09BB24FF6A962934204D0E36836
:10E5280004F10C010BB935E029461C4B1A781C4B39
:10E53800142000FB0233987C012804D908685B6822
:10E54800984200D10DE00023154F1A46F818857C33
:10E55800012D0BD90D684068854207D10F4BD2B207
:10E568001A7020463146FFF77FFF14E0143301325A
:10E57800C82BD2B2EAD120463246FFF7F5FE0AE0B0
:10E58800084B2046314604F12702FFF7A5FD02E0BB
:10E59800FE2000E0FC2040B2FEBD00BFE0BF00202E
:10E5A800E4BF0020937203082DE9F04F43890E2B36
:10E5B80087B004460D4640F2ED80406803788689AE
:10E5C800DA0713D5012B08D143787BB983785E2B02
:10E5D8000CD1637B43F0100307E072490622F2F77F
:10E5E8009FFF18B9637B43F008036373082E04D0B8
:10E5F800B6F5C16F40F0CE8014E095F82D3003F0E9
:10E608002003DBB2002B00F0C58020466FF00D011F
:10E61800F8F7F1FD002840F0BD8020462946FBF7B9
:10E62800C3FDBAE095F82D3003F02003DBB2002BD0
:10E6380000F0B0806389292B00D8ABE06668F389C5
:10E64800B3F5807F40F0A680B37C062B40F0A28013
:10E65800F77C042F40F09E80338A082B40F09A8084
:10E6680006F11C0A51463A4604A8F2F78BFF06F158
:10E6780026020392114605A83A46F2F783FF6B6813
:10E688002BB1059AD11A4A424A41019200E00193FE
:10E69800019B049806F11607002B0CBF4FF00208E7
:10E6A8004FF0010805F1270900283DD02946FBF75E
:10E6B80067FC0290002837D1049A02F0F002E02AA1
:10E6C80032D004A84146FFF739FD00282CDB364B31
:10E6D8004FF0140808FB00F803EB080102228A74C3
:10E6E8008D6001F1100B284604310093FDF70EF9F7
:10E6F800009B03EB080006220C303946F2F742FF74
:10E70800029A8BF80320009B53F808B0BBF1000F66
:10E718000AD043F80820284659464A463B46FFF7A0
:10E72800DBFC5846F8F792FDB38AB3F5807F03D037
:10E73800B3F5007F2ED129E0019B5BB30220F7F7E8
:10E7480047FCB082514604220398F2F71BFF291DAB
:10E7580004225046F2F716FF3946062206F1200039
:10E76800F2F710FF394606223046F2F70BFF49460A
:10E7780006223846F2F706FF4946B01D0622F2F790
:10E7880001FFAB6928462146984703E0284604A9BB
:10E79800F8F7F4F82046F8F759FD002007B0BDE86F
:10E7A800F08F00BF93720308E4BF002008B5FFF79D
:10E7B80037FD044941F288300022BDE80840FAF7E5
:10E7C800CBBF00BFB5E702082DE9F04FDFF8C480E2
:10E7D80085B000216422D8F800000B46F5F744FD07
:10E7E8000128F6D1DFF8B0A0DFF8B09001A800F05A
:10E7F8002FFE039E376817F4004701D0002416E067
:10E808000320BDF80410DDF808B00246F8F76BFDE8
:10E8180004460028F2D0054668686A890BEB0701B0
:10E82800F2F7B0FE6B892D68FF18002DF4D1DAF8E5
:10E8380000309A68012A88BF1E684FF00040002205
:10E8480002E03060F668013299688A42F9D3002202
:10E858009A60D9F800301B0604D58023C9F8003027
:10E868000A4B1A60002CB4D0094B196820460B6972
:10E878009847014618B12046F8F7E8FCA9E7D8F808
:10E8880000000A460B46F5F7EFFCAFE70890024098
:10E89800ACC00020B4C00020B00801201490024091
:10E8A80070B5194E35680C465DB90120294603221A
:10E8B800F5F769FB306020B129462A462B46F5F763
:10E8C8009FFB114B00211868FA220B46F5F7CCFC88
:10E8D800C0B10E4B1B6800259E6807E0701961687F
:10E8E8006289F2F74FFE63892468ED18002CF5D190
:10E8F800A8B200F0FDFD044B2146186822462346C5
:10E90800F5F77EFB002070BDB0C0002044EA00206F
:10E91800732330B580F82E30742380F82F30374BAE
:10E92800374D4361374B87B083610623044680F82F
:10E93800263004A8F5F70AFA9DF81030296884F8FB
:10E9480027309DF8113084F828309DF8123084F86B
:10E9580029309DF8133084F82A309DF8143084F853
:10E968002B309DF8153084F82C3040F2DC53A3840A
:10E97800222384F82D30244B1C6019B91420F5F794
:10E9880029FB286004F12701002000F049FD1F48F9
:10E998001F49204D052200F031FE1E481E49052260
:10E9A80000F000FE002405EB44100121013400F0C2
:10E9B8004BFE052CF7D1154D002405EB44104FF400
:10E9C8004001013400F03CFE052CF6D1002404235C
:10E9D80096228DE8180011490294234603941048A2
:10E9E800F5F720FD00F086FE41F288300D492246F9
:10E9F800FAF7B2FE204607B030BD00BFBDE40208FA
:10EA0800B4C00020A9E80208ACC0002048EA0020F1
:10EA180054090120B4080120E8EA00209F72030885
:10EA2800D1E70208B5E7020810B5002204460846F7
:10EA38000421F5F7A8FA2060002814BF00206FF021
:10EA4800000010BD1FB50B4A019112680068002331
:10EA5800039301A91AB103AAF5F78AFB02E013464A
:10EA6800F5F7CEFAC0B2013818BF6FF0000005B054
:10EA780000BD00BFB8C000202DE9F34107460C4691
:10EA88009046F5F733FE054604B901ACB8F1000F1E
:10EA980015D0134B1E6816B1F6F742F9FEE7386831
:10EAA800214642463346F5F7DFFB012803D1F5F747
:10EAB8001DFE401B11E026604FF0FF300DE00023E3
:10EAC800386821464FF0FF32F5F7CEFB0128F6D122
:10EAD800F5F70CFE401B08BF0120BDE8FC8100BF14
:10EAE800B8C0002010B504460120F5F717FB2060D8
:10EAF800002814BF00206FF0000010BD10B50446B8
:10EB0800002120684FF0FF320B46F5F7ADFB0128D6
:10EB1800F6D110BD002100680A460B46F5F770BA19
:10EB28007047F5F7E3BD70B586B006460A9C1546F2
:10EB3800009405AA0024019202949AB2039408460C
:10EB48002B463146F5F76EFC01280CBF0598204688
:10EB580006B070BD08B5034B1B680BB9F6F7E8F8AB
:10EB6800012008BDB8C00020024B1B680BB9F6F79E
:10EB78000BB97047B8C0002038B5204C204D238809
:10EB88005A1CB3F5167F228014D90020F4F786FFAB
:10EB9800F7F779F940F2F230F5F7DAFEBFF34F8F65
:10EBA800184A194BD16801F4E0610B43D360BFF3F5
:10EBB8004F8FFEE7154B1A78D2B1002214481A700D
:10EBC80095F85D3000F12E0185F82F30F2F70EFF31
:10EBD800104800F12E01F2F709FF0F4800F12E014D
:10EBE800F2F704FFF7F74FF90C4B1868F5F7F2FC4A
:10EBF8004FF47A70F5F7ACFEC1E700BFBEC0002045
:10EC0800D8C0002000ED00E00400FA05F40400205C
:10EC1800DAC00020E9C00020F8C00020C0C00020F1
:10EC280030B5484D85B000241CB1012C40F08580DA
:10EC380004E04548F8F70EF801247EE0424882686F
:10EC480043680292C26801930392002B45D0F7F7FC
:10EC5800E9FF95F8CE3201A803B11BE0FBF77AFA79
:10EC68003A4902463A48F4F737FD02A8FBF772FA28
:10EC7800364902463748F4F72FFD03A8FBF76AFA2E
:10EC8800324902463448F4F727FD95F82F3001A899
:10EC980085F85D30FBF75EFA2C4902462F48F4F7F9
:10ECA8001BFD02A8FBF756FA284902462C48F4F740
:10ECB80013FD03A8FBF74EFA244902462948F4F746
:10ECC8000BFD3220F5F744FE042000F0BBF9264B7B
:10ECD8001868F5F77FFC02242FE0036A5B7B032B9F
:10ECE8002BD9F7F79FFF95F8CE324BB11B48FBF7AE
:10ECF800DEF901901A48FBF7DAF90290194808E0A2
:10ED08001348FBF7D4F901901248FBF7D0F90290A9
:10ED18001148FBF7CCF901A902AA03AB03900A48F2
:10ED2800F8F7F0F93220F5F713FE042000F08AF91D
:10ED38000D4B1868F5F74EFC0324FA20F5F708FE8A
:10ED480072E700BFD8C000206CE70020D8FB02089B
:10ED5800DAC00020F8C00020E9C0002008C1002067
:10ED680026C1002017C10020C4C0002030B50020F3
:10ED7800364C8DB00146F7F709F994F82F50002367
:10ED880084F8CE3225B1049305930693009328E0C6
:10ED9800A01CFBF78CF9049004F12000FBF787F91D
:10EDA800059004F11100FBF782F994F82F300690D2
:10EDB800A11C04F1300084F85D30F2F717FE04F16D
:10EDC800200104F14E00F2F711FE04F1110104F1E3
:10EDD8003F00F2F70BFE07A81D49A21CF4F77CFCC4
:10EDE80000951C4B1C4801931C4B04A905AA0293CF
:10EDF80006ABF8F795F91848F8F7BAF91648F8F78E
:10EE0800C7F9124B93F82F307BB102230093144BB0
:10EE1800144801930023029303934FF4807212491C
:10EE2800F5F700FB114B01221A70084B93F8CE320C
:10EE380053B10F4A0F4801920023009302930393A2
:10EE48000D498022F5F7EEFA0DB030BDD8C000208C
:10EE5800A672030819E902086CE70020555F02084A
:10EE6800C4C0002029EC0208AC720308BCC0002012
:10EE7800C0C0002081EB0208B772030810B5124C1D
:10EE880094F82F2094F85D309A4204D00120F4F7CA
:10EE980005FE012010BDA01C04F13001F3F784F831
:10EEA8000028F3D004F1110004F13F01F3F77CF8D6
:10EEB8000028EBD004F1200004F14E01F3F774F8B8
:10EEC8000028E3D0002010BDD8C0002083681B783C
:10EED800022B01D0032B03D10B1F58425841704716
:10EEE80000207047134682681278013A10B50C4624
:10EEF8000C2A12D8DFE802F00A07070A0A0A0A0AE7
:10EF08000A0A0A0A0A0000221A6010BD03491846B4
:10EF18002246BDE81040FCF777BB10BDB8E80020DA
:10EF2800012838B514466BD1022393710B1F9360E7
:10EF380011F8043C013B0C2B62D8DFE803F0070D05
:10EF4800121E242A30363C42484E54002E4D2F487B
:10EF58002946F4F755FC4BE02C482B49F4F762FDA1
:10EF680003E02A482849F4F76BFD012323700323A3
:10EF780063700223A370042340E0234D23482946ED
:10EF8800F4F7E4FB34E0204D20482946F4F7B0FBC1
:10EF98002EE01D4D1D482946F4F7ADFB28E01A4D1B
:10EFA8001A482946F4F7A8FB22E0174D17482946C6
:10EFB800F4F7A8FB1CE0144D14482946F4F7A8FB05
:10EFC80016E0114D11482946F4F7A8FB10E00E4D44
:10EFD8000E482946F4F7A8FB0AE00B4D0B482946D2
:10EFE800F4F7A8FB04E0084D08482946F4F7BAFBF3
:10EFF8000123237063700423A3702B78A38038BD8A
:10F008000023237038BD00BFC8C00020B8E8002026
:10F0180008B5136882681278022A02D0032A10D130
:10F0280008E0012B0DD1032000F00CF8BDE80840E2
:10F03800F6F722BF012B04D10020BDE80840F6F7FF
:10F048002BBF08BD1FB50D4B8DF8070003EBC000A3
:10F05800C37893B10A4C2068F5F79AF982B22AB9B5
:10F0680020680DF10F011346F5F7FEF8002220681D
:10F078000DF107011346F4F7C3FF1FBDBCE90020DB
:10F08800B8E9002038B5154C154D04F1FA012046B1
:10F09800F2F7ACFC29462046F2F794FB20461149CA
:10F0A800F2F790FB29462046F2F78CFB04F1C801E1
:10F0B8002046F2F787FB29462046F2F783FB04F542
:10F0C800F9712046F2F77EFB2046F2F7EDFC06497F
:10F0D80008702046BDE83840FCF7A0BB36C10020C8
:10F0E800F72D0308D4FB0208C9C0002010B5044658
:10F0F800F2F7DAFC034908702046BDE81040FCF737
:10F10800DFBB00BFD0C0002010B50446F2F7CCFC2E
:10F11800034908702046BDE81040FCF7DBBB00BF80
:10F12800D1C0002010B5054C2146FAF742FF002057
:10F138002146BDE81040FEF7D9BC00BFCCC0002076
:10F1480070B50720B4B00121F3F7D6FB01214FF4C5
:10F158008040F3F7DDFB0120F3F718FC8623002439
:10F168000225039364488DF81050032303A98DF8F2
:10F1780011308DF812408DF81340F3F717FB012179
:10F188000B225D48F3F75BFB0B225B482946F3F73C
:10F1980056FB0B2207215848F3F751FB4FF46053F5
:10F1A8005648039303A9F3F701FB0B210A4653487A
:10F1B800F3F745FB0C210B225048F3F740FB0B22D9
:10F1C8000D214E48F3F73BFB32234D48039303A927
:10F1D800F3F7ECFA4A4801210B22F3F730FB4848D1
:10F1E80004210B22F3F72BFB0B2245480521F3F7EB
:10F1F80026FB4FF40056012342488DF8103003A92E
:10F208008DF8133003968DF812408DF81150F3F7EE
:10F21800CDFA3C483146F3F710FB019444F61F63DE
:10F2280002E0019A01320192019A9A42F9D93548CD
:10F238004FF40051F3F7FFFA0023019344F61F63DC
:10F2480002E0019A01320192019A9A42F9D94FF0EB
:10F2580060600121F3F750FB00F068F800F0FEF958
:10F2680000F004FA0128FBD005A800F06CF84FF470
:10F2780000730F934FF0007326932E934FF480334F
:10F288002F934FF4800301254FF4001230934FF46D
:10F29800005300242892319304224FF480432946D6
:10F2A80005A82D92339305950C94109413941694F5
:10F2B800189419941A9425942A942B9400F080FA9F
:10F2C800114E29463060114800F0E2F94FF44070C1
:10F2D800F3F7ECF83D238DF8083002A805238DF8E4
:10F2E80009308DF80A408DF80B50F3F7E9F83368C8
:10F2F80003B9FEE734B070BD0000024000040240CC
:10F308000008024000100240D4C000204000010064
:10F3180084B0002301900393019B01E0039B013B10
:10F328000393039B002BF9D104B0704708B5012162
:10F338004FF00070F3F7F8FA4FF000700021BDE8C5
:10F348000840F3F7F1BA4FF4804242614FF400628B
:10F358000262402202642022426480220123426623
:10F368004FF080620360C0F8802000234FF00072E5
:10F3780043608360C36003618361C36143628362E6
:10F38800C362036343638363C3638364C3640365C2
:10F3980043658365C36503668366C366036743671E
:10F3A8008367C367C0F88420C0F8A4204FF4803274
:10F3B800C0F8A8204FF480024FF40011C0F8AC2028
:10F3C8004FF40052C0F88830C0F88C10C0F8903064
:10F3D800C0F89430C0F89830C0F89C30C0F8A0301D
:10F3E800C0F8B020C0F8B430C0F8B830704700009A
:10F3F800044B1A6810B142F0080201E022F008023A
:10F408001A60704700800240044B1A6810B142F03D
:10F41800040201E022F004021A60704700800240F2
:10F428000B794A7943EA0222074BC2508A78CB7893
:10F43800120442EA03620B781A434B7842EA032229
:10F44800024BC250704700BF4080024044800240D7
:10F4580037B500230193244B1A68244B01241B68F9
:10F4680033E00199013101911968890505D51968B9
:10F47800C90502D41360946009E01968C90508D465
:10F488001968890500D504E0916801319160DB684D
:10F498001BE0164A1360144A1268536091680131E0
:10F4A80091609168012908BF136019689468C1F3D5
:10F4B8000D410439012C8ABF12689A6892680B4C76
:10F4C800DD6880E80600256007E01968002906DA8B
:10F4D800064A1360002303604360836003E00199D8
:10F4E8000429BED9F4E73EBDB008012040EA002057
:10F4F800294B1B681A68002AF0B548DB40F2F45221
:10F50800904217D9B0FBF2F402FB140292B2A1B2F6
:10F518000AB1013101E001290CD0204D00F2F4506C
:10F5280005FB0105ED04ED0C1A46002040F2F456E7
:10F538004F1E0CE01A68C00442F04052C00C1A601A
:10F5480058601A6842F000421A60DA6814E018B984
:10F558001C6844F080541C60B842566004D114689A
:10F5680044F00054146055601468013044F00044BD
:10F5780014608842D268EAD3074B1A60084B5A696C
:10F58800500706D504225A6100225A6001E0002083
:10F59800F0BD0120F0BD00BF44EA00200CFAFFFFD7
:10F5A80000900240114BF0B51860002400F12003D0
:10F5B8004FF0004544F2F456571E0FE0BC422CBFF2
:10F5C80084469C4643F8181C43F8205C43F81C6C9E
:10F5D80043F814CC0134203301F2F4519442EDD1B4
:10F5E800034B044AD860044B1A60F0BD40EA00207F
:10F5F8000090024034EA0020B00801200E4BF0B51C
:10F608001860002400F120034FF48015561E0DE009
:10F61800B4422CBF07461F4643F8181C43F8205C29
:10F6280043F8147C0134203301F2F4519442EFD1B1
:10F63800024B1861F0BD00BF44EA00200090024070
:10F648000368194301607047436811B123F0004310
:10F6580001E043F00043436070470000024B1A6822
:10F6680042F001021A60704700900240024B18688D
:10F6780000F00100704700BF00900240034B5B6937
:10F6880018420CBF00200120704700BF00900240C4
:10F69800044BDA6909B1104301E022EA0000D8619D
:10F6A800704700BF00900240014B5861704700BF8F
:10F6B80000900240024B9A6942F480129A617047A6
:10F6C80000900240044B9A6910B142F4005201E0E4
:10F6D80022F400529A61704700900240044B9A69E4
:10F6E80010B142F0020201E022F002029A61704772
:10F6F8000090024008B50120FFF77AFEFFF7DAFF15
:10F708000120FFF781FE0120FFF7DCFF0120BDE8A3
:10F718000840FFF7E3BF000082B000230193114BBC
:10F728001A69C00602F01C02890142EA104201F47B
:10F73800F8610A4342F001021A610B4A019901314A
:10F7480001911969C90702D501999142F6D9074B68
:10F75800019A9A421DBF034B586980B2002002B03B
:10F76800704700BF00800240FEFF0400FFFF040056
:10F7780013B5002301930F4B1C695A6104F01C0454
:10F7880044F00304C006890144EA104401F4F86116
:10F798000C43094A1C610199013101911969C80793
:10F7A80002D501999142F6D90198044BC01A18BFA5
:10F7B80001201CBD00800240FEFF0400FFFF040082
:10F7C800F0B587B00023904F00930446019302A838
:10F7D8000E463D69F3F74AF8039B8C4A8C499A1800
:10F7E8008A4225F01C0502D845F0080515E0894A2B
:10F7F80089499A188A4202D845F00C050DE0874AD3
:10F8080087499A188A4208D9864A9A18864B9A4292
:10F8180094BF45F0040545F010053D6130460021D0
:10F828004FF40042FFF7A4FF08B90020E9E07F4841
:10F83800FFF76EFD2168002950D07D4D019B3046B1
:10F84800013301210193FFF767FF00F0040080B244
:10F8580010B9019BAB42F1D9019A764B9A42E4D098
:10F86800002130464FF480520191FFF781FF0028B4
:10F87800DBD06F4D019B3046013301210193FFF727
:10F888004BFF00F0200080B210B9019BAB42F1D9C8
:10F89800019A684B9A42C8D000251F21304601952D
:10F8A800FFF73AFF00F01C0008280BD002D8042804
:10F8B80023D110E00E280AD012281ED14FF400637D
:10F8C800236200E025624FF48043636115E04FF442
:10F8D8000063236200E0256265610EE0226A6369C5
:10F8E800D20842EA5302304692B2FFF741FF00289D
:10F8F8009BD06FF07F40FFF70BFD434B4E4A1968D2
:10F90800A0680A4061680843E16808432169084320
:10F9180061690843A1690843E1690843216A08430A
:10F92800616A0843A16A0843E16A0843216B0843F6
:10F93800616B01430A431A60A26BE16B1143226CAD
:10F948001143626C1143A26C1143E26C1143226DA6
:10F958001143626D0A435A60A26D9A60E26DDA60E3
:10F96800626EA16E98691143E26E1143226F1143D2
:10F97800626F11434FF6417202400A43216E42EA18
:10F9880001419961E16FA26F0A43DA6103F580537F
:10F998002A4A9969D4F884000A40D4F880100843A8
:10F9A800D4F888100843D4F88C100843D4F8901081
:10F9B8000843D4F894100843D4F898100843D4F8AE
:10F9C8009C100843D4F8A01001430A439A61D4F864
:10F9D800A820D4F8A4101143D4F8AC2041F40001B5
:10F9E8001143D4F8B0201143D4F8B8200A43D4F80E
:10F9F800B41042EA81021A601A6842F080021A6062
:10FA0800012007B0F0BD00BF0080024000D3CEFE49
:10FA1800BFE1E40040F1E9FD3F787D0100796CFC2D
:10FA2800FF596202001F0AFA7FF0FA02FFFF0F0077
:10FA3800FEFF0400FFFF04000F8120FF233FDEF8D4
:10FA4800002100F004B80D4B5B58435004310C48BA
:10FA58000C4B42189A42FFF4F6AF0B4A00F003B879
:10FA6800002342F8043B094B9A42FFF4F9AFF2F73E
:10FA780093FFF1F729FDF3F739FA70477C7403080F
:10FA880000000020D0040020D00400201827012006
:10FA9800FFF7FEBF0020202020202020202028283B
:10FAA8002828282020202020202020202020202036
:10FAB8002020202020881010101010101010101076
:10FAC80010101010100404040404040404040410A6
:10FAD8001010101010104141414141410101010134
:10FAE80001010101010101010101010101010101FE
:10FAF800101010101010424242424242020202020A
:10FB080002020202020202020202020202020202CD
:10FB1800101010102000000000000000000000007D
:10FB280000000000000000000000000000000000CD
:10FB380000000000000000000000000000000000BD
:10FB480000000000000000000000000000000000AD
:10FB5800000000000000000000000000000000009D
:10FB6800000000000000000000000000000000008D
:10FB7800000000000000000000000000000000007D
:10FB8800000000000000000000000000000000006D
:10FB9800000000000000000057445400496E6974DA
:10FBA8005461736B00486172646661756C740D0A08
:10FBB80000256420D0B4D0BD2E20256420D1872E06
:10FBC80020256420D0BCD0B8D0BD2E00312E300006
:10FBD800257300747275650066616C7365006F6EDD
:10FBE800003139322E3136382E312E320031393249
:10FBF8002E3136382E312E31003235352E3235350C
:10FC08002E3235352E30007075626C6963004254AF
:10FC18002D3637303100302E302E302E300030382F
:10FC28002E30372E323031360045432D34432D34B3
:10FC3800442D30302D30302D3041004B4E2D303397
:10FC48002D30303030310054324F4B0049444C4550
:10FC5800000925630925750925750925750D0A000B
:10FC68004C610308B5290308C129030834040000BE
:10FC7800010000002F696E666F2E68746D6C0000BD
:10FC8800485454502F312E3120323030204F4B0DF4
:10FC98000A5365727665723A206C7749502F312E77
:10FCA800332E312028687474703A2F2F736176616F
:10FCB8006E6E61682E6E6F6E676E752E6F72672F2F
:10FCC80070726F6A656374732F6C776970290D0A97
:10FCD800436F6E74656E742D4C656E6774683A2058
:10FCE800313130320D0A436F6E6E656374696F6E21
:10FCF8003A20436C6F73650D0A436F6E74656E74BA
:10FD08002D747970653A20746578742F68746D6CF9
:10FD18000D0A436F6E74656E742D456E636F64696A
:10FD28006E673A20677A69700D0A0D0A1F8B080002
:10FD380000000000040A9D56DD6EDB36147E159621
:10FD4800DB450C58767337609280220BB60E4D1B3C
:10FD5800A019B05D0DB444DB6C2552A32827C1500F
:10FD68002049BBEEA2050A04BB18866E43DFC01B00
:10FD7800EA2D5DEAF415A837DA39A4E44488BB61B2
:10FD8800BB902DF2FCF2E3F71D3BBCF1C9BDADBD44
:10FD9800AF76B7C9D4E4591CE227C9989C4494C2E9
:10FDA8008AB3340E736E1849A64C97DC44B432E318
:10FDB800E023B0B9DDA93145C0BFA9C42CA25F06B4
:10FDC8005FDC0AB6545E30234619A72451D2700965
:10FDD80021B7B7239E4E781B2459CE233A137CBFF4
:10FDE80050DA5CF1DB17A99946299F8984076ED1FF
:10FDF800175218C1B2A04C58C6A3CD7ECE0E445E91
:10FE0800E5AB755572ED160C4A4637A1841126E309
:10FE1800B1FDD12EEB27F6A23EB26FEDBC7E6ACFC4
:10FE2800EA17E1D0DBC24CC88764AAF938A23913B3
:10FE380072909425259A67112DCD61C6CB29E706C6
:10FE4800320DFDF1472A3D8CC354CC4892B1B28C97
:10FE5800A864B311D3C47F05291FB32A33ED722CCC
:10FE68000E781A185540826B310166E4DA9BE290ED
:10FE7800354D0899F28301420F60F81A999A286C57
:10FE880081C10369DACF36E2034A440ADD735905B2
:10FE980002706E5CABAC8D87E6DA8EE0D57BE34B07
:10FEA8000C875F5B38B6BF024E47760E782DEA9313
:10FEB800FAA87EE6ABA3FFD5182081117252FA7E0C
:10FEC80063FB33841D6380BDB06FEC5FF66C7D9877
:10FED8009063D53D224B8C980129D65F151E1CCB0B
:10FEE8000E2B60A587E00A9CFB9A150500E950686F
:10FEF8007806679B6EBE271B18420007319BB14CE2
:10FF0800A440512583913A40E0B0C258E9DC99EF0A
:10FF1800DFDDD9C55E29C1FE948CA8EB3C99084A5F
:10FF280080F25305293EDDDE833883946BF1F68B2E
:10FF3800A6AD1527CC2870B9C059C393B6DE52496F
:10FF48000ED5B5E3823D05EC16F66DFD8238FC7FD3
:10FF580003D69E20FA06B4B73EC6755A1546E4285D
:10FF68002AE73874155C95D8BE84BB780D39CFEB79
:10FF7800E7AB348E2F2AE5D9DA881FE0164FEC9CC0
:10FF8800D877EE22CFEC9FF6774C82570B6FF34E63
:10FF98009A422B40707DE95360CF517D8C7A234083
:10FFA800A95F3A81E3FD19D725A0BAAE879D5B5BAF
:10FFB80004E8F71AD1A88F3B71394B589AA26EAE54
:10FFC8009FF51516B467C0BD65FDCCBE2176097DC9
:10FFD80023878F3A29604E48A72844B503D6A93D00
:10FFE800C7B20817443D6DA3E250C8A232C41C161C
:08FFF80030AD0C3F8049E52704
:020000040803EF
:1000000097DA972DF59AD746B448A200D9A81528B3
:10001000194655C6E504261ADDBC8993E97AEF2F07
:10002000F1A400F0857D07CF393C7F401B4B38CDD4
:10003000E2DFDB280FCB3B2A714CF63AC856ABFF08
:10004000DBCF4F0E3A000FB00436385C41CF9E88AC
:10005000EF072451394C22C00739B65AFCD72686FF
:100060004E437138AA8C51B2C1DD2F285132C94498
:10007000F230A29A9B4A4B5256A35C98DB20D48D57
:100080005EFFC6E66A6E8E8C24F004851639D3872F
:10009000305D5E819CBE8393CC1157101628C22719
:1000A000850BC10B832F3F60FD9C2F132D8AABB7AF
:1000B0003E7CC066CCEF5252EAA4F9CD7850E28D76
:1000C000FAFD38FCC7A878C2CDE7F7EFDDDDB81C34
:1000D00025FD7125DD78D990BD6F3FDCA08D967B25
:1000E0000321815B9FEDEDDC89E4C06FF6C19C3B91
:1000F000DD76AD6E0F8DAD1ABBE666171D2E55D79A
:100100007559EDBB128DC4BA2E8DF0D0C10BA86B02
:10011000767B68F43AE80D60B8561C5A776B34ACBD
:10012000387969BBC25BF468F972E9D0ECF42B93BF
:10013000EC32CD7284C2247DC94DFBDBF335FC1B50
:1001400091139E8265CDEEA30EBAF0BF419B0D0ABE
:10015000BF530B523F069DCF516820BBE730EC5098
:1001600075F5E3FA7BCF0CE2AC4B37481603DA7B2C
:10017000D4FBF8F28A87EE0FD2DFD1C282D33009E6
:1001800000002F73657474696E67732E68746D6CEC
:100190000000485454502F312E3120323030204F3F
:1001A0004B0D0A5365727665723A206C7749502F71
:1001B000312E332E312028687474703A2F2F7361DA
:1001C00076616E6E61682E6E6F6E676E752E6F72E1
:1001D000672F70726F6A656374732F6C776970290B
:1001E0000D0A436F6E74656E742D4C656E6774688E
:1001F0003A20323037330D0A436F6E6E656374698F
:100200006F6E3A20436C6F73650D0A436F6E7465B1
:100210006E742D747970653A20746578742F6874E3
:100220006D6C0D0A436F6E74656E742D456E636F51
:1002300064696E673A20677A69700D0A0D0A1F8B30
:10024000080000000000040AB558DD6EDCC6157E0B
:10025000159A69835D40DC956C2428EC25815676DF
:10026000035F241512A76EAE8C5972B43B11FF4A7E
:100270000E77A51A06643B4D03246880F62628DA1B
:10028000187D83B522278A64CB409F807CA37E673C
:1002900086E4CE52F27F7CB112399C39FFE73B7382
:1002A000CEE8C2D53F6CDEF86CEB9A359551E88DFF
:1002B000E8AF15B278E2DA36DE380BBC51C425B3AC
:1002C000FC29CB722E5DBB90DBCE6FF04DAD4EA501
:1002D0004C1DFEE742CC5CFB4FCEA7BF7536932882
:1002E00065528C436E5B7E124B1EE3C8F56B2E0F7E
:1002F00026BC3914B388BBF64CF0799A64D2D8374F
:1003000017819CBA019F099F3BEA654DC4420A16BA
:100310003AB9CF42EE6EAC456C574445D4BE17395E
:10032000CFD40B034B771D2CA49021F7CAFF948BDD
:10033000EA6E75AFDA2F4FCB9FCBE3F26834D45F10
:1003400046A18877AC69C6B75D3B62221EF8796E1C
:100350005B190F5D3B977B21CFA79C4BD0196AE5BA
:10036000C749B0E78D0231B344E0DA7E52C4D29976
:10037000672CC58E95C52099C7584BBDF25FE0F834
:10038000A4E67C529E948FAA7DAB7C58DD2F0FF1A2
:1003900078CF2A9FD24AF9A8FCA95C943F54FBF875
:1003A000F023DE9E58D5DF9A0FD6284F596C308C3B
:1003B0008B68CC33DB7B6F34A42F9E55DDC59163F6
:1003C0001C7D521E0E46C314E2421A43A429F7773D
:1003D0003E4D0326F916837EDE683BC9228BF95217
:1003E00024315C6BC17BD3040AA5494ECA42EC7F21
:1003F0009407A079581E55F7CA4724E542D9EEA4C0
:10040000FAC6C2EA49F5AD551E547F856E87E502EE
:100410008F96D2E1C7F2A87C6C61F12124390505E1
:10042000A88BA723DAFD94CE575F61C701D95F8BF4
:1004300029E2B4904AB3741ED896DC4B110A2944C1
:100440009C2719DEFD108FAE4DC23A143E5912DAC8
:10045000561A329F4F9330E0996B970F9682B5FBF7
:10046000C3642262DBCAC55F40EDE23AD463BB21BC
:100470008F2788267BE37DDBD211D7B2F146E34C90
:10048000FFB4385A8A712165022ACACF61927387F4
:100490000EB43CC632B6F0730224077C61CD5858C6
:1004A000805BF93DECF55869BDB03D6B6452CC8B77
:1004B000712428C0B5560D85BCF07D4E9493D80F9D
:1004C00085BFE3DA1997451623C7E0B5AD9B577B87
:1004D000FDB50B1BAB1CC8980B1812DEA9BE81C35F
:1004E0008664A2C6EB4BDFD79C62361BB30C6AD383
:1004F0003F27E0DBAC0865F3BA2D7679E0C8A409A4
:10050000E195330E453D851A45B7376275A28838A7
:10051000E0BB030287561BD83C2141D8AA14CD89E1
:1005200077B421231E178E802BEBAD45D85803C21C
:100530003512E151EFA6070F097A2E63AF76FD82DF
:10054000CC4DF9557DADB9D37EF30C604A8A7892D3
:10055000AFCA4BB13F03069D870CA443978A88B767
:10056000134DC12BBF43427F8160DE07EB45F5256C
:10057000C5F792F5B0006E9E710161444A71A261A7
:10058000432121749B6E9C2B009647300DED455CFA
:1005900009E42DF2D41927BB6436A2AFD2973ED31B
:1005A0000362A3C9E456577F229659FDC1B51B3893
:1005B000D8E09364636CC3A1DAD3FA5D6F506C9793
:1005C000EB7000818569CD77F2384A9741ACCD78E0
:1005D000838D6DEF938F3EDC5A9A61E54CCCE51C20
:1005E000A6FE2F390AB971507DBDC49473FDD73171
:1005F00022692A79949A3203F8A8849056B5C0B437
:1006000012AA8885BBC16E0579815B8AF7E31A70EF
:10061000170899FB3A685AA85CA14348BF4A9F1043
:10062000C8B988B531E0D102941DC3FB5F54F747C8
:10063000C3F18A1C0AAE265952504A856CCC430B32
:100640004BAECD772529712B023891DB8F80F44F8B
:10065000AA6F091C01FCC86742CA2FCB05828F0E06
:1006600079A39C87DC978D7A8A6C8D8296C2152738
:100670008F744099946B74339710349A144852BD18
:10068000F8DF62B3AE1C0AF90C1121D73F21042A0E
:1006900065537CE8AD158870B2AD4506875B53A104
:1006A000EA862E478AE8990C78A15518A21B65079F
:1006B000D51075E517B60B6877ED42ECDEAE5DD868
:1006C0006EC72EDA26672C63C6D577CAF6A728FE32
:1006D0000886F218370518E46E7B497888AAFAB3C1
:1006E000AAAD3F94A75495A93CEBC001043D270C4B
:1006F0008D3451654563491D6766916ABFD6F61A08
:10070000331DB4BECC00F69488AB2B285A532A81F3
:10071000EDFA2712B78C5E1FC50FCE3CC64DE1EF38
:100720005046D5A9368CB4058CB06B48FEF2996161
:1007300052EE68A498BD9508309876228012E88C15
:10074000FF9F95192D99B7901926EDAE5DDE5A667B
:10075000184C3B763133C37C6E6AD66AD141C522D0
:10076000AC57556F861BED0B0A812E4CCF45792374
:100770001633DC786EF9491415E83550013EC6BBD6
:10078000853E46BFB7314C9E34F346020EDBF26421
:1007900042B54E9A0ED5DAE4DD55F39EFA1EE08995
:1007A0009818A2CD3321B929DB4D5A7873E1BA7478
:1007B0006BE9CE2CBF40BC88C50C77E1EB5BC07108
:1007C0002AF5FBD442A0DBD9785DA32D09D6122DE2
:1007D00017CED8A6FD8402BDC2FDE21B73BFD8D4DC
:1007E0000E9347D737EDB74B1DFE97DE98FFA53325
:1007F000FCC1A3869125981034AB7B56735FA8B3D8
:10080000045B0DF0EFDE915E7C257B6EDE1894DBE1
:10081000C25187EC6A7AB45F6B4F06531FB73992A7
:10082000593F2DCB08BD1B35E4012ADE096E6A75E0
:100830000DB1AE6F39287887082ED4458B9A205495
:10084000C0537511BF8732434DF35DDDDFD7C56DF2
:1008500009B9462689940501DA9A556A60D3CE080B
:10086000541D3E302E63AF98F035875ADD865F37D2
:100870006A26B8167764F88A4A264D035E376E40BA
:10088000B3E64AD4BB1C2396EF2042FF8DAB2BD995
:1008900009BDFB5398EF102F7437C758C430DB2BBA
:1008A000E09B22DB6629B1508C4D2CD7CFA9A5C681
:1008B0002AAEAD063A9737D6D77F4D7B55B35DF755
:1008C000FF4DE75D5FC79B3E39CD44C4B2BDB37DEC
:1008D000B2EEAB7F8F4E28D7AD325A43C4074611D4
:1008E000F5F4013D322E478A055AF297E1D574F5A9
:1008F0002A40F9CCC9385A2695D80F41F994AEC48C
:10090000AF446FCEB2989A121DF18AE0384988E25E
:10091000038248C8B91CFFFC446E7945FAED0CA16E
:1009200011B850C31ED0FFBE3B8B519D9752A29D64
:10093000C5B4CCF4E888AA578B2F7AE095FB994888
:1009400065ED1F2A75C3CFD98CE9550C5A32BF1EED
:100950009E7D4EEDE250AFA35578DE29EFEA671F8A
:10096000DDBA79ED7703348FF900E62DD2DE6D1113
:100970005CB6815BAA3F5DC3306F33497604CF2FED
:100980005F58BFD3BF32A319864C31E29B89F48FE5
:10099000346FB9828DAAB747870BD7FFAA67635A0E
:1009A000E8D4BAF707CD4065BB88D5A4ABD7BF8DD7
:1009B0002DC6D0AE3F50C13808448EA9D21EEEB02D
:1009C00061E2EFD84448019631327BC6D63B6AEFEC
:1009D000723CF43A4CE304179897E2A9762A96A45D
:1009E000A70ECA7339361A5BB889DF9E635C93CC55
:1009F00007504DCD11067AD88996D09C8BDCD970E2
:100A0000DD09979B1F5CEF61FE846F031A21F4DF01
:100A10007D178F3744C49342F6F8DA06BFD437F80F
:100A2000AB183E570046532CFAACC8AC2D89339016
:100A3000ECBDBC1768C0AA66A9CFB0FF9AF226ED3C
:100A4000E85D58EFF7EF5C5946DF508DB0FF0F0BB4
:100A5000405D3DD21600002F6D61696E2E6A7300F5
:100A6000000000485454502F312E312032303020B5
:100A70004F4B0D0A5365727665723A206C77495078
:100A80002F312E332E312028687474703A2F2F7333
:100A90006176616E6E61682E6E6F6E676E752E6F19
:100AA00072672F70726F6A656374732F6C776970E9
:100AB000290D0A436F6E74656E742D4C656E6774F4
:100AC000683A20373739320D0A436F6E6E656374AA
:100AD000696F6E3A20436C6F73650D0A436F6E74D5
:100AE000656E742D747970653A206170706C6963FD
:100AF0006174696F6E2F782D6A61766173637269B4
:100B000070740D0A436F6E74656E742D456E636F5D
:100B100064696E673A20677A69700D0A4361636899
:100B2000652D436F6E74726F6C3A207072697661D6
:100B300074652C206D61782D6167653D38363430E1
:100B4000300D0A0D0A1F8B080000000000040ACDBA
:100B50005C7973DCC695FF2A20A250030F381CEA8B
:100B6000B093198253BA6C2B6B1D2BD1EB64298681
:100B700085A36706E20C300630A218925549BC39AD
:100B8000AAEC8AABBC7FECD6D66EA5F61B385E2BE2
:100B900051ECC4A9DA4F407EA3FDBDD7DD4003333D
:100BA00094E4A376B7128B83461FAF5FBFFBBDC62D
:100BB000709E84459C26D68596EF1C65A298678911
:100BC00015A5E17C2A92A23312C5AD89A09FD70F4B
:100BD0006F47E87132D4FDF1EA469AEEC782C6D972
:100BE000F35C587991C56161F78769D67AE26756F7
:100BF000E095F384DCD30DBDA093CF2671D1B2FB79
:100C000096EDB891D7ED479B616722925131EE473F
:100C1000EDB67344238517EE44BBBAAB673BFD7852
:100C2000D8123BDD5DCFF31D05E3419C44E94167EC
:100C30009E883CF46702AF37769D13F9D2B62B3805
:100C4000F30A4E377043B940E4F96DDBB3DB6A1247
:100C50003545C0EB845B5D0D45220EAC9B7E21FAD1
:100C6000A28369B6E32996219CF02FA77DF9F56E42
:100C7000F7B5F0B50D7199B612B5B129F1741667D3
:100C800022C7D4A253A46FDDD97E08A424A39673EF
:100C9000D2C0851755204662220A5161B3D99560AA
:100CA000ADA6DE1ECF5DABBB61FDC84FAC8D1FBED8
:100CB000D1B5BADD1EFD7FC3C2727D63E7433F122B
:100CC000B7939CCEC7EFE4C5E14474D2991FC6C563
:100CD000A1D775CB730C5A72B7A137F3B35CBC398B
:100CE00049FDA2D5E8CF7869856DAFD3BDEC6C6DB9
:100CF000AC782B4051A38F17F6E9E8222F13EFCFE2
:100D0000455EBC99F94097AD9E7084512B704E4E54
:100D1000808972E9C82FFC371948C0A0A9C6F776A8
:100D2000FCD08D42374EF68618EDA6F342FE981D94
:100D3000646EE0177B386EBC4C44B65788E98C9AD9
:100D40000A9CCC440C0B37BF9F1E88CCCDAFA34D63
:100D50006487BB6E000A0B367D4D610128AC44CB25
:100D60004E0082298109C722DC7F58E0B4014CD5AE
:100D70003CF3133191CDBE1B6854059D423C05FDEB
:100D8000270558A3AF28D21FB440DE8CE7309DA4BE
:100D90009977ED9D6B0FEEECBDF5E0D6ADBBEE9314
:100DA0003406023A0CF7DBDB77DEF12E6EE698DBD9
:100DB0000A277E0E7299FAD9FE5ABA6F6F6DAE533A
:100DC000F3D6C576E838BDA5F33DB875F39566F35F
:100DD0002753FF717DC26A5B04429809DA2DC8A3CC
:100DE000C9ADFCE2A6120238C81149809603FEADD7
:100DF0004893FB28E1D0B2A3F8098E98CE3034F6A0
:100E0000E8F7C3CE30CEF2E2C6389E447D27E8F83C
:100E1000B39948227E44CFEA9DA391185430D24121
:100E2000DD9B831817696DA34EBF900E90389335E4
:100E3000D0E75567B3EB68D28C62481BFFD0B39301
:100E40003411765F4C72C17B0DCF25D2708148255D
:100E5000B9B4F8F0F5BC151BE916BD52707C6C07EF
:100E60009334DCB72B0843C561C14B392C200EBB32
:100E70007A2E87052FE5B0B0C161892820B80A48CD
:100E8000A07C2F1CFBC94800F7A07340049CD945E7
:100E90003617B6E72DE9B5BABA62B68AA7229C170B
:100EA00022728E96B5421C3064BE6790D5C54DD077
:100EB0008415479E8D339F1CAE69384091B3ADD3E6
:100EC0004F4EFF7AFAFCF42FA79FF2DF67AE75FA58
:100ED000F9E997671F5BA77F3BFB39BF788617F45B
:100EE000DF73349EFDE2F4D9D92FF1F8D9D98767A1
:100EF000BFB2D0FAE9D92FCE7E899E5FA1F10B6AED
:100F000078869F7F38FB15FEFD9C877F656124BA3C
:100F1000FE8D5A30F633CCF0737A87611F75ACD3EF
:100F20007FE5497E73FACC4207AC6261F407E8F9C9
:100F3000C1D92F69B93FD0DC67BF2508CE3EB44E7A
:100F40003FB368F93374A7BEE8BDD1B500FC73BCEC
:100F5000C580CEE6FA6C6BD3B7C699187A76982618
:100F600020EB69271CC5B6E6EEA0482CFCB716D1CD
:100F70000964F6D6E9EF9781B5B9EE83FD81B5AD89
:100F80008B90965A050769740896CA45565C176097
:100F90003030AC5B7F191273DD4D239143433AAE81
:100FA00022D80BAD26E21D104725EE5248D0B0D80E
:100FB0009BA6495CA4994115D880F9862965058DC1
:100FC000E8B957D141A3E17C12D82AE920124FE2B7
:100FD00050AC892C4B8183CD60091500F59F9D7D18
:100FE0007CFAA7B38F700AD6BBF71FF2D95AC0326A
:100FF000CE9B89E52B1CE5977C0E9FAE6CAE070A55
:1010000061DF29DA6A7012D2486E588D0DAFAEB624
:101010001A2DDECA860BA4D74777A054213BE9746A
:101020000CB968DB86E2C1994EFFC19FC4D086B07F
:10103000C394ACF03D4C05111BED85E9743AC7191A
:101040001DC25E0AA8F5208B0B516B0EA979EA2709
:101050003E88EBF67DB6ABCC864B6811B52E97D1AA
:1010600032A49678E6475186A7113D8D0EF06B2C81
:101070007BE6FBF81D7B2D3427C50CD4F7249EA1FD
:10108000058A5F4B6ABC89C6211A3BAC3A45747C21
:10109000DC52FB10B7EFD3BC22CF5B43D7B66EDF79
:1010A0005FC3D97D0E9E7A86539587C9CCFB673E78
:1010B000D6CF4E3FB51D0C8E8141C75D9C62B438C2
:1010C000C56F212C7E77FAA7970C1CBBF6E9A7D633
:1010D000E9BF93B838FD827E4A7120C5C9F36AD151
:1010E00065AB8658F5F43F596CB0F0B01EDEBD73A9
:1010F000DFDAA80695905E9BCC205A6130C3FC05D0
:1011000073DA0F706CD68DEAD816B6561B10B8F687
:101110007B74A22F1C51E1335A0A168E7861956AAE
:101120008C583A0644508E892BC1B0887FC3EE2973
:10113000058FB41D4AF53F89A1FD9519641A00F683
:10114000E97F805749A67F0ABE7D8E53FB081214A3
:10115000C2194707690CE96FB783B6BD62BBEB3FA5
:101160006D5DBABAD35DBBBA7B7C097FAEECE29F02
:101170001FEE1EEF74377607FC93FF19388F3AFF86
:1011800037FD2EACC3E4CBC9327EE24FE6C219ACC8
:10119000747BC41C78529CBB16A44FC10C350B0742
:1011A0000CB361B0BAC6ED36EC5691F9F0B5489A79
:1011B0009756E5D7C7EE27449F507B7F3DFB989419
:1011C000E77F31A24969FE1AD4CE2AF32FA07952C3
:1011D0007D9F42F17D80BED0669F43F97C79FA47BE
:1011E000D28052DF4AC5FA5BEEF31149DCE7F4F630
:1011F000EC7767BFC3C1DC9D4F039195FBDE54CFF5
:10120000C17781873B7172C77F4A28A81CB3172119
:101210000162CC870F437232EF4CE3249ECEA710BD
:1012200064469BFF94DB489C0524980CCD280186DE
:101230007C83B5A248556C8D06ADC814CCA7FF427F
:10124000682935FD33CB6E876D08025818A4F1BFAD
:101250000262608A90B5F02159121A59D44F90F465
:101260007F213944245D4110BDD1D6F0DBAE4BA6C1
:1012700010EC13AC3B7CF57569EFEE7891D76B02FF
:10128000E91509121EEFFA4F8929FDB59F5D5BFB39
:10129000C7DDF685758DD6BA04205B071A1B9082D0
:1012A000D34D24422893B946D4F947457B2059743D
:1012B0008690F88284C497D4CA561689EFE77404DE
:1012C00064A57D417620EC3B0B54FEFCEC9F88A886
:1012D0006D37FA0ED8339F07D3B87813FA38871AC8
:1012E000867A2743AE659F7E82E5B0AEB421A549DC
:1012F00078F61B02D5228B9340C47F00CEB45DD913
:10130000D024F2A84CD53FD32606B603D3416AD5E4
:10131000B53881FA2C1FB592D514BE737957D22CEB
:1013200069642861D95DF19DDB341B06342935429F
:101330004575E44EE0B199E67ADD0170B13FD3CE58
:101340006BF8074E6F19354BEF563B3BCAD3310450
:101350001C8207D18FEFBC733325455831753FF29E
:1013600054A4052FDF2E8AD9031923185080A5DE37
:10137000D4A3A66B08493D113FBE173C8689DAB25B
:10138000EFC46196E6E9B0E850DFEDEDFB304422B2
:10139000604924ADC0F5D926E1A8511F8D09194D2A
:1013A0008739F9F172BF9E367971A4573C2FEA70E4
:1013B00007F6E881798106EA3CCFDD4BDDAEE789AF
:1013C000416B7610DDCE6FA45986B5B97B3E83B8EC
:1013D00011DB70F85D5B4F06AFA9389C8974688596
:1013E000ABAB2109FDC9612B82CB0EACE629222DC6
:1013F0009374D4B26FB1A90B1312E0E6F07BCDE089
:10140000071B4DF7DFBBA90D3E69DC61711C1FABEB
:101410001878DB0B0C164A2A0F9C8181699BA7C2A6
:1014200048F2390633C4130ED20C7E571BA6C5FDF5
:101430007B0FB72B57146BF9D209BD0D7FBE18C7B0
:1014400039B0516DCF713710606342E229DF9DC121
:101450002615F7312191140736CAA3678F9A244FB6
:1014600098CE930291B864B18F7284CB1E2DE0C7E1
:101470009FC091014FFD1E8C41FE1B98DDB00658A8
:10148000D02EDA0B30979D1E4E07E143192A1CE837
:10149000693E21AE947E1D736035ABFDCDD7D287FA
:1014A0000C9B5FEDAD0A925CEDC39105F66010FBFD
:1014B0009396EE09C42A95020C06ABAB3E605DE93B
:1014C000E2904236EA81653AAF16ACE79EEAB04256
:1014D0001D40808A2FCA9ED2895C0785075B781FD2
:1014E000ACAD95485E838D09550C3C5751A4C00D99
:1014F0004E5C0A4056429D8C7219B0728E703E75D9
:101500001B9D0F575BFD14D4BC56204019C0B7A7D4
:10151000184EEE071311D96EF5D3A1D5C92F78D582
:10152000BE539F3C8757E98DF016E62E61C9C4343F
:101530007D22968153C1F0923E6AED17F432D014A9
:1015400027C354D9630DB70BB4CC58965CC83E97EB
:101550003E1EEC4CF32693FE94026365636498167A
:101560006A6A61AAD64BE41D20F401BD467A8FB4A5
:10157000E2D9AFD90AC748C3F5A98F0117C385813E
:10158000E7441A873D982FF11776081B6ACF5E3A19
:101590001E8ECCE9BF61C45FF03F525EF0A3C179FB
:1015A000886218238D60F47980BF9295DA300A1E24
:1015B0005964164CFF3FD805F07556FC6F64B44B68
:1015C0005D7A1BE4022EFF4E8C82E7707FF82CE4DC
:1015D000199E7D2C8D8226450E4062E474523BB1EB
:1015E000145B27AD6FA69891B4F8D1C37B77FF97B2
:1015F000B4B2FDD62D681DD6CCA4A85FA8934973BC
:10160000FBAEE82FEA66BFA19BA1998447BBA0A0CF
:101610004A2E60B8D79557D012A48021AB972A5C88
:101620004A58BD75BB94E46EA8C8126116C8418EB5
:10163000D741FB412487DED73E6598B23264F80B70
:10164000196164C34FEAB5CFC07A9F73FC810DD88E
:101650006506A1E30286204DBF2510CAD37BC6CE06
:10166000355C4198AC7F52E02C89B97C05A2C3C29D
:1016700073D6F1DF6EF7D8E11F208C2834A7CC5E3B
:10168000B284297EFA1C4D5F9C7DB034E6C3EB87A3
:10169000C8997CE7B661206D43930A919861FB8BF2
:1016A0008CC51EE562AC6EA531414EFE347F2090A4
:1016B0006ECAC76072CD2C36FDC8D384ED2ABB7DBF
:1016C000C72FC69DCC47DA710ACBBA54FD484F18D4
:1016D00049A215E49AE244EC0DFD7842BA5366A49F
:1016E00008D58D4EE9C11E65AE90A5E26E2A634510
:1016F0001D31EADA0D307CA5E56B99B96B371CF228
:10170000A33EB1CB8E66CEC9587E20F34FC817F5E5
:10171000ECEF5DBA748907DC7CC1CC37CD99B9E3B5
:10172000D79959E5EBCE075C7560E8FF198A8FE021
:10173000AF067D9DA5744AF0FCB5748FDA62BA914C
:1017400084A991A67B19CA90773C7F21BCA435BEA1
:10175000CFBB913D1B73C3F0D351F6A527022AA03E
:1017600094E6F94BA80ED532D588E652254D2D5D6D
:10177000A94A9A9EBF58D587D6FBEF4F6FA863D270
:10178000E9D605DC510EF6A5FBA304ED1E6568CF76
:101790005F98365576E363E3040B2F5F7BB700C198
:1017A000A462A5A5DBF6277E36AD2DEC77B8CD9DDE
:1017B00017E17DE27D4490F07399B38C374B5CE880
:1017C000A6EF8C5E0D6FDA65074A99E12EF40B9552
:1017D0000C80FE5A3559232DF79A28E9C23120256D
:1017E000A41D1CC44F29F640B152987D3002E12E51
:1017F0005114FB4B88F4DF6871CB915498761F9E8F
:101800003EEBC073387FB9ABF014E04B55A26F9A32
:10181000C7E289C872D304562E49E23F89473E7217
:10182000431D147764D746B074E1A3FA104B917846
:101830007A0FD9C33B0F6FDF42158752A36B280B7A
:1018400040F673C9A8CED42FC2716B7D3B8B234C5D
:10185000D2792D7BF2A8B7B1F1A8B3CE51D4958D32
:101860000A1C40CEC94AD80FA61CD6CDACA66AE841
:10187000820831121FD238078C651BC998661AA5D9
:10188000EC557F415D17722B65DFC61BEA5C2E822B
:10189000E87BD9AF6AAC7541B07DB1CB65EA523A0D
:1018A00040EC58107E392743AFD8EFD2CDA303398F
:1018B00021BB57BA913C1E6AAE3B7998841A5CFAF8
:1018C0004793E0122A46B725AD2735FC7E0B32340C
:1018D000C9ECE12C4EAEA71CE945B110150A25A3B1
:1018E0002A84C2F45E951640EBAAC4822A3A725C3E
:1018F0000E55A8C0AF170C82DED1896B73E9C45DA9
:101900005499408B58660FA435CCC74ED9D1B373C8
:10191000090898045088D9CB46521F0F9E19B27AF5
:10192000613CF527F9CB06E87E1EF26464D9864057
:1019300072B59FFCFAE1B63F229049F3CDE61087DD
:101940007D0A6BE80AA881849B5F55F868E45AD445
:1019500040891370061CB639E66392688237A8E1A5
:1019600081BBF4BA0A9D182A214996A0B03E907A0C
:10197000F490B47421388D020E9E9CC1A15A95EA50
:1019800009D55BDDDD067C8B80D49790B05573481C
:101990006E712416515CA5D3E10D6450B10C901802
:1019A000D5E07A71678A1D56A695DD86A3521F2D54
:1019B000D74464F0C56B8AFAA817764602D65C73E2
:1019C000ADB9A620D49664DAF66C44CB6B182BDF45
:1019D00001F8F2B7B7BC4BDB7E776663C197F7BB04
:1019E00049613B7950C8D7DE7A02E9FC4E0C9A87F0
:1019F000B2378ED3B5A72954C0C1588889EA8D7CE7
:101A000067341177A8F93D6A767776C9B27E85A9E1
:101A10006EDEBBC3C31E22A43BF9F6D3ED8B438E0F
:101A20003DCA9525587F270E6963AF0E132699C1CD
:101A3000F4CF6B9BC32CF7A9F16B4D3307E2F95040
:101A4000F2229D9D870EA47019A106E008416785CA
:101A5000BBB342F51B3C7EE138F4A0AFB5020C8E5F
:101A6000578007E9E1F3E04149E539F0E841AF0487
:101A70008FEEDC80E744591A39985A249D83382A1E
:101A8000C69B6FBCFE43983FD069B0244A53AF1E3B
:101A90007666170991B7F95A0CB30B9DD2249CC4F2
:101AA000E1BE57FA641CF93C7F028F332A8BF30F97
:101AB0005446A3270BC64E6455139757904786AAE2
:101AC000441A489E91AE4EA4E7D287294B15A9B57A
:101AD00072365CB805D4C2DE81AE60A486D28E3781
:101AE000CA19E58495B56D9637EA31A5994C1299D6
:101AF0008C5B7AA1AC5C5502492DDAF52CCB21B96F
:101B0000F1BA743A3114CB93F17EA3C82637A828D2
:101B10004C446EE9317AF6F786C3ABDDAB5D5BB55D
:101B2000FDE4D63BEFDC7B8F9ABB7E7445E8662EE6
:101B30006E44EBE5CB61D845E7250645AD4D171062
:101B400021DE590BA42F19C730B91B5DAD49EBE954
:101B50002A32C1CD8AA4E6840D7BBC319999E3E990
:101B60002BE3A433CBD222A5AC0E696CD6AA2641B6
:101B7000A9F8BEE18A33A3B2FA53CAEAC45D9C4A0B
:101B800069D96A26840B8C81A4593DFF9C810D186C
:101B900030D25649EFA69E2787C1E3F8C414F974E2
:101BA0009EBF992647540C7C2EF3E32F181E278DD9
:101BB000E12AA38EE1CC0D28A8DDF207F69A0D7B71
:101BC000A0AFD6F4032A3256F60E43314B0F5A1B00
:101BD0005D293A3420DA3472F4B00CD915D494BFAC
:101BE00016CAC251329722AFE5AFF9DF0F9DF5104B
:101BF000B97EDB6EE3378AAF65D267B3B62F3D5D42
